 windowsaccessbridge-32

 Timestamp is ffffffff (Sun Feb  7 06:28:15 2106)

 Preferred load address is 10000000

 Start         Length     Name                   Class
 0001:00000000 0001b6ebH .text$mn                CODE
 0001:0001b6eb 000000b9H .text$x                 CODE
 0002:00000000 0000015cH .idata$5                DATA
 0002:0000015c 00000004H .00cfg                  DATA
 0002:00000160 00000004H .CRT$XCA                DATA
 0002:00000164 00000004H .CRT$XCZ                DATA
 0002:00000168 00000004H .CRT$XIA                DATA
 0002:0000016c 00000010H .CRT$XIC                DATA
 0002:0000017c 00000004H .CRT$XIZ                DATA
 0002:00000180 00000004H .CRT$XPA                DATA
 0002:00000184 00000008H .CRT$XPX                DATA
 0002:0000018c 00000004H .CRT$XPXA               DATA
 0002:00000190 00000004H .CRT$XPZ                DATA
 0002:00000194 00000004H .CRT$XTA                DATA
 0002:00000198 00000008H .CRT$XTZ                DATA
 0002:0000019c 00000000H .gfids$y                DATA
 0002:000001a0 000089a0H .rdata                  DATA
 0002:00008b40 00000180H .rdata$r                DATA
 0002:00008cc0 0000002cH .rdata$sxdata           DATA
 0002:00008cec 00000304H .rdata$zzzdbg           DATA
 0002:00008ff0 00000004H .rtc$IAA                DATA
 0002:00008ff4 00000004H .rtc$IZZ                DATA
 0002:00008ff8 00000004H .rtc$TAA                DATA
 0002:00008ffc 00000004H .rtc$TZZ                DATA
 0002:00009000 00000720H .xdata$x                DATA
 0002:00009720 00000e44H .edata                  DATA
 0002:0000a564 00000028H .idata$2                DATA
 0002:0000a58c 00000014H .idata$3                DATA
 0002:0000a5a0 0000015cH .idata$4                DATA
 0002:0000a6fc 0000063aH .idata$6                DATA
 0003:00000000 000008d0H .data                   DATA
 0003:000008d0 00000098H .data$r                 DATA
 0003:00000968 00000a7cH .bss                    DATA
 0004:00000000 00000120H .rsrc$01                DATA
 0004:00000120 00000638H .rsrc$02                DATA

  Address         Publics by Value              Rva+Base       Lib:Object

 0000:00000000       ___guard_fids_count        00000000     <absolute>
 0000:00000000       ___hybrid_code_map_count   00000000     <absolute>
 0000:00000000       ___guard_iat_count         00000000     <absolute>
 0000:00000000       ___dynamic_value_reloc_table 00000000     <absolute>
 0000:00000000       ___guard_longjmp_count     00000000     <absolute>
 0000:00000000       __except_list              00000000     <absolute>
 0000:00000000       ___guard_fids_table        00000000     <absolute>
 0000:00000000       ___guard_longjmp_table     00000000     <absolute>
 0000:00000000       ___hybrid_auxiliary_iat    00000000     <absolute>
 0000:00000000       ___guard_iat_table         00000000     <absolute>
 0000:00000000       ___volatile_metadata       00000000     <absolute>
 0000:00000000       ___enclave_config          00000000     <absolute>
 0000:00000000       ___hybrid_code_map         00000000     <absolute>
 0000:0000000b       ___safe_se_handler_count   0000000b     <absolute>
 0000:00000100       ___guard_flags             00000100     <absolute>
 0000:00000000       ___ImageBase               10000000     <linker-defined>
 0001:00000000       _PrintDebugString          10001000 f   AccessBridgeDebug.obj
 0001:0000004a       ___local_stdio_printf_options 1000104a f i AccessBridgeDebug.obj
 0001:00000050       __vfprintf_l               10001050 f i AccessBridgeDebug.obj
 0001:00000073       _finalizeFileLogger        10001073 f   AccessBridgeDebug.obj
 0001:0000008b       _fprintf                   1000108b f i AccessBridgeDebug.obj
 0001:000000a3       _getTimeStamp              100010a3 f   AccessBridgeDebug.obj
 0001:000000d1       _initializeFileLogger      100010d1 f   AccessBridgeDebug.obj
 0001:00000191       _printf                    10001191 f i AccessBridgeDebug.obj
 0001:000001ae       ??0AccessBridgeEventHandler@@QAE@XZ 100011ae f   AccessBridgeEventHandler.obj
 0001:00000209       @_guard_check_icall_nop@4  10001209 f   LIBCMT:guard_support.obj
 0001:00000209       ??1AccessBridgeEventHandler@@QAE@XZ 10001209 f   AccessBridgeEventHandler.obj
 0001:00000209       ??1AccessBridgeMessageQueue@@QAE@XZ 10001209 f   AccessBridgeMessageQueue.obj
 0001:0000020a       ?fireCaretUpdate@AccessBridgeEventHandler@@QAEXJ_J0@Z 1000120a f   AccessBridgeEventHandler.obj
 0001:0000022c       ?fireFocusGained@AccessBridgeEventHandler@@QAEXJ_J0@Z 1000122c f   AccessBridgeEventHandler.obj
 0001:0000024e       ?fireFocusLost@AccessBridgeEventHandler@@QAEXJ_J0@Z 1000124e f   AccessBridgeEventHandler.obj
 0001:00000270       ?fireJavaShutdown@AccessBridgeEventHandler@@QAEXJ@Z 10001270 f   AccessBridgeEventHandler.obj
 0001:00000281       ?fireMenuCanceled@AccessBridgeEventHandler@@QAEXJ_J0@Z 10001281 f   AccessBridgeEventHandler.obj
 0001:000002a3       ?fireMenuDeselected@AccessBridgeEventHandler@@QAEXJ_J0@Z 100012a3 f   AccessBridgeEventHandler.obj
 0001:000002c5       ?fireMenuSelected@AccessBridgeEventHandler@@QAEXJ_J0@Z 100012c5 f   AccessBridgeEventHandler.obj
 0001:000002e7       ?fireMouseClicked@AccessBridgeEventHandler@@QAEXJ_J0@Z 100012e7 f   AccessBridgeEventHandler.obj
 0001:00000309       ?fireMouseEntered@AccessBridgeEventHandler@@QAEXJ_J0@Z 10001309 f   AccessBridgeEventHandler.obj
 0001:0000032b       ?fireMouseExited@AccessBridgeEventHandler@@QAEXJ_J0@Z 1000132b f   AccessBridgeEventHandler.obj
 0001:0000034d       ?fireMousePressed@AccessBridgeEventHandler@@QAEXJ_J0@Z 1000134d f   AccessBridgeEventHandler.obj
 0001:0000036f       ?fireMouseReleased@AccessBridgeEventHandler@@QAEXJ_J0@Z 1000136f f   AccessBridgeEventHandler.obj
 0001:00000391       ?firePopupMenuCanceled@AccessBridgeEventHandler@@QAEXJ_J0@Z 10001391 f   AccessBridgeEventHandler.obj
 0001:000003b3       ?firePopupMenuWillBecomeInvisible@AccessBridgeEventHandler@@QAEXJ_J0@Z 100013b3 f   AccessBridgeEventHandler.obj
 0001:000003d5       ?firePopupMenuWillBecomeVisible@AccessBridgeEventHandler@@QAEXJ_J0@Z 100013d5 f   AccessBridgeEventHandler.obj
 0001:000003f7       ?firePropertyActiveDescendentChange@AccessBridgeEventHandler@@QAEXJ_J000@Z 100013f7 f   AccessBridgeEventHandler.obj
 0001:00000425       ?firePropertyCaretChange@AccessBridgeEventHandler@@QAEXJ_J0HH@Z 10001425 f   AccessBridgeEventHandler.obj
 0001:0000044d       ?firePropertyChildChange@AccessBridgeEventHandler@@QAEXJ_J000@Z 1000144d f   AccessBridgeEventHandler.obj
 0001:0000047b       ?firePropertyDescriptionChange@AccessBridgeEventHandler@@QAEXJ_J0PAG1@Z 1000147b f   AccessBridgeEventHandler.obj
 0001:000004a3       ?firePropertyNameChange@AccessBridgeEventHandler@@QAEXJ_J0PAG1@Z 100014a3 f   AccessBridgeEventHandler.obj
 0001:000004cb       ?firePropertySelectionChange@AccessBridgeEventHandler@@QAEXJ_J0@Z 100014cb f   AccessBridgeEventHandler.obj
 0001:000004ed       ?firePropertyStateChange@AccessBridgeEventHandler@@QAEXJ_J0PAG1@Z 100014ed f   AccessBridgeEventHandler.obj
 0001:00000515       ?firePropertyTableModelChange@AccessBridgeEventHandler@@QAEXJ_J0PAG1@Z 10001515 f   AccessBridgeEventHandler.obj
 0001:0000053d       ?firePropertyTextChange@AccessBridgeEventHandler@@QAEXJ_J0@Z 1000153d f   AccessBridgeEventHandler.obj
 0001:0000055f       ?firePropertyValueChange@AccessBridgeEventHandler@@QAEXJ_J0PAG1@Z 1000155f f   AccessBridgeEventHandler.obj
 0001:00000587       ?firePropertyVisibleDataChange@AccessBridgeEventHandler@@QAEXJ_J0@Z 10001587 f   AccessBridgeEventHandler.obj
 0001:000005a9       ?setCaretUpdateFP@AccessBridgeEventHandler@@QAEXP6AXJ_J0@ZPAVWinAccessBridge@@@Z 100015a9 f   AccessBridgeEventHandler.obj
 0001:000005db       ?setFocusGainedFP@AccessBridgeEventHandler@@QAEXP6AXJ_J0@ZPAVWinAccessBridge@@@Z 100015db f   AccessBridgeEventHandler.obj
 0001:0000060d       ?setFocusLostFP@AccessBridgeEventHandler@@QAEXP6AXJ_J0@ZPAVWinAccessBridge@@@Z 1000160d f   AccessBridgeEventHandler.obj
 0001:0000063f       ?setJavaShutdownFP@AccessBridgeEventHandler@@QAEXP6AXJ@ZPAVWinAccessBridge@@@Z 1000163f f   AccessBridgeEventHandler.obj
 0001:0000067c       ?setMenuCanceledFP@AccessBridgeEventHandler@@QAEXP6AXJ_J0@ZPAVWinAccessBridge@@@Z 1000167c f   AccessBridgeEventHandler.obj
 0001:000006b9       ?setMenuDeselectedFP@AccessBridgeEventHandler@@QAEXP6AXJ_J0@ZPAVWinAccessBridge@@@Z 100016b9 f   AccessBridgeEventHandler.obj
 0001:000006f6       ?setMenuSelectedFP@AccessBridgeEventHandler@@QAEXP6AXJ_J0@ZPAVWinAccessBridge@@@Z 100016f6 f   AccessBridgeEventHandler.obj
 0001:00000733       ?setMouseClickedFP@AccessBridgeEventHandler@@QAEXP6AXJ_J0@ZPAVWinAccessBridge@@@Z 10001733 f   AccessBridgeEventHandler.obj
 0001:00000765       ?setMouseEnteredFP@AccessBridgeEventHandler@@QAEXP6AXJ_J0@ZPAVWinAccessBridge@@@Z 10001765 f   AccessBridgeEventHandler.obj
 0001:00000797       ?setMouseExitedFP@AccessBridgeEventHandler@@QAEXP6AXJ_J0@ZPAVWinAccessBridge@@@Z 10001797 f   AccessBridgeEventHandler.obj
 0001:000007c9       ?setMousePressedFP@AccessBridgeEventHandler@@QAEXP6AXJ_J0@ZPAVWinAccessBridge@@@Z 100017c9 f   AccessBridgeEventHandler.obj
 0001:00000806       ?setMouseReleasedFP@AccessBridgeEventHandler@@QAEXP6AXJ_J0@ZPAVWinAccessBridge@@@Z 10001806 f   AccessBridgeEventHandler.obj
 0001:00000843       ?setPopupMenuCanceledFP@AccessBridgeEventHandler@@QAEXP6AXJ_J0@ZPAVWinAccessBridge@@@Z 10001843 f   AccessBridgeEventHandler.obj
 0001:00000880       ?setPopupMenuWillBecomeInvisibleFP@AccessBridgeEventHandler@@QAEXP6AXJ_J0@ZPAVWinAccessBridge@@@Z 10001880 f   AccessBridgeEventHandler.obj
 0001:000008bd       ?setPopupMenuWillBecomeVisibleFP@AccessBridgeEventHandler@@QAEXP6AXJ_J0@ZPAVWinAccessBridge@@@Z 100018bd f   AccessBridgeEventHandler.obj
 0001:000008fa       ?setPropertyActiveDescendentChangeFP@AccessBridgeEventHandler@@QAEXP6AXJ_J000@ZPAVWinAccessBridge@@@Z 100018fa f   AccessBridgeEventHandler.obj
 0001:0000093a       ?setPropertyCaretChangeFP@AccessBridgeEventHandler@@QAEXP6AXJ_J0HH@ZPAVWinAccessBridge@@@Z 1000193a f   AccessBridgeEventHandler.obj
 0001:0000096f       ?setPropertyChangeFP@AccessBridgeEventHandler@@QAEXP6AXJ_J0PAG11@ZPAVWinAccessBridge@@@Z 1000196f f   AccessBridgeEventHandler.obj
 0001:000009a1       ?setPropertyChildChangeFP@AccessBridgeEventHandler@@QAEXP6AXJ_J000@ZPAVWinAccessBridge@@@Z 100019a1 f   AccessBridgeEventHandler.obj
 0001:000009e1       ?setPropertyDescriptionChangeFP@AccessBridgeEventHandler@@QAEXP6AXJ_J0PAG1@ZPAVWinAccessBridge@@@Z 100019e1 f   AccessBridgeEventHandler.obj
 0001:00000a16       ?setPropertyNameChangeFP@AccessBridgeEventHandler@@QAEXP6AXJ_J0PAG1@ZPAVWinAccessBridge@@@Z 10001a16 f   AccessBridgeEventHandler.obj
 0001:00000a4b       ?setPropertySelectionChangeFP@AccessBridgeEventHandler@@QAEXP6AXJ_J0@ZPAVWinAccessBridge@@@Z 10001a4b f   AccessBridgeEventHandler.obj
 0001:00000a80       ?setPropertyStateChangeFP@AccessBridgeEventHandler@@QAEXP6AXJ_J0PAG1@ZPAVWinAccessBridge@@@Z 10001a80 f   AccessBridgeEventHandler.obj
 0001:00000ab5       ?setPropertyTableModelChangeFP@AccessBridgeEventHandler@@QAEXP6AXJ_J0PAG1@ZPAVWinAccessBridge@@@Z 10001ab5 f   AccessBridgeEventHandler.obj
 0001:00000af5       ?setPropertyTextChangeFP@AccessBridgeEventHandler@@QAEXP6AXJ_J0@ZPAVWinAccessBridge@@@Z 10001af5 f   AccessBridgeEventHandler.obj
 0001:00000b2a       ?setPropertyValueChangeFP@AccessBridgeEventHandler@@QAEXP6AXJ_J0PAG1@ZPAVWinAccessBridge@@@Z 10001b2a f   AccessBridgeEventHandler.obj
 0001:00000b5f       ?setPropertyVisibleDataChangeFP@AccessBridgeEventHandler@@QAEXP6AXJ_J0@ZPAVWinAccessBridge@@@Z 10001b5f f   AccessBridgeEventHandler.obj
 0001:00000b9f       ??0AccessBridgeJavaVMInstance@@QAE@PAUHWND__@@0JPAV0@@Z 10001b9f f   AccessBridgeJavaVMInstance.obj
 0001:00000be6       ??1AccessBridgeJavaVMInstance@@QAE@XZ 10001be6 f   AccessBridgeJavaVMInstance.obj
 0001:00000c30       ?findABJavaVMInstanceFromJavaHWND@AccessBridgeJavaVMInstance@@QAEPAV1@PAUHWND__@@@Z 10001c30 f   AccessBridgeJavaVMInstance.obj
 0001:00000c6c       ?findAccessBridgeWindow@AccessBridgeJavaVMInstance@@QAEPAUHWND__@@J@Z 10001c6c f   AccessBridgeJavaVMInstance.obj
 0001:00000cb3       ?initiateIPC@AccessBridgeJavaVMInstance@@QAEJXZ 10001cb3 f   AccessBridgeJavaVMInstance.obj
 0001:00000d71       ?sendMemoryPackage@AccessBridgeJavaVMInstance@@QAEHPADJ@Z 10001d71 f   AccessBridgeJavaVMInstance.obj
 0001:00000e35       ?sendPackage@AccessBridgeJavaVMInstance@@QAEJPADJ@Z 10001e35 f   AccessBridgeJavaVMInstance.obj
 0001:00000e8a       __vsnprintf_l              10001e8a f i AccessBridgeJavaVMInstance.obj
 0001:00000ebc       _sprintf                   10001ebc f i AccessBridgeJavaVMInstance.obj
 0001:00000ed6       ??0AccessBridgeMessageQueue@@QAE@XZ 10001ed6 f   AccessBridgeMessageQueue.obj
 0001:00000ee9       ??0AccessBridgeQueueElement@@QAE@PADH@Z 10001ee9 f   AccessBridgeMessageQueue.obj
 0001:00000f3a       ??0bad_alloc@std@@QAE@ABV01@@Z 10001f3a f i AccessBridgeMessageQueue.obj
 0001:00000f52       ??0bad_alloc@std@@QAE@XZ   10001f52 f i AccessBridgeMessageQueue.obj
 0001:00000f6a       ??0exception@std@@QAE@ABV01@@Z 10001f6a f i AccessBridgeMessageQueue.obj
 0001:00000f93       ??1AccessBridgeQueueElement@@QAE@XZ 10001f93 f   AccessBridgeMessageQueue.obj
 0001:00000f9c       ??1bad_alloc@std@@UAE@XZ   10001f9c f i AccessBridgeMessageQueue.obj
 0001:00000f9c       ??1bad_exception@std@@UAE@XZ 10001f9c f i libvcruntime:frame.obj
 0001:00000f9c       ??1bad_array_new_length@std@@UAE@XZ 10001f9c f i LIBCMT:throw_bad_alloc.obj
 0001:00000fad       ??_Ebad_alloc@std@@UAEPAXI@Z 10001fad f i AccessBridgeMessageQueue.obj
 0001:00000fad       ??_Gbad_alloc@std@@UAEPAXI@Z 10001fad f i AccessBridgeMessageQueue.obj
 0001:00000fad       ??_Eexception@std@@UAEPAXI@Z 10001fad f i AccessBridgeMessageQueue.obj
 0001:00000fad       ??_Gexception@std@@UAEPAXI@Z 10001fad f i AccessBridgeMessageQueue.obj
 0001:00000fd7       ?add@AccessBridgeMessageQueue@@QAE?AW4QueueReturns@@PAVAccessBridgeQueueElement@@@Z 10001fd7 f   AccessBridgeMessageQueue.obj
 0001:00001073       ?getEventsWaiting@AccessBridgeMessageQueue@@QAEHXZ 10002073 f   AccessBridgeMessageQueue.obj
 0001:00001077       ?getRemoveLockSetting@AccessBridgeMessageQueue@@QAEHXZ 10002077 f   AccessBridgeMessageQueue.obj
 0001:0000107b       ?remove@AccessBridgeMessageQueue@@QAE?AW4QueueReturns@@PAPAVAccessBridgeQueueElement@@@Z 1000207b f   AccessBridgeMessageQueue.obj
 0001:00001116       ?setRemoveLock@AccessBridgeMessageQueue@@QAE?AW4QueueReturns@@H@Z 10002116 f   AccessBridgeMessageQueue.obj
 0001:0000112c       ?what@exception@std@@UBEPBDXZ 1000212c f i AccessBridgeMessageQueue.obj
 0001:0000113a       ?initBroadcastMessageIDs@@YAHXZ 1000213a f   AccessBridgeMessages.obj
 0001:0000116c       _Windows_run               1000216c f   AccessBridgeWindowsEntryPoints.obj
 0001:0000117b       _activateAccessibleHyperlink 1000217b f   AccessBridgeWindowsEntryPoints.obj
 0001:000011a2       _addAccessibleSelectionFromContext 100021a2 f   AccessBridgeWindowsEntryPoints.obj
 0001:000011c2       _clearAccessibleSelectionFromContext 100021c2 f   AccessBridgeWindowsEntryPoints.obj
 0001:000011de       _doAccessibleActions       100021de f   AccessBridgeWindowsEntryPoints.obj
 0001:00001205       _getAccessibleActions      10002205 f   AccessBridgeWindowsEntryPoints.obj
 0001:00001228       _getAccessibleChildFromContext 10002228 f   AccessBridgeWindowsEntryPoints.obj
 0001:0000124d       _getAccessibleContextAt    1000224d f   AccessBridgeWindowsEntryPoints.obj
 0001:00001277       _getAccessibleContextFromHWND 10002277 f   AccessBridgeWindowsEntryPoints.obj
 0001:00001296       _getAccessibleContextInfo  10002296 f   AccessBridgeWindowsEntryPoints.obj
 0001:000012b9       _getAccessibleContextWithFocus 100022b9 f   AccessBridgeWindowsEntryPoints.obj
 0001:000012d8       _getAccessibleHyperlink    100022d8 f   AccessBridgeWindowsEntryPoints.obj
 0001:000012ff       _getAccessibleHyperlinkCount 100022ff f   AccessBridgeWindowsEntryPoints.obj
 0001:0000131f       _getAccessibleHypertext    1000231f f   AccessBridgeWindowsEntryPoints.obj
 0001:00001342       _getAccessibleHypertextExt 10002342 f   AccessBridgeWindowsEntryPoints.obj
 0001:00001369       _getAccessibleHypertextLinkIndex 10002369 f   AccessBridgeWindowsEntryPoints.obj
 0001:0000138d       _getAccessibleIcons        1000238d f   AccessBridgeWindowsEntryPoints.obj
 0001:000013b0       _getAccessibleKeyBindings  100023b0 f   AccessBridgeWindowsEntryPoints.obj
 0001:000013d3       _getAccessibleParentFromContext 100023d3 f   AccessBridgeWindowsEntryPoints.obj
 0001:000013f4       _getAccessibleRelationSet  100023f4 f   AccessBridgeWindowsEntryPoints.obj
 0001:00001417       _getAccessibleSelectionCountFromContext 10002417 f   AccessBridgeWindowsEntryPoints.obj
 0001:00001437       _getAccessibleSelectionFromContext 10002437 f   AccessBridgeWindowsEntryPoints.obj
 0001:0000145c       _getAccessibleTableCellInfo 1000245c f   AccessBridgeWindowsEntryPoints.obj
 0001:00001486       _getAccessibleTableColumn  10002486 f   AccessBridgeWindowsEntryPoints.obj
 0001:000014aa       _getAccessibleTableColumnDescription 100024aa f   AccessBridgeWindowsEntryPoints.obj
 0001:000014cf       _getAccessibleTableColumnHeader 100024cf f   AccessBridgeWindowsEntryPoints.obj
 0001:000014f2       _getAccessibleTableColumnSelectionCount 100024f2 f   AccessBridgeWindowsEntryPoints.obj
 0001:00001512       _getAccessibleTableColumnSelections 10002512 f   AccessBridgeWindowsEntryPoints.obj
 0001:00001539       _getAccessibleTableIndex   10002539 f   AccessBridgeWindowsEntryPoints.obj
 0001:00001561       _getAccessibleTableInfo    10002561 f   AccessBridgeWindowsEntryPoints.obj
 0001:00001584       _getAccessibleTableRow     10002584 f   AccessBridgeWindowsEntryPoints.obj
 0001:000015a8       _getAccessibleTableRowDescription 100025a8 f   AccessBridgeWindowsEntryPoints.obj
 0001:000015cd       _getAccessibleTableRowHeader 100025cd f   AccessBridgeWindowsEntryPoints.obj
 0001:000015f0       _getAccessibleTableRowSelectionCount 100025f0 f   AccessBridgeWindowsEntryPoints.obj
 0001:00001610       _getAccessibleTableRowSelections 10002610 f   AccessBridgeWindowsEntryPoints.obj
 0001:00001637       _getAccessibleTextAttributes 10002637 f   AccessBridgeWindowsEntryPoints.obj
 0001:0000165e       _getAccessibleTextInfo     1000265e f   AccessBridgeWindowsEntryPoints.obj
 0001:00001688       _getAccessibleTextItems    10002688 f   AccessBridgeWindowsEntryPoints.obj
 0001:000016af       _getAccessibleTextLineBounds 100026af f   AccessBridgeWindowsEntryPoints.obj
 0001:000016d9       _getAccessibleTextRange    100026d9 f   AccessBridgeWindowsEntryPoints.obj
 0001:00001706       _getAccessibleTextRect     10002706 f   AccessBridgeWindowsEntryPoints.obj
 0001:0000172d       _getAccessibleTextSelectionInfo 1000272d f   AccessBridgeWindowsEntryPoints.obj
 0001:00001750       _getActiveDescendent       10002750 f   AccessBridgeWindowsEntryPoints.obj
 0001:00001771       _getCaretLocation          10002771 f   AccessBridgeWindowsEntryPoints.obj
 0001:00001798       _getCurrentAccessibleValueFromContext 10002798 f   AccessBridgeWindowsEntryPoints.obj
 0001:000017bf       _getEventsWaiting          100027bf f   AccessBridgeWindowsEntryPoints.obj
 0001:000017d0       _getHWNDFromAccessibleContext 100027d0 f   AccessBridgeWindowsEntryPoints.obj
 0001:000017ef       _getMaximumAccessibleValueFromContext 100027ef f   AccessBridgeWindowsEntryPoints.obj
 0001:00001816       _getMinimumAccessibleValueFromContext 10002816 f   AccessBridgeWindowsEntryPoints.obj
 0001:0000183d       _getObjectDepth            1000283d f   AccessBridgeWindowsEntryPoints.obj
 0001:0000185d       _getParentWithRole         1000285d f   AccessBridgeWindowsEntryPoints.obj
 0001:00001882       _getParentWithRoleElseRoot 10002882 f   AccessBridgeWindowsEntryPoints.obj
 0001:000018a7       _getTextAttributesInRange  100028a7 f   AccessBridgeWindowsEntryPoints.obj
 0001:000018d4       _getTopLevelHWND           100028d4 f   AccessBridgeWindowsEntryPoints.obj
 0001:00001918       _getTopLevelObject         10002918 f   AccessBridgeWindowsEntryPoints.obj
 0001:00001939       _getVersionInfo            10002939 f   AccessBridgeWindowsEntryPoints.obj
 0001:00001951       _getVirtualAccessibleName  10002951 f   AccessBridgeWindowsEntryPoints.obj
 0001:00001978       _getVisibleChildren        10002978 f   AccessBridgeWindowsEntryPoints.obj
 0001:0000199f       _getVisibleChildrenCount   1000299f f   AccessBridgeWindowsEntryPoints.obj
 0001:000019be       _isAccessibleChildSelectedFromContext 100029be f   AccessBridgeWindowsEntryPoints.obj
 0001:000019e1       _isAccessibleTableColumnSelected 100029e1 f   AccessBridgeWindowsEntryPoints.obj
 0001:00001a04       _isAccessibleTableRowSelected 10002a04 f   AccessBridgeWindowsEntryPoints.obj
 0001:00001a27       _isJavaWindow              10002a27 f   AccessBridgeWindowsEntryPoints.obj
 0001:00001a3e       _isSameObject              10002a3e f   AccessBridgeWindowsEntryPoints.obj
 0001:00001a7e       _releaseJavaObject         10002a7e f   AccessBridgeWindowsEntryPoints.obj
 0001:00001a9a       _removeAccessibleSelectionFromContext 10002a9a f   AccessBridgeWindowsEntryPoints.obj
 0001:00001aba       _requestFocus              10002aba f   AccessBridgeWindowsEntryPoints.obj
 0001:00001ad9       _selectAllAccessibleSelectionFromContext 10002ad9 f   AccessBridgeWindowsEntryPoints.obj
 0001:00001af5       _selectTextRange           10002af5 f   AccessBridgeWindowsEntryPoints.obj
 0001:00001b1c       _setCaretPosition          10002b1c f   AccessBridgeWindowsEntryPoints.obj
 0001:00001b3f       _setCaretUpdateFP          10002b3f f   AccessBridgeWindowsEntryPoints.obj
 0001:00001b53       _setFocusGainedFP          10002b53 f   AccessBridgeWindowsEntryPoints.obj
 0001:00001b67       _setFocusLostFP            10002b67 f   AccessBridgeWindowsEntryPoints.obj
 0001:00001b7b       _setJavaShutdownFP         10002b7b f   AccessBridgeWindowsEntryPoints.obj
 0001:00001b8f       _setMenuCanceledFP         10002b8f f   AccessBridgeWindowsEntryPoints.obj
 0001:00001ba3       _setMenuDeselectedFP       10002ba3 f   AccessBridgeWindowsEntryPoints.obj
 0001:00001bb7       _setMenuSelectedFP         10002bb7 f   AccessBridgeWindowsEntryPoints.obj
 0001:00001bcb       _setMouseClickedFP         10002bcb f   AccessBridgeWindowsEntryPoints.obj
 0001:00001bdf       _setMouseEnteredFP         10002bdf f   AccessBridgeWindowsEntryPoints.obj
 0001:00001bf3       _setMouseExitedFP          10002bf3 f   AccessBridgeWindowsEntryPoints.obj
 0001:00001c07       _setMousePressedFP         10002c07 f   AccessBridgeWindowsEntryPoints.obj
 0001:00001c1b       _setMouseReleasedFP        10002c1b f   AccessBridgeWindowsEntryPoints.obj
 0001:00001c2f       _setPopupMenuCanceledFP    10002c2f f   AccessBridgeWindowsEntryPoints.obj
 0001:00001c43       _setPopupMenuWillBecomeInvisibleFP 10002c43 f   AccessBridgeWindowsEntryPoints.obj
 0001:00001c57       _setPopupMenuWillBecomeVisibleFP 10002c57 f   AccessBridgeWindowsEntryPoints.obj
 0001:00001c6b       _setPropertyActiveDescendentChangeFP 10002c6b f   AccessBridgeWindowsEntryPoints.obj
 0001:00001c7f       _setPropertyCaretChangeFP  10002c7f f   AccessBridgeWindowsEntryPoints.obj
 0001:00001c93       _setPropertyChangeFP       10002c93 f   AccessBridgeWindowsEntryPoints.obj
 0001:00001ca7       _setPropertyChildChangeFP  10002ca7 f   AccessBridgeWindowsEntryPoints.obj
 0001:00001cbb       _setPropertyDescriptionChangeFP 10002cbb f   AccessBridgeWindowsEntryPoints.obj
 0001:00001ccf       _setPropertyNameChangeFP   10002ccf f   AccessBridgeWindowsEntryPoints.obj
 0001:00001ce3       _setPropertySelectionChangeFP 10002ce3 f   AccessBridgeWindowsEntryPoints.obj
 0001:00001cf7       _setPropertyStateChangeFP  10002cf7 f   AccessBridgeWindowsEntryPoints.obj
 0001:00001d0b       _setPropertyTableModelChangeFP 10002d0b f   AccessBridgeWindowsEntryPoints.obj
 0001:00001d1f       _setPropertyTextChangeFP   10002d1f f   AccessBridgeWindowsEntryPoints.obj
 0001:00001d33       _setPropertyValueChangeFP  10002d33 f   AccessBridgeWindowsEntryPoints.obj
 0001:00001d47       _setPropertyVisibleDataChangeFP 10002d47 f   AccessBridgeWindowsEntryPoints.obj
 0001:00001d5b       _setTextContents           10002d5b f   AccessBridgeWindowsEntryPoints.obj
 0001:00001d7e       ??0WinAccessBridge@@QAE@PAUHINSTANCE__@@@Z 10002d7e f   WinAccessBridge.obj
 0001:00001dfc       ??1WinAccessBridge@@QAE@XZ 10002dfc f   WinAccessBridge.obj
 0001:00001eb9       ?JavaVMDestroyed@WinAccessBridge@@QAEXPAUHWND__@@@Z 10002eb9 f   WinAccessBridge.obj
 0001:00001f53       ?activateAccessibleHyperlink@WinAccessBridge@@QAEHJ_J0@Z 10002f53 f   WinAccessBridge.obj
 0001:00001ff9       ?addAccessibilityEventNotification@WinAccessBridge@@QAEX_J@Z 10002ff9 f   WinAccessBridge.obj
 0001:00002085       ?addAccessibleSelectionFromContext@WinAccessBridge@@QAEXJ_JH@Z 10003085 f   WinAccessBridge.obj
 0001:000020e5       ?addJavaEventNotification@WinAccessBridge@@QAEX_J@Z 100030e5 f   WinAccessBridge.obj
 0001:00002171       ?clearAccessibleSelectionFromContext@WinAccessBridge@@QAEXJ_J@Z 10003171 f   WinAccessBridge.obj
 0001:000021cb       ?doAccessibleActions@WinAccessBridge@@QAEHJ_JPAUAccessibleActionsToDoTag@@PAJ@Z 100031cb f   WinAccessBridge.obj
 0001:000022b9       ?getAccessibleActions@WinAccessBridge@@QAEHJ_JPAUAccessibleActionsTag@@@Z 100032b9 f   WinAccessBridge.obj
 0001:0000239c       ?getAccessibleChildFromContext@WinAccessBridge@@QAE_JJ_JJ@Z 1000339c f   WinAccessBridge.obj
 0001:00002422       ?getAccessibleContextAt@WinAccessBridge@@QAEHJ_JJJPA_J@Z 10003422 f   WinAccessBridge.obj
 0001:000024c8       ?getAccessibleContextFromHWND@WinAccessBridge@@QAEHPAUHWND__@@PAJPA_J@Z 100034c8 f   WinAccessBridge.obj
 0001:000025c3       ?getAccessibleContextInfo@WinAccessBridge@@QAEHJ_JPAUAccessibleContextInfoTag@@@Z 100035c3 f   WinAccessBridge.obj
 0001:000026a2       ?getAccessibleContextWithFocus@WinAccessBridge@@QAEHPAUHWND__@@PAJPA_J@Z 100036a2 f   WinAccessBridge.obj
 0001:00002742       ?getAccessibleHyperlink@WinAccessBridge@@QAEHJ_JJPAUAccessibleHyperlinkInfoTag@@@Z 10003742 f   WinAccessBridge.obj
 0001:00002820       ?getAccessibleHyperlinkCount@WinAccessBridge@@QAEJJ_J@Z 10003820 f   WinAccessBridge.obj
 0001:000028d1       ?getAccessibleHypertext@WinAccessBridge@@QAEHJ_JPAUAccessibleHypertextInfoTag@@@Z 100038d1 f   WinAccessBridge.obj
 0001:000029b4       ?getAccessibleHypertextExt@WinAccessBridge@@QAEHJ_JJPAUAccessibleHypertextInfoTag@@@Z 100039b4 f   WinAccessBridge.obj
 0001:00002ac9       ?getAccessibleHypertextLinkIndex@WinAccessBridge@@QAEJJ_JJ@Z 10003ac9 f   WinAccessBridge.obj
 0001:00002b82       ?getAccessibleIcons@WinAccessBridge@@QAEHJ_JPAUAccessibleIconsTag@@@Z 10003b82 f   WinAccessBridge.obj
 0001:00002c65       ?getAccessibleKeyBindings@WinAccessBridge@@QAEHJ_JPAUAccessibleKeyBindingsTag@@@Z 10003c65 f   WinAccessBridge.obj
 0001:00002d5e       ?getAccessibleParentFromContext@WinAccessBridge@@QAE_JJ_J@Z 10003d5e f   WinAccessBridge.obj
 0001:00002ddd       ?getAccessibleRelationSet@WinAccessBridge@@QAEHJ_JPAUAccessibleRelationSetInfoTag@@@Z 10003ddd f   WinAccessBridge.obj
 0001:00002ebe       ?getAccessibleSelectionCountFromContext@WinAccessBridge@@QAEHJ_J@Z 10003ebe f   WinAccessBridge.obj
 0001:00002f25       ?getAccessibleSelectionFromContext@WinAccessBridge@@QAE_JJ_JH@Z 10003f25 f   WinAccessBridge.obj
 0001:00002f96       ?getAccessibleTableCellInfo@WinAccessBridge@@QAEHJ_JJJPAUAccessibleTableCellInfoTag@@@Z 10003f96 f   WinAccessBridge.obj
 0001:00003076       ?getAccessibleTableColumn@WinAccessBridge@@QAEJJ_JJ@Z 10004076 f   WinAccessBridge.obj
 0001:0000311e       ?getAccessibleTableColumnDescription@WinAccessBridge@@QAE_JJ_JJ@Z 1000411e f   WinAccessBridge.obj
 0001:000031cc       ?getAccessibleTableColumnHeader@WinAccessBridge@@QAEHJ_JPAUAccessibleTableInfoTag@@@Z 100041cc f   WinAccessBridge.obj
 0001:00003281       ?getAccessibleTableColumnSelectionCount@WinAccessBridge@@QAEJJ_J@Z 10004281 f   WinAccessBridge.obj
 0001:0000331d       ?getAccessibleTableColumnSelections@WinAccessBridge@@QAEHJ_JJPAJ@Z 1000431d f   WinAccessBridge.obj
 0001:00003401       ?getAccessibleTableIndex@WinAccessBridge@@QAEJJ_JJJ@Z 10004401 f   WinAccessBridge.obj
 0001:000034b5       ?getAccessibleTableInfo@WinAccessBridge@@QAEHJ_JPAUAccessibleTableInfoTag@@@Z 100044b5 f   WinAccessBridge.obj
 0001:0000356f       ?getAccessibleTableRow@WinAccessBridge@@QAEJJ_JJ@Z 1000456f f   WinAccessBridge.obj
 0001:00003617       ?getAccessibleTableRowDescription@WinAccessBridge@@QAE_JJ_JJ@Z 10004617 f   WinAccessBridge.obj
 0001:000036c5       ?getAccessibleTableRowHeader@WinAccessBridge@@QAEHJ_JPAUAccessibleTableInfoTag@@@Z 100046c5 f   WinAccessBridge.obj
 0001:0000377a       ?getAccessibleTableRowSelectionCount@WinAccessBridge@@QAEJJ_J@Z 1000477a f   WinAccessBridge.obj
 0001:00003816       ?getAccessibleTableRowSelections@WinAccessBridge@@QAEHJ_JJPAJ@Z 10004816 f   WinAccessBridge.obj
 0001:000038f5       ?getAccessibleTextAttributes@WinAccessBridge@@QAEHJ_JJPAUAccessibleTextAttributesInfoTag@@@Z 100048f5 f   WinAccessBridge.obj
 0001:000039a9       ?getAccessibleTextInfo@WinAccessBridge@@QAEHJ_JPAUAccessibleTextInfoTag@@JJ@Z 100049a9 f   WinAccessBridge.obj
 0001:00003a77       ?getAccessibleTextItems@WinAccessBridge@@QAEHJ_JPAUAccessibleTextItemsInfoTag@@J@Z 10004a77 f   WinAccessBridge.obj
 0001:00003b5b       ?getAccessibleTextLineBounds@WinAccessBridge@@QAEHJ_JJPAJ1@Z 10004b5b f   WinAccessBridge.obj
 0001:00003bfd       ?getAccessibleTextRange@WinAccessBridge@@QAEHJ_JJJPAGF@Z 10004bfd f   WinAccessBridge.obj
 0001:00003cda       ?getAccessibleTextRect@WinAccessBridge@@QAEHJ_JPAUAccessibleTextRectInfoTag@@J@Z 10004cda f   WinAccessBridge.obj
 0001:00003d70       ?getAccessibleTextSelectionInfo@WinAccessBridge@@QAEHJ_JPAUAccessibleTextSelectionInfoTag@@@Z 10004d70 f   WinAccessBridge.obj
 0001:00003e1a       ?getActiveDescendent@WinAccessBridge@@QAE_JJ_J@Z 10004e1a f   WinAccessBridge.obj
 0001:00003e99       ?getCaretLocation@WinAccessBridge@@QAEHJ_JPAUAccessibleTextRectInfoTag@@J@Z 10004e99 f   WinAccessBridge.obj
 0001:00003f2f       ?getCurrentAccessibleValueFromContext@WinAccessBridge@@QAEHJ_JPAGF@Z 10004f2f f   WinAccessBridge.obj
 0001:00003fc4       ?getEventsWaiting@WinAccessBridge@@QAEHXZ 10004fc4 f   WinAccessBridge.obj
 0001:00003fd2       ?getHWNDFromAccessibleContext@WinAccessBridge@@QAEPAUHWND__@@J_J@Z 10004fd2 f   WinAccessBridge.obj
 0001:00004053       ?getMaximumAccessibleValueFromContext@WinAccessBridge@@QAEHJ_JPAGF@Z 10005053 f   WinAccessBridge.obj
 0001:000040e8       ?getMinimumAccessibleValueFromContext@WinAccessBridge@@QAEHJ_JPAGF@Z 100050e8 f   WinAccessBridge.obj
 0001:0000417d       ?getObjectDepth@WinAccessBridge@@QAEHJ_J@Z 1000517d f   WinAccessBridge.obj
 0001:000041f8       ?getParentWithRole@WinAccessBridge@@QAE_JJ_JPBG@Z 100051f8 f   WinAccessBridge.obj
 0001:000042f5       ?getParentWithRoleElseRoot@WinAccessBridge@@QAE_JJ_JPBG@Z 100052f5 f   WinAccessBridge.obj
 0001:000043b8       ?getTextAttributesInRange@WinAccessBridge@@QAEHJ_JHHPAUAccessibleTextAttributesInfoTag@@PAF@Z 100053b8 f   WinAccessBridge.obj
 0001:000044c4       ?getTopLevelObject@WinAccessBridge@@QAE_JJ_J@Z 100054c4 f   WinAccessBridge.obj
 0001:00004543       ?getVersionInfo@WinAccessBridge@@QAEHJPAUAccessBridgeVersionInfoTag@@@Z 10005543 f   WinAccessBridge.obj
 0001:000045f7       ?getVirtualAccessibleName@WinAccessBridge@@QAEHJ_JPAGH@Z 100055f7 f   WinAccessBridge.obj
 0001:000046d3       ?getVisibleChildren@WinAccessBridge@@QAEHJ_JHPAUVisibleChildenInfoTag@@@Z 100056d3 f   WinAccessBridge.obj
 0001:00004785       ?getVisibleChildrenCount@WinAccessBridge@@QAEHJ_J@Z 10005785 f   WinAccessBridge.obj
 0001:00004800       ?initWindow@WinAccessBridge@@QAEHXZ 10005800 f   WinAccessBridge.obj
 0001:00004840       ?isAccessibleChildSelectedFromContext@WinAccessBridge@@QAEHJ_JH@Z 10005840 f   WinAccessBridge.obj
 0001:000048ad       ?isAccessibleTableColumnSelected@WinAccessBridge@@QAEHJ_JJ@Z 100058ad f   WinAccessBridge.obj
 0001:00004952       ?isAccessibleTableRowSelected@WinAccessBridge@@QAEHJ_JJ@Z 10005952 f   WinAccessBridge.obj
 0001:000049f7       ?isJavaWindow@WinAccessBridge@@QAEHPAUHWND__@@@Z 100059f7 f   WinAccessBridge.obj
 0001:00004a90       ?isSameObject@WinAccessBridge@@QAEHJ_J0@Z 10005a90 f   WinAccessBridge.obj
 0001:00004b4b       ?preProcessPackage@WinAccessBridge@@QAEXPADJ@Z 10005b4b f   WinAccessBridge.obj
 0001:00004bd8       ?processPackage@WinAccessBridge@@QAEXPADJ@Z 10005bd8 f   WinAccessBridge.obj
 0001:00005360       ?queuePackage@WinAccessBridge@@QAEHPADJ@Z 10006360 f   WinAccessBridge.obj
 0001:000053b8       ?receiveAQueuedPackage@WinAccessBridge@@QAEHXZ 100063b8 f   WinAccessBridge.obj
 0001:000054ae       ?releaseJavaObject@WinAccessBridge@@QAEXJ_J@Z 100064ae f   WinAccessBridge.obj
 0001:00005527       ?removeAccessibilityEventNotification@WinAccessBridge@@QAEX_J@Z 10006527 f   WinAccessBridge.obj
 0001:000055b3       ?removeAccessibleSelectionFromContext@WinAccessBridge@@QAEXJ_JH@Z 100065b3 f   WinAccessBridge.obj
 0001:00005613       ?removeJavaEventNotification@WinAccessBridge@@QAEX_J@Z 10006613 f   WinAccessBridge.obj
 0001:0000569f       ?rendezvousWithNewJavaDLL@WinAccessBridge@@QAEJPAUHWND__@@J@Z 1000669f f   WinAccessBridge.obj
 0001:0000575f       ?requestFocus@WinAccessBridge@@QAEHJ_J@Z 1000675f f   WinAccessBridge.obj
 0001:000057d4       ?selectAllAccessibleSelectionFromContext@WinAccessBridge@@QAEXJ_J@Z 100067d4 f   WinAccessBridge.obj
 0001:0000582e       ?selectTextRange@WinAccessBridge@@QAEHJ_JHH@Z 1000682e f   WinAccessBridge.obj
 0001:000058b3       ?sendMemoryPackage@WinAccessBridge@@QAEHPADJPAUHWND__@@@Z 100068b3 f   WinAccessBridge.obj
 0001:00005901       ?sendPackage@WinAccessBridge@@QAEXPADJPAUHWND__@@@Z 10006901 f   WinAccessBridge.obj
 0001:0000592d       ?setCaretPosition@WinAccessBridge@@QAEHJ_JH@Z 1000692d f   WinAccessBridge.obj
 0001:000059a8       ?setCaretUpdateFP@WinAccessBridge@@QAEXP6AXJ_J0@Z@Z 100069a8 f   WinAccessBridge.obj
 0001:000059b8       ?setFocusGainedFP@WinAccessBridge@@QAEXP6AXJ_J0@Z@Z 100069b8 f   WinAccessBridge.obj
 0001:000059c8       ?setFocusLostFP@WinAccessBridge@@QAEXP6AXJ_J0@Z@Z 100069c8 f   WinAccessBridge.obj
 0001:000059d8       ?setJavaShutdownFP@WinAccessBridge@@QAEXP6AXJ@Z@Z 100069d8 f   WinAccessBridge.obj
 0001:000059e8       ?setMenuCanceledFP@WinAccessBridge@@QAEXP6AXJ_J0@Z@Z 100069e8 f   WinAccessBridge.obj
 0001:000059f8       ?setMenuDeselectedFP@WinAccessBridge@@QAEXP6AXJ_J0@Z@Z 100069f8 f   WinAccessBridge.obj
 0001:00005a08       ?setMenuSelectedFP@WinAccessBridge@@QAEXP6AXJ_J0@Z@Z 10006a08 f   WinAccessBridge.obj
 0001:00005a18       ?setMouseClickedFP@WinAccessBridge@@QAEXP6AXJ_J0@Z@Z 10006a18 f   WinAccessBridge.obj
 0001:00005a28       ?setMouseEnteredFP@WinAccessBridge@@QAEXP6AXJ_J0@Z@Z 10006a28 f   WinAccessBridge.obj
 0001:00005a38       ?setMouseExitedFP@WinAccessBridge@@QAEXP6AXJ_J0@Z@Z 10006a38 f   WinAccessBridge.obj
 0001:00005a48       ?setMousePressedFP@WinAccessBridge@@QAEXP6AXJ_J0@Z@Z 10006a48 f   WinAccessBridge.obj
 0001:00005a58       ?setMouseReleasedFP@WinAccessBridge@@QAEXP6AXJ_J0@Z@Z 10006a58 f   WinAccessBridge.obj
 0001:00005a68       ?setPopupMenuCanceledFP@WinAccessBridge@@QAEXP6AXJ_J0@Z@Z 10006a68 f   WinAccessBridge.obj
 0001:00005a78       ?setPopupMenuWillBecomeInvisibleFP@WinAccessBridge@@QAEXP6AXJ_J0@Z@Z 10006a78 f   WinAccessBridge.obj
 0001:00005a88       ?setPopupMenuWillBecomeVisibleFP@WinAccessBridge@@QAEXP6AXJ_J0@Z@Z 10006a88 f   WinAccessBridge.obj
 0001:00005a98       ?setPropertyActiveDescendentChangeFP@WinAccessBridge@@QAEXP6AXJ_J000@Z@Z 10006a98 f   WinAccessBridge.obj
 0001:00005aa8       ?setPropertyCaretChangeFP@WinAccessBridge@@QAEXP6AXJ_J0HH@Z@Z 10006aa8 f   WinAccessBridge.obj
 0001:00005ab8       ?setPropertyChangeFP@WinAccessBridge@@QAEXP6AXJ_J0PAG11@Z@Z 10006ab8 f   WinAccessBridge.obj
 0001:00005ac8       ?setPropertyChildChangeFP@WinAccessBridge@@QAEXP6AXJ_J000@Z@Z 10006ac8 f   WinAccessBridge.obj
 0001:00005ad8       ?setPropertyDescriptionChangeFP@WinAccessBridge@@QAEXP6AXJ_J0PAG1@Z@Z 10006ad8 f   WinAccessBridge.obj
 0001:00005ae8       ?setPropertyNameChangeFP@WinAccessBridge@@QAEXP6AXJ_J0PAG1@Z@Z 10006ae8 f   WinAccessBridge.obj
 0001:00005af8       ?setPropertySelectionChangeFP@WinAccessBridge@@QAEXP6AXJ_J0@Z@Z 10006af8 f   WinAccessBridge.obj
 0001:00005b08       ?setPropertyStateChangeFP@WinAccessBridge@@QAEXP6AXJ_J0PAG1@Z@Z 10006b08 f   WinAccessBridge.obj
 0001:00005b18       ?setPropertyTableModelChangeFP@WinAccessBridge@@QAEXP6AXJ_J0PAG1@Z@Z 10006b18 f   WinAccessBridge.obj
 0001:00005b28       ?setPropertyTextChangeFP@WinAccessBridge@@QAEXP6AXJ_J0@Z@Z 10006b28 f   WinAccessBridge.obj
 0001:00005b38       ?setPropertyValueChangeFP@WinAccessBridge@@QAEXP6AXJ_J0PAG1@Z@Z 10006b38 f   WinAccessBridge.obj
 0001:00005b48       ?setPropertyVisibleDataChangeFP@WinAccessBridge@@QAEXP6AXJ_J0@Z@Z 10006b48 f   WinAccessBridge.obj
 0001:00005b58       ?setTextContents@WinAccessBridge@@QAEHJ_JPBG@Z 10006b58 f   WinAccessBridge.obj
 0001:00005c1a       _AccessBridgeDialogProc@16 10006c1a f   WinAccessBridge.obj
 0001:00005d28       _DllMain@12                10006d28 f   WinAccessBridge.obj
 0001:00005da5       ??_U@YAPAXI@Z              10006da5 f   LIBCMT:new_array.obj
 0001:00005dae       ??_V@YAXPAX@Z              10006dae f   LIBCMT:delete_array.obj
 0001:00005dc0       __aulldiv                  10006dc0 f   LIBCMT:ulldiv.obj
 0001:00005e28       @__security_check_cookie@4 10006e28 f   LIBCMT:secchk.obj
 0001:00005e39       ??3@YAXPAXI@Z              10006e39 f   LIBCMT:delete_scalar_size.obj
 0001:00005e47       ??_Etype_info@@UAEPAXI@Z   10006e47 f i LIBCMT:std_type_info_static.obj
 0001:00005e47       ??_Gtype_info@@UAEPAXI@Z   10006e47 f i LIBCMT:std_type_info_static.obj
 0001:00005e6a       ??2@YAPAXI@Z               10006e6a f   LIBCMT:new_scalar.obj
 0001:00005ea0       __alloca_probe             10006ea0 f   LIBCMT:chkstk.obj
 0001:00005ea0       __chkstk                   10006ea0 f   LIBCMT:chkstk.obj
 0001:000061ef       __DllMainCRTStartup@12     100071ef f   LIBCMT:dll_dllmain.obj
 0001:00006212       ??3@YAXPAX@Z               10007212 f   LIBCMT:delete_scalar.obj
 0001:00006217       ___raise_securityfailure   10007217 f   LIBCMT:gs_report.obj
 0001:0000623f       ___report_gsfailure        1000723f f   LIBCMT:gs_report.obj
 0001:00006338       ??0bad_array_new_length@std@@QAE@ABV01@@Z 10007338 f i LIBCMT:throw_bad_alloc.obj
 0001:00006353       ??0bad_array_new_length@std@@QAE@XZ 10007353 f i LIBCMT:throw_bad_alloc.obj
 0001:0000636b       ??_Ebad_exception@std@@UAEPAXI@Z 1000736b f i libvcruntime:frame.obj
 0001:0000636b       ??_Gbad_exception@std@@UAEPAXI@Z 1000736b f i libvcruntime:frame.obj
 0001:0000636b       ??_Ebad_array_new_length@std@@UAEPAXI@Z 1000736b f i LIBCMT:throw_bad_alloc.obj
 0001:0000636b       ??_Gbad_array_new_length@std@@UAEPAXI@Z 1000736b f i LIBCMT:throw_bad_alloc.obj
 0001:00006398       ?__scrt_throw_std_bad_alloc@@YAXXZ 10007398 f   LIBCMT:throw_bad_alloc.obj
 0001:000063b5       ?__scrt_throw_std_bad_array_new_length@@YAXXZ 100073b5 f   LIBCMT:throw_bad_alloc.obj
 0001:0000641f       ___security_init_cookie    1000741f f   LIBCMT:gs_support.obj
 0001:0000646a       ?__scrt_initialize_type_info@@YAXXZ 1000746a f   LIBCMT:tncleanup.obj
 0001:00006476       ?__scrt_uninitialize_type_info@@YAXXZ 10007476 f   LIBCMT:tncleanup.obj
 0001:00006482       ___local_stdio_scanf_options 10007482 f i LIBCMT:default_local_stdio_options.obj
 0001:00006488       ___scrt_initialize_default_local_stdio_options 10007488 f   LIBCMT:default_local_stdio_options.obj
 0001:000064e9       ___scrt_acquire_startup_lock 100074e9 f   LIBCMT:utility.obj
 0001:0000651b       ___scrt_dllmain_after_initialize_c 1000751b f   LIBCMT:utility.obj
 0001:00006546       ___scrt_dllmain_before_initialize_c 10007546 f   LIBCMT:utility.obj
 0001:00006554       ___scrt_dllmain_crt_thread_attach 10007554 f   LIBCMT:utility.obj
 0001:00006573       ___scrt_dllmain_crt_thread_detach 10007573 f   LIBCMT:utility.obj
 0001:00006580       ___scrt_dllmain_exception_filter 10007580 f   LIBCMT:utility.obj
 0001:000065b4       ___scrt_dllmain_uninitialize_c 100075b4 f   LIBCMT:utility.obj
 0001:000065d7       ___scrt_dllmain_uninitialize_critical 100075d7 f   LIBCMT:utility.obj
 0001:000065e4       ___scrt_initialize_crt     100075e4 f   LIBCMT:utility.obj
 0001:0000661d       ___scrt_initialize_onexit_tables 1000761d f   LIBCMT:utility.obj
 0001:000066c2       ___scrt_is_nonwritable_in_current_image 100076c2 f   LIBCMT:utility.obj
 0001:00006756       ___scrt_release_startup_lock 10007756 f   LIBCMT:utility.obj
 0001:00006773       ___scrt_uninitialize_crt   10007773 f   LIBCMT:utility.obj
 0001:0000679b       ___scrt_get_dyn_tls_init_callback 1000779b f   LIBCMT:dyn_tls_init.obj
 0001:000067a1       ___scrt_fastfail           100077a1 f   LIBCMT:utility_desktop.obj
 0001:000068bb       __crt_debugger_hook        100078bb f   LIBCMT:utility_desktop.obj
 0001:000068c3       __RTC_Initialize           100078c3 f   LIBCMT:initsect.obj
 0001:000068ef       __RTC_Terminate            100078ef f   LIBCMT:initsect.obj
 0001:00006920       __SEH_prolog4              10007920 f   LIBCMT:sehprolg4.obj
 0001:00006966       __SEH_epilog4              10007966 f   LIBCMT:sehprolg4.obj
 0001:0000697b       ___isa_available_init      1000797b f   LIBCMT:cpu_disp.obj
 0001:00006b12       __get_startup_argv_mode    10007b12 f   LIBCMT:argv_mode.obj
 0001:00006b16       ___scrt_is_ucrt_dll_in_use 10007b16 f   LIBCMT:ucrt_detection.obj
 0001:00006b30       _memcpy                    10007b30 f   libvcruntime:memcpy.obj
 0001:000070b0       _memset                    100080b0 f   libvcruntime:memset.obj
 0001:0000720a       ___std_exception_copy      1000820a f   libvcruntime:std_exception.obj
 0001:0000726d       ___std_exception_destroy   1000826d f   libvcruntime:std_exception.obj
 0001:0000728c       __CxxThrowException@8      1000828c f   libvcruntime:throw.obj
 0001:00007340       __except_handler4          10008340 f   libvcruntime:chandler4.obj
 0001:00007497       ___std_type_info_compare   10008497 f   libvcruntime:std_type_info.obj
 0001:000074d3       ___std_type_info_destroy_list 100084d3 f   libvcruntime:std_type_info.obj
 0001:000074f6       ___vcrt_initialize         100084f6 f   libvcruntime:initialization.obj
 0001:0000751f       ___vcrt_thread_attach      1000851f f   libvcruntime:initialization.obj
 0001:0000752a       ___vcrt_thread_detach      1000852a f   libvcruntime:initialization.obj
 0001:00007535       ___vcrt_uninitialize       10008535 f   libvcruntime:initialization.obj
 0001:00007554       ___vcrt_uninitialize_critical 10008554 f   libvcruntime:initialization.obj
 0001:00007560       __local_unwind4            10008560 f   libvcruntime:exsup4.obj
 0001:00007638       __seh_longjmp_unwind4@4    10008638 f   libvcruntime:exsup4.obj
 0001:00007660       @_EH4_CallFilterFunc@8     10008660 f   libvcruntime:exsup4.obj
 0001:00007678       @_EH4_TransferToHandler@8  10008678 f   libvcruntime:exsup4.obj
 0001:00007694       @_EH4_GlobalUnwind2@8      10008694 f   libvcruntime:exsup4.obj
 0001:000076b0       @_EH4_LocalUnwind@16       100086b0 f   libvcruntime:exsup4.obj
 0001:000076c7       ___except_validate_context_record 100086c7 f   libvcruntime:jbcxrval.obj
 0001:000076f7       ___except_validate_jump_buffer 100086f7 f   libvcruntime:jbcxrval.obj
 0001:00007724       ___vcrt_freefls@4          10008724 f   libvcruntime:per_thread_data.obj
 0001:00007740       ___vcrt_freeptd            10008740 f   libvcruntime:per_thread_data.obj
 0001:00007776       ___vcrt_getptd             10008776 f   libvcruntime:per_thread_data.obj
 0001:00007784       ___vcrt_getptd_noexit      10008784 f   libvcruntime:per_thread_data.obj
 0001:00007816       ___vcrt_initialize_ptd     10008816 f   libvcruntime:per_thread_data.obj
 0001:00007849       ___vcrt_uninitialize_ptd   10008849 f   libvcruntime:per_thread_data.obj
 0001:00007864       ___vcrt_initialize_locks   10008864 f   libvcruntime:locks.obj
 0001:000078a0       ___vcrt_uninitialize_locks 100088a0 f   libvcruntime:locks.obj
 0001:000078cf       ??$__crt_fast_encode_pointer@PAX@@YAPAXQAX@Z 100088cf f i libvcruntime:winapi_downlevel.obj
 0001:00007a1f       ___vcrt_FlsAlloc           10008a1f f   libvcruntime:winapi_downlevel.obj
 0001:00007a5a       ___vcrt_FlsFree            10008a5a f   libvcruntime:winapi_downlevel.obj
 0001:00007a95       ___vcrt_FlsGetValue        10008a95 f   libvcruntime:winapi_downlevel.obj
 0001:00007ad0       ___vcrt_FlsSetValue        10008ad0 f   libvcruntime:winapi_downlevel.obj
 0001:00007b0e       ___vcrt_InitializeCriticalSectionEx 10008b0e f   libvcruntime:winapi_downlevel.obj
 0001:00007b55       ___vcrt_initialize_winapi_thunks 10008b55 f   libvcruntime:winapi_downlevel.obj
 0001:00007b7e       ___vcrt_uninitialize_winapi_thunks 10008b7e f   libvcruntime:winapi_downlevel.obj
 0001:00007bb0       ___vcrt_initialize_pure_virtual_call_handler 10008bb0 f   libvcruntime:purevirt_data.obj
 0001:00007bc0       __global_unwind2           10008bc0 f   libvcruntime:exsup.obj
 0001:00007c26       __local_unwind2            10008c26 f   libvcruntime:exsup.obj
 0001:00007caa       __abnormal_termination     10008caa f   libvcruntime:exsup.obj
 0001:00007cd0       __NLG_Notify1              10008cd0 f   libvcruntime:exsup.obj
 0001:00007cdc       __NLG_Notify               10008cdc f   libvcruntime:exsup.obj
 0001:00007cf3       __NLG_Dispatch             10008cf3     libvcruntime:exsup.obj
 0001:00007cf3       __NLG_Dispatch2            10008cf3     libvcruntime:exsup.obj
 0001:00007cfb       __NLG_Call                 10008cfb f   libvcruntime:exsup.obj
 0001:00007cfd       __NLG_Return2              10008cfd     libvcruntime:exsup.obj
 0001:00007cfe       ?GetRangeOfTrysToCheck@__FrameHandler3@@SA?AU?$pair@Viterator@TryBlockMap@__FrameHandler3@@V123@@std@@AAVTryBlockMap@1@HH@Z 10008cfe f   libvcruntime:trnsctrl.obj
 0001:00007d80       ?_CallCatchBlock2@@YAPAXPAUEHRegistrationNode@@PBU_s_FuncInfo@@PAXHK@Z 10008d80 f   libvcruntime:trnsctrl.obj
 0001:00007dde       ?_CallSETranslator@@YAHPAUEHExceptionRecord@@PAUEHRegistrationNode@@PAX2PBU_s_FuncInfo@@H1@Z 10008dde f   libvcruntime:trnsctrl.obj
 0001:00007eb9       ?_JumpToContinuation@@YGXPAXPAUEHRegistrationNode@@@Z 10008eb9 f   libvcruntime:trnsctrl.obj
 0001:00007ee9       ?_UnwindNestedFrames@@YGXPAUEHRegistrationNode@@PAUEHExceptionRecord@@@Z 10008ee9 f   libvcruntime:trnsctrl.obj
 0001:00007f3c       __CatchGuardHandler        10008f3c f   libvcruntime:trnsctrl.obj
 0001:00007f6d       __CreateFrameInfo          10008f6d f   libvcruntime:trnsctrl.obj
 0001:00007f91       __FindAndUnlinkFrame       10008f91 f   libvcruntime:trnsctrl.obj
 0001:00007fd6       __TranslatorGuardHandler   10008fd6 f   libvcruntime:trnsctrl.obj
 0001:00008073       ___CxxFrameHandler3        10009073 f   libvcruntime:trnsctrl.obj
 0001:000087a0       ??$TypeMatchHelper@V__FrameHandler3@@@@YAHPBU_s_HandlerType@@PBU_s_CatchableType@@PBU_s_ThrowInfo@@@Z 100097a0 f i libvcruntime:frame.obj
 0001:0000882e       ??$__InternalCxxFrameHandler@V__FrameHandler3@@@@YA?AW4_EXCEPTION_DISPOSITION@@PAUEHExceptionRecord@@PAUEHRegistrationNode@@PAU_CONTEXT@@PAXPBU_s_FuncInfo@@H1E@Z 1000982e f i libvcruntime:frame.obj
 0001:00008930       ??0bad_exception@std@@QAE@ABV01@@Z 10009930 f i libvcruntime:frame.obj
 0001:0000894b       ??0bad_exception@std@@QAE@XZ 1000994b f i libvcruntime:frame.obj
 0001:00008963       ??8type_info@@QBE_NABV0@@Z 10009963 f i libvcruntime:frame.obj
 0001:00008bca       ?FrameUnwindToEmptyState@__FrameHandler3@@SAXPAUEHRegistrationNode@@PAXPBU_s_FuncInfo@@@Z 10009bca f   libvcruntime:frame.obj
 0001:00008be2       ?FrameUnwindToState@__FrameHandler3@@SAXPAUEHRegistrationNode@@PAXPBU_s_FuncInfo@@H@Z 10009be2 f   libvcruntime:frame.obj
 0001:00008d64       ?_CallMemberFunction1@@YGXQAX00@Z 10009d64 f i libvcruntime:frame.obj
 0001:00008d74       ?_CallMemberFunction2@@YGXQAX00H@Z 10009d74 f i libvcruntime:frame.obj
 0001:00008d87       ?getESTypes@__FrameHandler3@@SAPBU_s_ESTypeList@@PBU_s_FuncInfo@@@Z 10009d87 f i libvcruntime:frame.obj
 0001:00008da0       __CallSettingFrame@12      10009da0 f   libvcruntime:lowhelpr.obj
 0001:00008dc7       __NLG_Return               10009dc7     libvcruntime:lowhelpr.obj
 0001:00008dec       _unexpected                10009dec f   libvcruntime:unexpected.obj
 0001:00008e09       ?GetCurrentState@__FrameHandler3@@SAHPAUEHRegistrationNode@@PAXPBU_s_FuncInfo@@@Z 10009e09 f   libvcruntime:ehstate.obj
 0001:00008e26       ?SetState@__FrameHandler3@@SAXPAUEHRegistrationNode@@PBU_s_FuncInfo@@H@Z 10009e26 f   libvcruntime:ehstate.obj
 0001:00008e34       ___DestructExceptionObject 10009e34 f   libvcruntime:ehhelpers.obj
 0001:00008ed4       ?_CallMemberFunction0@@YGXQAX0@Z 10009ed4 f i libvcruntime:ehhelpers.obj
 0001:00008ee1       __IsExceptionObjectToBeDestroyed 10009ee1 f   libvcruntime:ehhelpers.obj
 0001:00008f07       ___AdjustPointer           10009f07 f   libvcruntime:ehhelpers.obj
 0001:00008f2c       ___FrameUnwindFilter       10009f2c f   libvcruntime:ehhelpers.obj
 0001:00008f71       ___std_terminate           10009f71 f   libvcruntime:ehhelpers.obj
 0001:00008f80       _memmove                   10009f80 f   libvcruntime:memmove.obj
 0001:00009500       _strlen                    1000a500 f   libucrt:strlen.obj
 0001:00009590       _strncat                   1000a590 f   libucrt:strncat.obj
 0001:000096d0       _strncpy                   1000a6d0 f   libucrt:strncpy.obj
 0001:000097f4       ___acrt_initialize_stdio   1000a7f4 f   libucrt:_file.obj
 0001:000098bc       ___acrt_iob_func           1000a8bc f   libucrt:_file.obj
 0001:000098cc       ___acrt_uninitialize_stdio 1000a8cc f   libucrt:_file.obj
 0001:00009918       __lock_file                1000a918 f   libucrt:_file.obj
 0001:0000992c       __unlock_file              1000a92c f   libucrt:_file.obj
 0001:00009b0f       ??$count@D@formatting_buffer@__crt_stdio_output@@QBEIXZ 1000ab0f f i libucrt:output.obj
 0001:00009b27       ??$ensure_buffer_is_big_enough@D@formatting_buffer@__crt_stdio_output@@QAE_NIAAV__crt_cached_ptd_host@@@Z 1000ab27 f i libucrt:output.obj
 0001:00009ba8       ??$is_overflow_condition@K@__crt_strtox@@YA_NIK@Z 1000aba8 f i libucrt:output.obj
 0001:00009bdc       ??$is_wide_character_specifier@D@__crt_stdio_output@@YA_N_KDW4length_modifier@0@@Z 1000abdc f i libucrt:output.obj
 0001:00009c0d       ??$parse_integer@KV?$c_string_character_source@D@__crt_strtox@@$0A@@__crt_strtox@@YAKAAV__crt_cached_ptd_host@@V?$c_string_character_source@D@0@H_N@Z 1000ac0d f i libucrt:output.obj
 0001:00009e1c       ??$scratch_data@D@formatting_buffer@__crt_stdio_output@@QAEPADXZ 1000ae1c f i libucrt:output.obj
 0001:00009e3a       ??$type_case_integer@$07@?$output_processor@DV?$stream_output_adapter@D@__crt_stdio_output@@V?$standard_base@DV?$stream_output_adapter@D@__crt_stdio_output@@@2@@__crt_stdio_output@@AAE_N_N@Z 1000ae3a f i libucrt:output.obj
 0001:00009e3a       ??$type_case_integer@$07@?$output_processor@DV?$string_output_adapter@D@__crt_stdio_output@@V?$standard_base@DV?$string_output_adapter@D@__crt_stdio_output@@@2@@__crt_stdio_output@@AAE_N_N@Z 1000ae3a f i libucrt:output.obj
 0001:00009fc7       ??$type_case_integer@$09@?$output_processor@DV?$stream_output_adapter@D@__crt_stdio_output@@V?$standard_base@DV?$stream_output_adapter@D@__crt_stdio_output@@@2@@__crt_stdio_output@@AAE_N_N@Z 1000afc7 f i libucrt:output.obj
 0001:00009fc7       ??$type_case_integer@$09@?$output_processor@DV?$string_output_adapter@D@__crt_stdio_output@@V?$standard_base@DV?$string_output_adapter@D@__crt_stdio_output@@@2@@__crt_stdio_output@@AAE_N_N@Z 1000afc7 f i libucrt:output.obj
 0001:0000a154       ??$type_case_integer@$0BA@@?$output_processor@DV?$stream_output_adapter@D@__crt_stdio_output@@V?$standard_base@DV?$stream_output_adapter@D@__crt_stdio_output@@@2@@__crt_stdio_output@@AAE_N_N@Z 1000b154 f i libucrt:output.obj
 0001:0000a154       ??$type_case_integer@$0BA@@?$output_processor@DV?$string_output_adapter@D@__crt_stdio_output@@V?$standard_base@DV?$string_output_adapter@D@__crt_stdio_output@@@2@@__crt_stdio_output@@AAE_N_N@Z 1000b154 f i libucrt:output.obj
 0001:0000a2e1       ??$type_case_integer_parse_into_buffer@I$07@?$output_processor@DV?$string_output_adapter@D@__crt_stdio_output@@V?$standard_base@DV?$string_output_adapter@D@__crt_stdio_output@@@2@@__crt_stdio_output@@AAEXI_N@Z 1000b2e1 f i libucrt:output.obj
 0001:0000a2e1       ??$type_case_integer_parse_into_buffer@I$07@?$output_processor@DV?$stream_output_adapter@D@__crt_stdio_output@@V?$standard_base@DV?$stream_output_adapter@D@__crt_stdio_output@@@2@@__crt_stdio_output@@AAEXI_N@Z 1000b2e1 f i libucrt:output.obj
 0001:0000a344       ??$type_case_integer_parse_into_buffer@I$09@?$output_processor@DV?$stream_output_adapter@D@__crt_stdio_output@@V?$standard_base@DV?$stream_output_adapter@D@__crt_stdio_output@@@2@@__crt_stdio_output@@AAEXI_N@Z 1000b344 f i libucrt:output.obj
 0001:0000a344       ??$type_case_integer_parse_into_buffer@I$09@?$output_processor@DV?$string_output_adapter@D@__crt_stdio_output@@V?$standard_base@DV?$string_output_adapter@D@__crt_stdio_output@@@2@@__crt_stdio_output@@AAEXI_N@Z 1000b344 f i libucrt:output.obj
 0001:0000a3cb       ??$type_case_integer_parse_into_buffer@I$0BA@@?$output_processor@DV?$stream_output_adapter@D@__crt_stdio_output@@V?$standard_base@DV?$stream_output_adapter@D@__crt_stdio_output@@@2@@__crt_stdio_output@@AAEXI_N@Z 1000b3cb f i libucrt:output.obj
 0001:0000a3cb       ??$type_case_integer_parse_into_buffer@I$0BA@@?$output_processor@DV?$string_output_adapter@D@__crt_stdio_output@@V?$standard_base@DV?$string_output_adapter@D@__crt_stdio_output@@@2@@__crt_stdio_output@@AAEXI_N@Z 1000b3cb f i libucrt:output.obj
 0001:0000a448       ??$type_case_integer_parse_into_buffer@_K$07@?$output_processor@DV?$stream_output_adapter@D@__crt_stdio_output@@V?$standard_base@DV?$stream_output_adapter@D@__crt_stdio_output@@@2@@__crt_stdio_output@@AAEX_K_N@Z 1000b448 f i libucrt:output.obj
 0001:0000a448       ??$type_case_integer_parse_into_buffer@_K$07@?$output_processor@DV?$string_output_adapter@D@__crt_stdio_output@@V?$standard_base@DV?$string_output_adapter@D@__crt_stdio_output@@@2@@__crt_stdio_output@@AAEX_K_N@Z 1000b448 f i libucrt:output.obj
 0001:0000a4c0       ??$type_case_integer_parse_into_buffer@_K$09@?$output_processor@DV?$stream_output_adapter@D@__crt_stdio_output@@V?$standard_base@DV?$stream_output_adapter@D@__crt_stdio_output@@@2@@__crt_stdio_output@@AAEX_K_N@Z 1000b4c0 f i libucrt:output.obj
 0001:0000a4c0       ??$type_case_integer_parse_into_buffer@_K$09@?$output_processor@DV?$string_output_adapter@D@__crt_stdio_output@@V?$standard_base@DV?$string_output_adapter@D@__crt_stdio_output@@@2@@__crt_stdio_output@@AAEX_K_N@Z 1000b4c0 f i libucrt:output.obj
 0001:0000a567       ??$type_case_integer_parse_into_buffer@_K$0BA@@?$output_processor@DV?$stream_output_adapter@D@__crt_stdio_output@@V?$standard_base@DV?$stream_output_adapter@D@__crt_stdio_output@@@2@@__crt_stdio_output@@AAEX_K_N@Z 1000b567 f i libucrt:output.obj
 0001:0000a567       ??$type_case_integer_parse_into_buffer@_K$0BA@@?$output_processor@DV?$string_output_adapter@D@__crt_stdio_output@@V?$standard_base@DV?$string_output_adapter@D@__crt_stdio_output@@@2@@__crt_stdio_output@@AAEX_K_N@Z 1000b567 f i libucrt:output.obj
 0001:0000a5f1       ??0?$output_adapter_data@DV?$string_output_adapter@D@__crt_stdio_output@@@__crt_stdio_output@@IAE@ABV?$string_output_adapter@D@1@_KQBDAAV__crt_cached_ptd_host@@QAD@Z 1000b5f1 f i libucrt:output.obj
 0001:0000a5f1       ??0?$output_adapter_data@DV?$stream_output_adapter@D@__crt_stdio_output@@@__crt_stdio_output@@IAE@ABV?$stream_output_adapter@D@1@_KQBDAAV__crt_cached_ptd_host@@QAD@Z 1000b5f1 f i libucrt:output.obj
 0001:0000a660       ??0__crt_cached_ptd_host@@QAE@QAU__crt_locale_pointers@@@Z 1000b660 f i libucrt:output.obj
 0001:0000a6c0       ??1__crt_cached_ptd_host@@QAE@XZ 1000b6c0 f i libucrt:output.obj
 0001:0000a6fc       ??1formatting_buffer@__crt_stdio_output@@QAE@XZ 1000b6fc f i libucrt:output.obj
 0001:0000a716       ??4?$__crt_unique_heap_ptr@DU__crt_internal_free_policy@@@@QAEAAV0@$$QAV0@@Z 1000b716 f i libucrt:output.obj
 0001:0000a7d6       ?crop_zeroes@__crt_stdio_output@@YAXPADQAU__crt_locale_pointers@@@Z 1000b7d6 f i libucrt:output.obj
 0001:0000a836       ?find_next_state@?$output_processor@DV?$stream_output_adapter@D@__crt_stdio_output@@V?$standard_base@DV?$stream_output_adapter@D@__crt_stdio_output@@@2@@__crt_stdio_output@@ABE?AW4state@2@DW432@@Z 1000b836 f i libucrt:output.obj
 0001:0000a836       ?find_next_state@?$output_processor@DV?$string_output_adapter@D@__crt_stdio_output@@V?$standard_base@DV?$string_output_adapter@D@__crt_stdio_output@@@2@@__crt_stdio_output@@ABE?AW4state@2@DW432@@Z 1000b836 f i libucrt:output.obj
 0001:0000a871       ?force_decimal_point@__crt_stdio_output@@YAXPADQAU__crt_locale_pointers@@@Z 1000b871 f i libucrt:output.obj
 0001:0000a8d0       ?force_synchronize_per_thread_data@__crt_cached_ptd_host@@AAEPAU__acrt_ptd@@XZ 1000b8d0 f i libucrt:output.obj
 0001:0000a920       ?get_raw_ptd@__crt_cached_ptd_host@@QAEPAU__acrt_ptd@@XZ 1000b920 f i libucrt:output.obj
 0001:0000a97c       ?parse_int_from_format_string@?$output_processor@DV?$string_output_adapter@D@__crt_stdio_output@@V?$standard_base@DV?$string_output_adapter@D@__crt_stdio_output@@@2@@__crt_stdio_output@@AAE_NQAH@Z 1000b97c f i libucrt:output.obj
 0001:0000a97c       ?parse_int_from_format_string@?$output_processor@DV?$stream_output_adapter@D@__crt_stdio_output@@V?$standard_base@DV?$stream_output_adapter@D@__crt_stdio_output@@@2@@__crt_stdio_output@@AAE_NQAH@Z 1000b97c f i libucrt:output.obj
 0001:0000a9f4       ?process@?$output_processor@DV?$stream_output_adapter@D@__crt_stdio_output@@V?$standard_base@DV?$stream_output_adapter@D@__crt_stdio_output@@@2@@__crt_stdio_output@@QAEHXZ 1000b9f4 f i libucrt:output.obj
 0001:0000aca4       ?process@?$output_processor@DV?$string_output_adapter@D@__crt_stdio_output@@V?$standard_base@DV?$string_output_adapter@D@__crt_stdio_output@@@2@@__crt_stdio_output@@QAEHXZ 1000bca4 f i libucrt:output.obj
 0001:0000af78       ?state_case_size@?$output_processor@DV?$stream_output_adapter@D@__crt_stdio_output@@V?$standard_base@DV?$stream_output_adapter@D@__crt_stdio_output@@@2@@__crt_stdio_output@@AAE_NXZ 1000bf78 f i libucrt:output.obj
 0001:0000b0d1       ?state_case_size@?$output_processor@DV?$string_output_adapter@D@__crt_stdio_output@@V?$standard_base@DV?$string_output_adapter@D@__crt_stdio_output@@@2@@__crt_stdio_output@@AAE_NXZ 1000c0d1 f i libucrt:output.obj
 0001:0000b22a       ?state_case_type@?$output_processor@DV?$stream_output_adapter@D@__crt_stdio_output@@V?$standard_base@DV?$stream_output_adapter@D@__crt_stdio_output@@@2@@__crt_stdio_output@@AAE_NXZ 1000c22a f i libucrt:output.obj
 0001:0000b56c       ?state_case_type@?$output_processor@DV?$string_output_adapter@D@__crt_stdio_output@@V?$standard_base@DV?$string_output_adapter@D@__crt_stdio_output@@@2@@__crt_stdio_output@@AAE_NXZ 1000c56c f i libucrt:output.obj
 0001:0000b8cb       ?to_integer_size@__crt_stdio_output@@YAIW4length_modifier@1@@Z 1000c8cb f i libucrt:output.obj
 0001:0000b91f       ?type_case_Z@?$output_processor@DV?$stream_output_adapter@D@__crt_stdio_output@@V?$standard_base@DV?$stream_output_adapter@D@__crt_stdio_output@@@2@@__crt_stdio_output@@AAE_NXZ 1000c91f f i libucrt:output.obj
 0001:0000b91f       ?type_case_Z@?$output_processor@DV?$string_output_adapter@D@__crt_stdio_output@@V?$standard_base@DV?$string_output_adapter@D@__crt_stdio_output@@@2@@__crt_stdio_output@@AAE_NXZ 1000c91f f i libucrt:output.obj
 0001:0000b982       ?type_case_a@?$output_processor@DV?$stream_output_adapter@D@__crt_stdio_output@@V?$standard_base@DV?$stream_output_adapter@D@__crt_stdio_output@@@2@@__crt_stdio_output@@AAE_NXZ 1000c982 f i libucrt:output.obj
 0001:0000b982       ?type_case_a@?$output_processor@DV?$string_output_adapter@D@__crt_stdio_output@@V?$standard_base@DV?$string_output_adapter@D@__crt_stdio_output@@@2@@__crt_stdio_output@@AAE_NXZ 1000c982 f i libucrt:output.obj
 0001:0000bb13       ?type_case_c_tchar@?$output_processor@DV?$stream_output_adapter@D@__crt_stdio_output@@V?$standard_base@DV?$stream_output_adapter@D@__crt_stdio_output@@@2@@__crt_stdio_output@@AAE_ND@Z 1000cb13 f i libucrt:output.obj
 0001:0000bb13       ?type_case_c_tchar@?$output_processor@DV?$string_output_adapter@D@__crt_stdio_output@@V?$standard_base@DV?$string_output_adapter@D@__crt_stdio_output@@@2@@__crt_stdio_output@@AAE_ND@Z 1000cb13 f i libucrt:output.obj
 0001:0000bba8       ?type_case_n@?$output_processor@DV?$string_output_adapter@D@__crt_stdio_output@@V?$standard_base@DV?$string_output_adapter@D@__crt_stdio_output@@@2@@__crt_stdio_output@@AAE_NXZ 1000cba8 f i libucrt:output.obj
 0001:0000bba8       ?type_case_n@?$output_processor@DV?$stream_output_adapter@D@__crt_stdio_output@@V?$standard_base@DV?$stream_output_adapter@D@__crt_stdio_output@@@2@@__crt_stdio_output@@AAE_NXZ 1000cba8 f i libucrt:output.obj
 0001:0000bc2d       ?type_case_o@?$output_processor@DV?$stream_output_adapter@D@__crt_stdio_output@@V?$standard_base@DV?$stream_output_adapter@D@__crt_stdio_output@@@2@@__crt_stdio_output@@AAE_NXZ 1000cc2d f i libucrt:output.obj
 0001:0000bc2d       ?type_case_o@?$output_processor@DV?$string_output_adapter@D@__crt_stdio_output@@V?$standard_base@DV?$string_output_adapter@D@__crt_stdio_output@@@2@@__crt_stdio_output@@AAE_NXZ 1000cc2d f i libucrt:output.obj
 0001:0000bc4a       ?type_case_p@?$output_processor@DV?$stream_output_adapter@D@__crt_stdio_output@@V?$standard_base@DV?$stream_output_adapter@D@__crt_stdio_output@@@2@@__crt_stdio_output@@AAE_NXZ 1000cc4a f i libucrt:output.obj
 0001:0000bc4a       ?type_case_p@?$output_processor@DV?$string_output_adapter@D@__crt_stdio_output@@V?$standard_base@DV?$string_output_adapter@D@__crt_stdio_output@@@2@@__crt_stdio_output@@AAE_NXZ 1000cc4a f i libucrt:output.obj
 0001:0000bc60       ?type_case_s@?$output_processor@DV?$stream_output_adapter@D@__crt_stdio_output@@V?$standard_base@DV?$stream_output_adapter@D@__crt_stdio_output@@@2@@__crt_stdio_output@@AAE_NXZ 1000cc60 f i libucrt:output.obj
 0001:0000bc60       ?type_case_s@?$output_processor@DV?$string_output_adapter@D@__crt_stdio_output@@V?$standard_base@DV?$string_output_adapter@D@__crt_stdio_output@@@2@@__crt_stdio_output@@AAE_NXZ 1000cc60 f i libucrt:output.obj
 0001:0000bcd2       ?unget@?$c_string_character_source@D@__crt_strtox@@QAEXD@Z 1000ccd2 f i libucrt:output.obj
 0001:0000bd00       ?update_locale_slow@__crt_cached_ptd_host@@AAEXXZ 1000cd00 f i libucrt:output.obj
 0001:0000bd5b       ?validate@?$c_string_character_source@D@__crt_strtox@@QBE_NXZ 1000cd5b f i libucrt:output.obj
 0001:0000bd76       ?validate@?$stream_output_adapter@D@__crt_stdio_output@@QBE_NAAV__crt_cached_ptd_host@@@Z 1000cd76 f i libucrt:output.obj
 0001:0000bdae       ?validate@?$string_output_adapter@D@__crt_stdio_output@@QBE_NAAV__crt_cached_ptd_host@@@Z 1000cdae f i libucrt:output.obj
 0001:0000bddf       ?validate_stream_is_ansi_if_required@?$__acrt_stdio_char_traits@D@@SA_NQAU_iobuf@@@Z 1000cddf f i libucrt:output.obj
 0001:0000be66       ?write_character@?$output_adapter_common@DV?$stream_output_adapter@D@__crt_stdio_output@@@__crt_stdio_output@@QBEXDQAHAAV__crt_cached_ptd_host@@@Z 1000ce66 f i libucrt:output.obj
 0001:0000be88       ?write_character_without_count_update@?$stream_output_adapter@D@__crt_stdio_output@@QBE_NDAAV__crt_cached_ptd_host@@@Z 1000ce88 f i libucrt:output.obj
 0001:0000bec2       ?write_string@?$stream_output_adapter@D@__crt_stdio_output@@QBEXQBDHQAHAAV__crt_cached_ptd_host@@@Z 1000cec2 f i libucrt:output.obj
 0001:0000beee       ?write_string@?$string_output_adapter@D@__crt_stdio_output@@QBEXQBDHQAHAAV__crt_cached_ptd_host@@@Z 1000ceee f i libucrt:output.obj
 0001:0000bf55       ?write_string_impl@?$output_adapter_common@DV?$stream_output_adapter@D@__crt_stdio_output@@@__crt_stdio_output@@IBEXQBDHQAHAAV__crt_cached_ptd_host@@@Z 1000cf55 f i libucrt:output.obj
 0001:0000bfd4       ___acrt_locale_get_ctype_array_value 1000cfd4 f i libucrt:output.obj
 0001:0000bff6       ___stdio_common_vfprintf   1000cff6 f   libucrt:output.obj
 0001:0000c09a       ___stdio_common_vsprintf   1000d09a f   libucrt:output.obj
 0001:0000c200       _fclose                    1000d200 f   libucrt:fclose.obj
 0001:0000c2e7       _fopen                     1000d2e7 f   libucrt:fopen.obj
 0001:0000c3ea       _getenv                    1000d3ea f   libucrt:getenv.obj
 0001:0000c400       _strcmp                    1000d400 f   libucrt:strcmp.obj
 0001:0000c490       _strcpy                    1000d490 f   libucrt:strcat.obj
 0001:0000c4a0       _strcat                    1000d4a0 f   libucrt:strcat.obj
 0001:0000c588       _free                      1000d588 f   libucrt:free.obj
 0001:0000c5a3       _malloc                    1000d5a3 f   libucrt:malloc.obj
 0001:0000c5ae       _wcsncpy                   1000d5ae f   libucrt:wcsncpy.obj
 0001:0000c5ee       ??$__crt_fast_decode_pointer@P6GXPAXK0@Z@@YAP6GXPAXK0@ZQ6GX0K0@Z@Z 1000d5ee f i libucrt:exit.obj
 0001:0000c5ee       ??$__crt_fast_decode_pointer@P6AXH@Z@@YAP6AXH@ZQ6AXH@Z@Z 1000d5ee f i libucrt:signal.obj
 0001:0000c5ee       ??$__crt_fast_decode_pointer@P6AHI@Z@@YAP6AHI@ZQ6AHI@Z@Z 1000d5ee f i libucrt:new_handler.obj
 0001:0000c609       ___acrt_initialize_new_handler 1000d609 f   libucrt:new_handler.obj
 0001:0000c618       __callnewh                 1000d618 f   libucrt:new_handler.obj
 0001:0000c644       __query_new_handler        1000d644 f   libucrt:new_handler.obj
 0001:0000c69b       __initterm                 1000d69b f   libucrt:initterm.obj
 0001:0000c6c6       __initterm_e               1000d6c6 f   libucrt:initterm.obj
 0001:0000c6f4       __seh_filter_dll           1000d6f4 f   libucrt:exception_filter.obj
 0001:0000c714       __seh_filter_exe           1000d714 f   libucrt:exception_filter.obj
 0001:0000cb34       ___acrt_initialize_thread_local_exit_callback 1000db34 f   libucrt:exit.obj
 0001:0000cb43       __cexit                    1000db43 f   libucrt:exit.obj
 0001:0000cb52       __exit                     1000db52 f   libucrt:exit.obj
 0001:0000cb68       __is_c_termination_complete 1000db68 f   libucrt:exit.obj
 0001:0000ce20       ___acrt_allocate_buffer_for_argv 1000de20 f   libucrt:argv_parsing.obj
 0001:0000ce6f       __configure_narrow_argv    1000de6f f   libucrt:argv_parsing.obj
 0001:0000d0ca       ___dcrt_get_or_create_narrow_environment_nolock 1000e0ca f   libucrt:environment_initialization.obj
 0001:0000d0cf       ___dcrt_uninitialize_environments_nolock 1000e0cf f   libucrt:environment_initialization.obj
 0001:0000d120       __initialize_narrow_environment 1000e120 f   libucrt:environment_initialization.obj
 0001:0000d25a       __execute_onexit_table     1000e25a f   libucrt:onexit.obj
 0001:0000d298       __initialize_onexit_table  1000e298 f   libucrt:onexit.obj
 0001:0000d2e8       ___acrt_uninitialize_command_line 1000e2e8 f   libucrt:argv_data.obj
 0001:0000d3bf       ___acrt_initialize         1000e3bf f   libucrt:initialization.obj
 0001:0000d3d1       ___acrt_thread_attach      1000e3d1 f   libucrt:initialization.obj
 0001:0000d3dc       ___acrt_thread_detach      1000e3dc f   libucrt:initialization.obj
 0001:0000d3e4       ___acrt_uninitialize       1000e3e4 f   libucrt:initialization.obj
 0001:0000d414       ___acrt_uninitialize_critical 1000e414 f   libucrt:initialization.obj
 0001:0000d426       _terminate                 1000e426 f   libucrt:terminate.obj
 0001:0000d462       _strcpy_s                  1000e462 f   libucrt:strcpy_s.obj
 0001:0000d4c0       _strncmp                   1000e4c0 f   libucrt:strncmp.obj
 0001:0000d538       _abort                     1000e538 f   libucrt:abort.obj
 0001:0000d57c       _calloc                    1000e57c f   libucrt:calloc.obj
 0001:0000d587       _wcsncmp                   1000e587 f   libucrt:wcsncmp.obj
 0001:0000d5c1       ?check_synchronize_global_state_index@__crt_cached_ptd_host@@AAEIXZ 1000e5c1 f i libucrt:invalid_parameter.obj
 0001:0000d5ea       ___acrt_call_reportfault   1000e5ea f   libucrt:invalid_parameter.obj
 0001:0000d723       ___acrt_initialize_invalid_parameter_handler 1000e723 f   libucrt:invalid_parameter.obj
 0001:0000d732       __invalid_parameter        1000e732 f   libucrt:invalid_parameter.obj
 0001:0000d769       __invalid_parameter_internal 1000e769 f   libucrt:invalid_parameter.obj
 0001:0000d7e6       __invalid_parameter_noinfo 1000e7e6 f   libucrt:invalid_parameter.obj
 0001:0000d7f6       __invoke_watson            1000e7f6 f   libucrt:invalid_parameter.obj
 0001:0000d82a       ___acrt_errno_from_os_error 1000e82a f   libucrt:errno.obj
 0001:0000d86d       ___acrt_errno_map_os_error 1000e86d f   libucrt:errno.obj
 0001:0000d890       ___acrt_errno_map_os_error_ptd 1000e890 f   libucrt:errno.obj
 0001:0000d8b4       ___doserrno                1000e8b4 f   libucrt:errno.obj
 0001:0000d8c7       __errno                    1000e8c7 f   libucrt:errno.obj
 0001:0000d8da       __calloc_base              1000e8da f   libucrt:calloc_base.obj
 0001:0000d937       __free_base                1000e937 f   libucrt:free_base.obj
 0001:0000db29       ___acrt_AppPolicyGetProcessTerminationMethodInternal@4 1000eb29 f   libucrt:winapi_thunks.obj
 0001:0000db69       ___acrt_AreFileApisANSI@0  1000eb69 f   libucrt:winapi_thunks.obj
 0001:0000db88       ___acrt_CompareStringEx@36 1000eb88 f   libucrt:winapi_thunks.obj
 0001:0000dbe5       ___acrt_FlsAlloc@4         1000ebe5 f   libucrt:winapi_thunks.obj
 0001:0000dc24       ___acrt_FlsFree@4          1000ec24 f   libucrt:winapi_thunks.obj
 0001:0000dc63       ___acrt_FlsGetValue@4      1000ec63 f   libucrt:winapi_thunks.obj
 0001:0000dca2       ___acrt_FlsSetValue@8      1000eca2 f   libucrt:winapi_thunks.obj
 0001:0000dce4       ___acrt_InitializeCriticalSectionEx@12 1000ece4 f   libucrt:winapi_thunks.obj
 0001:0000dd2f       ___acrt_LCMapStringEx@36   1000ed2f f   libucrt:winapi_thunks.obj
 0001:0000dd8c       ___acrt_LocaleNameToLCID@8 1000ed8c f   libucrt:winapi_thunks.obj
 0001:0000ddbd       ___acrt_initialize_winapi_thunks 1000edbd f   libucrt:winapi_thunks.obj
 0001:0000ddd1       ___acrt_uninitialize_winapi_thunks 1000edd1 f   libucrt:winapi_thunks.obj
 0001:0000de07       __fcloseall                1000ee07 f   libucrt:closeall.obj
 0001:0000e08b       ___acrt_stdio_flush_nolock 1000f08b f   libucrt:fflush.obj
 0001:0000e0f4       __fflush_nolock            1000f0f4 f   libucrt:fflush.obj
 0001:0000e159       __flushall                 1000f159 f   libucrt:fflush.obj
 0001:0000e162       ___acrt_stdio_free_buffer_nolock 1000f162 f   libucrt:_freebuf.obj
 0001:0000e308       ___acrt_initialize_lowio   1000f308 f   libucrt:ioinit.obj
 0001:0000e368       ___acrt_uninitialize_lowio 1000f368 f   libucrt:ioinit.obj
 0001:0000e394       __malloc_base              1000f394 f   libucrt:malloc_base.obj
 0001:0000e3e2       _strnlen                   1000f3e2 f   libucrt:strnlen.obj
 0001:0000e504       _wcsnlen                   1000f504 f   libucrt:strnlen.obj
 0001:0000e6b4       ___acrt_update_locale_info 1000f6b4 f   libucrt:locale_update.obj
 0001:0000e6e1       ___acrt_update_locale_info_explicit 1000f6e1 f   libucrt:locale_update.obj
 0001:0000e712       ___acrt_update_multibyte_info 1000f712 f   libucrt:locale_update.obj
 0001:0000e73f       ___acrt_update_multibyte_info_explicit 1000f73f f   libucrt:locale_update.obj
 0001:0000e770       ?__acrt_fp_classify@@YA?AW4__acrt_fp_class@@ABN@Z 1000f770 f i libucrt:cvt.obj
 0001:0000f148       ___acrt_fp_format          10010148 f   libucrt:cvt.obj
 0001:0000f2c9       __wctomb_internal          100102c9 f   libucrt:wctomb.obj
 0001:0000f433       __mbtowc_internal          10010433 f   libucrt:mbtowc.obj
 0001:0000f566       __fileno                   10010566 f   libucrt:fileno.obj
 0001:0000f58d       __get_printf_count_output  1001058d f   libucrt:printf_count_output.obj
 0001:0000f5a2       __fputc_nolock_internal    100105a2 f   libucrt:fputc.obj
 0001:0000f5cf       ___acrt_should_use_temporary_buffer 100105cf f   libucrt:_sftbuf.obj
 0001:0000f60d       ___acrt_stdio_begin_temporary_buffering_nolock 1001060d f   libucrt:_sftbuf.obj
 0001:0000f6b8       ___acrt_stdio_end_temporary_buffering_nolock 100106b8 f   libucrt:_sftbuf.obj
 0001:0000fa34       ___acrt_freeptd            10010a34 f   libucrt:per_thread_data.obj
 0001:0000fa60       ___acrt_getptd             10010a60 f   libucrt:per_thread_data.obj
 0001:0000fb1b       ___acrt_getptd_head        10010b1b f   libucrt:per_thread_data.obj
 0001:0000fbb1       ___acrt_getptd_noexit      10010bb1 f   libucrt:per_thread_data.obj
 0001:0000fc62       ___acrt_getptd_noexit_explicit 10010c62 f   libucrt:per_thread_data.obj
 0001:0000fd05       ___acrt_initialize_ptd     10010d05 f   libucrt:per_thread_data.obj
 0001:0000fd31       ___acrt_uninitialize_ptd   10010d31 f   libucrt:per_thread_data.obj
 0001:0000fdb9       ___acrt_set_locale_changed 10010db9 f   libucrt:wsetlocale.obj
 0001:0000fdc4       ___acrt_uninitialize_locale 10010dc4 f   libucrt:wsetlocale.obj
 0001:0000fe7c       __close_internal           10010e7c f   libucrt:close.obj
 0001:0000ff1f       __close_nolock             10010f1f f   libucrt:close.obj
 0001:0000ff4f       __close_nolock_internal    10010f4f f   libucrt:close.obj
 0001:0000ffef       ?__acrt_stdio_allocate_stream@@YA?AV__crt_stdio_stream@@XZ 10010fef f   libucrt:stream.obj
 0001:00010058       ?__acrt_stdio_free_stream@@YAXV__crt_stdio_stream@@@Z 10011058 f   libucrt:stream.obj
 0001:00010155       ??$__acrt_stdio_parse_mode@D@@YA?AU__acrt_stdio_stream_mode@@QBD@Z 10011155 f i libucrt:openfile.obj
 0001:00010402       ?__acrt_stdio_parse_mode_D@@YA_NAAU__acrt_stdio_stream_mode@@@Z 10011402 f i libucrt:openfile.obj
 0001:0001041d       ?__acrt_stdio_parse_mode_T@@YA_NAAU__acrt_stdio_stream_mode@@@Z 1001141d f i libucrt:openfile.obj
 0001:0001043c       ?__acrt_stdio_parse_mode_b@@YA_NAAU__acrt_stdio_stream_mode@@@Z 1001143c f i libucrt:openfile.obj
 0001:0001045c       ?__acrt_stdio_parse_mode_c@@YA_NAAU__acrt_stdio_stream_mode@@AA_N@Z 1001145c f i libucrt:openfile.obj
 0001:0001047e       ?__acrt_stdio_parse_mode_n@@YA_NAAU__acrt_stdio_stream_mode@@AA_N@Z 1001147e f i libucrt:openfile.obj
 0001:000104a0       ?__acrt_stdio_parse_mode_plus@@YA_NAAU__acrt_stdio_stream_mode@@AA_N@Z 100114a0 f i libucrt:openfile.obj
 0001:000104d6       ?__acrt_stdio_parse_mode_t@@YA_NAAU__acrt_stdio_stream_mode@@@Z 100114d6 f i libucrt:openfile.obj
 0001:000104f6       ?__acrt_stdio_parse_mode_x@@YA_NAAU__acrt_stdio_stream_mode@@@Z 100114f6 f i libucrt:openfile.obj
 0001:00010516       __openfile                 10011516 f   libucrt:openfile.obj
 0001:00010521       ??0_LocaleUpdate@@QAE@QAU__crt_locale_pointers@@@Z 10011521 f i libucrt:wcsnicol.obj
 0001:000105a3       __strnicoll                100115a3 f   libucrt:strnicol.obj
 0001:000105cc       __strnicoll_l              100115cc f   libucrt:strnicol.obj
 0001:00010694       ___acrt_initialize_locks   10011694 f   libucrt:locks.obj
 0001:000106d5       ___acrt_lock               100116d5 f   libucrt:locks.obj
 0001:000106ec       ___acrt_uninitialize_locks 100116ec f   libucrt:locks.obj
 0001:0001071d       ___acrt_unlock             1001171d f   libucrt:locks.obj
 0001:00010734       ___acrt_app_verifier_enabled 10011734 f   libucrt:peb_access.obj
 0001:00010746       ___acrt_is_secure_process  10011746 f   libucrt:peb_access.obj
 0001:00010759       ___acrt_get_process_end_policy 10011759 f   libucrt:win_policies.obj
 0001:00010798       ??$__acrt_convert_wcs_mbs_cp@D_WV<lambda_62f6974d9771e494a5ea317cc32e971c>@@U__crt_win32_buffer_internal_dynamic_resizing@@@@YAHQBDAAV?$__crt_win32_buffer@_WU__crt_win32_buffer_internal_dynamic_resizing@@@@ABV<lambda_62f6974d9771e494a5ea317cc32e971c>@@I@Z 10011798 f i libucrt:argv_wildcards.obj
 0001:0001084a       ??$__acrt_convert_wcs_mbs_cp@_WDV<lambda_28bda7af82a03b66c1cb3803a755f95d>@@U__crt_win32_buffer_internal_dynamic_resizing@@@@YAHQB_WAAV?$__crt_win32_buffer@DU__crt_win32_buffer_internal_dynamic_resizing@@@@ABV<lambda_28bda7af82a03b66c1cb3803a755f95d>@@I@Z 1001184a f i libucrt:argv_wildcards.obj
 0001:00010910       ??$__acrt_mbs_to_wcs_cp@U__crt_win32_buffer_internal_dynamic_resizing@@@@YAHQBDAAV?$__crt_win32_buffer@_WU__crt_win32_buffer_internal_dynamic_resizing@@@@I@Z 10011910 f i libucrt:argv_wildcards.obj
 0001:00010e05       ??R<lambda_0fec1a7b3f42a53036604e18c2d5e07e>@@QBE@IQB_WQADI@Z 10011e05 f i libucrt:getmodulefilenamea.obj
 0001:00010e05       ??R<lambda_28bda7af82a03b66c1cb3803a755f95d>@@QBE@IQB_WQADI@Z 10011e05 f i libucrt:argv_wildcards.obj
 0001:00010e29       ?__acrt_get_utf8_acp_compatibility_codepage@@YAIXZ 10011e29 f i libucrt:argv_wildcards.obj
 0001:00010e68       ?_deallocate@?$__crt_win32_buffer@DU__crt_win32_buffer_internal_dynamic_resizing@@@@AAEXXZ 10011e68 f i libucrt:argv_wildcards.obj
 0001:00010e68       ?_deallocate@?$__crt_win32_buffer@_WU__crt_win32_buffer_internal_dynamic_resizing@@@@AAEXXZ 10011e68 f i libucrt:argv_wildcards.obj
 0001:00010e82       ?allocate@?$__crt_win32_buffer@DU__crt_win32_buffer_internal_dynamic_resizing@@@@QAEHI@Z 10011e82 f i libucrt:argv_wildcards.obj
 0001:00010ebe       ?allocate@?$__crt_win32_buffer@_WU__crt_win32_buffer_internal_dynamic_resizing@@@@QAEHI@Z 10011ebe f i libucrt:argv_wildcards.obj
 0001:00010efd       ?allocate@__crt_win32_buffer_internal_dynamic_resizing@@SAHQAPAXIABV__crt_win32_buffer_empty_debug_info@@@Z 10011efd f i libucrt:argv_wildcards.obj
 0001:00010fa3       ___acrt_expand_narrow_argv_wildcards 10011fa3 f   libucrt:argv_wildcards.obj
 0001:00010fae       ??$__acrt_convert_wcs_mbs_cp@_WDV<lambda_0fec1a7b3f42a53036604e18c2d5e07e>@@U__crt_win32_buffer_no_resizing@@@@YAHQB_WAAV?$__crt_win32_buffer@DU__crt_win32_buffer_no_resizing@@@@ABV<lambda_0fec1a7b3f42a53036604e18c2d5e07e>@@I@Z 10011fae f i libucrt:getmodulefilenamea.obj
 0001:00011070       ?allocate@?$__crt_win32_buffer@DU__crt_win32_buffer_no_resizing@@@@QAEHI@Z 10012070 f i libucrt:getmodulefilenamea.obj
 0001:00011097       ?set_to_nullptr@?$__crt_win32_buffer@DU__crt_win32_buffer_no_resizing@@@@QAEXXZ 10012097 f i libucrt:getmodulefilenamea.obj
 0001:000110ab       ___acrt_GetModuleFileNameA 100120ab f   libucrt:getmodulefilenamea.obj
 0001:000116c8       ___acrt_initialize_multibyte 100126c8 f   libucrt:mbctype.obj
 0001:00011710       ___acrt_update_thread_multibyte_data 10012710 f   libucrt:mbctype.obj
 0001:00011723       __setmbcp_nolock           10012723 f   libucrt:mbctype.obj
 0001:000119f9       __ismbblead                100129f9 f   libucrt:ismbbyte.obj
 0001:00011a11       ___acrt_initialize_command_line 10012a11 f   libucrt:argv_data.obj
 0001:00011ac2       ___acrt_MultiByteToWideChar 10012ac2 f   libucrt:multibytetowidechar.obj
 0001:00011b7c       ___acrt_WideCharToMultiByte 10012b7c f   libucrt:widechartomultibyte.obj
 0001:00011c1f       ___dcrt_get_narrow_environment_from_os 10012c1f f   libucrt:get_environment_from_os.obj
 0001:0001203e       ___dcrt_set_variable_in_narrow_environment_nolock 1001303e f   libucrt:setenv.obj
 0001:00012049       __recalloc_base            10013049 f   libucrt:recalloc.obj
 0001:000120b6       ___acrt_initialize_heap    100130b6 f   libucrt:heap_handle.obj
 0001:000120c7       ___acrt_uninitialize_heap  100130c7 f   libucrt:heap_handle.obj
 0001:000120d1       ___acrt_execute_initializers 100130d1 f   libucrt:shared_initialization.obj
 0001:00012139       ___acrt_execute_uninitializers 10013139 f   libucrt:shared_initialization.obj
 0001:0001223c       ___acrt_get_sigabrt_handler 1001323c f   libucrt:signal.obj
 0001:00012263       ___acrt_initialize_signal_handlers 10013263 f   libucrt:signal.obj
 0001:00012281       _raise                     10013281 f   libucrt:signal.obj
 0001:00012473       ___acrt_has_user_matherr   10013473 f   libucrt:matherr.obj
 0001:00012490       ___acrt_initialize_user_matherr 10013490 f   libucrt:matherr.obj
 0001:0001249f       ___acrt_invoke_user_matherr 1001349f f   libucrt:matherr.obj
 0001:000124d5       __query_new_mode           100134d5 f   libucrt:new_mode.obj
 0001:0001252c       ___acrt_DownlevelLocaleNameToLCID 1001352c f   libucrt:lcidtoname_downlevel.obj
 0001:000125fa       __commit                   100135fa f   libucrt:commit.obj
 0001:00012e19       __write                    10013e19 f   libucrt:write.obj
 0001:00012e50       __write_internal           10013e50 f   libucrt:write.obj
 0001:00012f61       __write_nolock             10013f61 f   libucrt:write.obj
 0001:0001317d       ___acrt_lowio_create_handle_array 1001417d f   libucrt:osfinfo.obj
 0001:000131f8       ___acrt_lowio_destroy_handle_array 100141f8 f   libucrt:osfinfo.obj
 0001:0001322d       ___acrt_lowio_ensure_fh_exists 1001422d f   libucrt:osfinfo.obj
 0001:000132cb       ___acrt_lowio_lock_fh      100142cb f   libucrt:osfinfo.obj
 0001:000132ee       ___acrt_lowio_set_os_handle 100142ee f   libucrt:osfinfo.obj
 0001:00013380       ___acrt_lowio_unlock_fh    10014380 f   libucrt:osfinfo.obj
 0001:000133a3       __alloc_osfhnd             100143a3 f   libucrt:osfinfo.obj
 0001:000134b6       __free_osfhnd              100144b6 f   libucrt:osfinfo.obj
 0001:00013547       __get_osfhandle            10014547 f   libucrt:osfinfo.obj
 0001:000135b1       ___acrt_add_locale_ref     100145b1 f   libucrt:locale_refcounting.obj
 0001:0001362e       ___acrt_free_locale        1001462e f   libucrt:locale_refcounting.obj
 0001:00013776       ___acrt_locale_add_lc_time_reference 10014776 f   libucrt:locale_refcounting.obj
 0001:0001379f       ___acrt_locale_free_lc_time_if_unreferenced 1001479f f   libucrt:locale_refcounting.obj
 0001:000137d0       ___acrt_locale_release_lc_time_reference 100147d0 f   libucrt:locale_refcounting.obj
 0001:000137f9       ___acrt_release_locale_ref 100147f9 f   libucrt:locale_refcounting.obj
 0001:0001387a       ___acrt_update_thread_locale_data 1001487a f   libucrt:locale_refcounting.obj
 0001:000138fb       __updatetlocinfoEx_nolock  100148fb f   libucrt:locale_refcounting.obj
 0001:000139fc       ___acrt_fp_strflt_to_string 100149fc f   libucrt:_fptostr.obj
 0001:00013b00       ?divide@__crt_strtox@@YA_KAAUbig_integer@1@ABU21@@Z 10014b00 f i libucrt:cfout.obj
 0001:00013fab       ___acrt_fltout             10014fab f   libucrt:cfout.obj
 0001:00015593       _fegetround                10016593 f   libucrt:fegetround.obj
 0001:000155a0       ?__c32rtomb_utf8@__crt_mbstring@@YAIPAD_UPAU_Mbstatet@@AAV__crt_cached_ptd_host@@@Z 100165a0 f   libucrt:c32rtomb.obj
 0001:0001567c       ?__mbrtowc_utf8@__crt_mbstring@@YAIPA_WPBDIPAU_Mbstatet@@AAV__crt_cached_ptd_host@@@Z 1001667c f   libucrt:mbrtowc.obj
 0001:000156bf       ?__mbsrtowcs_utf8@__crt_mbstring@@YAIPA_WPAPBDIPAU_Mbstatet@@AAV__crt_cached_ptd_host@@@Z 100166bf f   libucrt:mbrtowc.obj
 0001:00015a14       ___acrt_stdio_flush_and_write_narrow_nolock 10016a14 f   libucrt:_flsbuf.obj
 0001:00015a1f       __isatty                   10016a1f f   libucrt:isatty.obj
 0001:00015a75       ___acrt_locale_free_monetary 10016a75 f   libucrt:initmon.obj
 0001:00015b73       ___acrt_locale_free_numeric 10016b73 f   libucrt:initnum.obj
 0001:00015c01       ___acrt_locale_free_time   10016c01 f   libucrt:inittime.obj
 0001:00015ce5       ___acrt_GetStringTypeA     10016ce5 f   libucrt:getstringtypea.obj
 0001:00015de6       __freea_crt                10016de6 f i libucrt:getstringtypea.obj
 0001:00015e06       ___ascii_wcsnicmp          10016e06 f   libucrt:wcsnicmp.obj
 0001:00015e55       __strnicmp                 10016e55 f   libucrt:strnicmp.obj
 0001:00015ec2       __strnicmp_l               10016ec2 f   libucrt:strnicmp.obj
 0001:00016577       __sopen_nolock             10017577 f   libucrt:open.obj
 0001:000165e5       __sopen_s                  100175e5 f   libucrt:open.obj
 0001:00016605       __wsopen_nolock            10017605 f   libucrt:open.obj
 0001:00016bce       ___acrt_CompareStringA     10017bce f   libucrt:comparestringa.obj
 0001:00016c20       _qsort                     10017c20 f   libucrt:qsort.obj
 0001:000171c5       _strncpy_s                 100181c5 f   libucrt:strncpy_s.obj
 0001:000171d0       _strpbrk                   100181d0 f   libucrt:strpbrk.obj
 0001:00017210       __mbsdec                   10018210 f   libucrt:mbsdec.obj
 0001:00017227       __mbsdec_l                 10018227 f   libucrt:mbsdec.obj
 0001:000174a3       ___acrt_LCMapStringA       100184a3 f   libucrt:lcmapstringa.obj
 0001:000174fb       ___acrt_SetEnvironmentVariableA 100184fb f   libucrt:setenvironmentvariablea.obj
 0001:00017590       __msize_base               10018590 f   libucrt:msize.obj
 0001:000175c3       __realloc_base             100185c3 f   libucrt:realloc_base.obj
 0001:000177d4       __lseeki64                 100187d4 f   libucrt:lseek.obj
 0001:00017814       __lseeki64_nolock          10018814 f   libucrt:lseek.obj
 0001:00017854       __lseeki64_nolock_internal 10018854 f   libucrt:lseek.obj
 0001:00017872       __putwch_nolock            10018872 f   libucrt:putwch.obj
 0001:00017d80       __read_nolock              10018d80 f   libucrt:read.obj
 0001:0001810b       __query_app_type           1001910b f   libucrt:report_runtime_error.obj
 0001:00018111       __controlfp_s              10019111 f   libucrt:contrlfp.obj
 0001:00018170       _fegetenv                  10019170 f   libucrt:fegetenv.obj
 0001:0001818d       _fesetenv                  1001918d f   libucrt:fesetenv.obj
 0001:000181d9       _feholdexcept              100191d9 f   libucrt:feholdexcept.obj
 0001:00018230       __CIlog10                  10019230 f   libucrt:log10_impl.obj
 0001:0001826b       __CIlog10_default          1001926b f   libucrt:log10_impl.obj
 0001:0001827f       __log10_default            1001927f     libucrt:log10_impl.obj
 0001:00018340       _ceil                      10019340 f   libucrt:ceil_pentium4.obj
 0001:00018380       __ceil_pentium4            10019380 f   libucrt:ceil_pentium4.obj
 0001:00018726       ___acrt_fenv_get_common_round_control 10019726 f   libucrt:_fenvutils.obj
 0001:00018748       ___acrt_fenv_get_control   10019748 f   libucrt:_fenvutils.obj
 0001:000187c8       ___acrt_fenv_get_status    100197c8 f   libucrt:_fenvutils.obj
 0001:00018872       ___acrt_fenv_set_control   10019872 f   libucrt:_fenvutils.obj
 0001:000188ed       ___acrt_fenv_set_status    100198ed f   libucrt:_fenvutils.obj
 0001:000189e9       ?reset_and_return@__crt_mbstring@@YAIIPAU_Mbstatet@@@Z 100199e9 f   libucrt:common_utf8.obj
 0001:000189fd       ?return_illegal_sequence@__crt_mbstring@@YAIPAU_Mbstatet@@AAV__crt_cached_ptd_host@@@Z 100199fd f   libucrt:common_utf8.obj
 0001:00018a1f       ?__mbrtoc32_utf8@__crt_mbstring@@YAIPA_UPBDIPAU_Mbstatet@@AAV__crt_cached_ptd_host@@@Z 10019a1f f   libucrt:mbrtoc32.obj
 0001:00018bd0       ___acrt_stdio_allocate_buffer_nolock 10019bd0 f   libucrt:_getbuf.obj
 0001:00018c30       ___ascii_strnicmp          10019c30 f   libucrt:_strnicm.obj
 0001:00018c91       __get_fmode                10019c91 f   libucrt:setmode.obj
 0001:00018cbe       __setmode_nolock           10019cbe f   libucrt:setmode.obj
 0001:00018d8d       ??0__crt_seek_guard@@QAE@H_J@Z 10019d8d f i libucrt:chsize.obj
 0001:00018dda       __chsize_nolock            10019dda f   libucrt:chsize.obj
 0001:00018e11       __chsize_nolock_internal   10019e11 f   libucrt:chsize.obj
 0001:00018fa8       ___strncnt                 10019fa8 f   libucrt:strncnt.obj
 0001:00018fe3       ___dcrt_lowio_ensure_console_output_initialized 10019fe3 f   libucrt:initcon.obj
 0001:00019002       ___dcrt_terminate_console_output 1001a002 f   libucrt:initcon.obj
 0001:00019019       ___dcrt_write_console      1001a019 f   libucrt:initcon.obj
 0001:00019115       __clearfp                  1001a115 f   libucrt:ieee87.obj
 0001:000191f3       __control87                1001a1f3 f   libucrt:ieee87.obj
 0001:00019592       ___acrt_initialize_sse2    1001a592 f   libucrt:mathfcns.obj
 0001:000195b0       __CIlog10_pentium4         1001a5b0 f   libucrt:log10_pentium4.obj
 0001:000195c8       __log10_pentium4           1001a5c8     libucrt:log10_pentium4.obj
 0001:00019860       __fFEXP                    1001a860 f   libucrt:87tran.obj
 0001:000198b7       __rtinfpopse               1001a8b7     libucrt:87tran.obj
 0001:000198b9       __rtinfnpopse              1001a8b9     libucrt:87tran.obj
 0001:000198c9       __fFLN                     1001a8c9     libucrt:87tran.obj
 0001:0001997e       __rtinfpop                 1001a97e     libucrt:87tran.obj
 0001:00019980       __rtinfnpop                1001a980     libucrt:87tran.obj
 0001:00019990       __rtforexpinf              1001a990 f   libucrt:87tran.obj
 0001:0001999d       __ffexpm1                  1001a99d     libucrt:87tran.obj
 0001:00019a50       __trandisp1                1001aa50 f   libucrt:87disp.obj
 0001:00019ac5       __trandisp2                1001aac5 f   libucrt:87disp.obj
 0001:00019b5f       __rttospopde               1001ab5f     libucrt:87disp.obj
 0001:00019b64       __rttospop                 1001ab64     libucrt:87disp.obj
 0001:00019b70       __rtnospop                 1001ab70 f   libucrt:87disp.obj
 0001:00019b80       __rttosnpop                1001ab80 f   libucrt:87disp.obj
 0001:00019b81       __rtnospopde               1001ab81     libucrt:87disp.obj
 0001:00019b88       __rtzeropop                1001ab88     libucrt:87disp.obj
 0001:00019b8a       __rtzeronpop               1001ab8a     libucrt:87disp.obj
 0001:00019b90       __rtzerospop               1001ab90 f   libucrt:87disp.obj
 0001:00019b9d       __rtonepop                 1001ab9d     libucrt:87disp.obj
 0001:00019ba0       __rtonenpop                1001aba0 f   libucrt:87disp.obj
 0001:00019bb0       __tosnan1                  1001abb0 f   libucrt:87disp.obj
 0001:00019be0       __nosnan2                  1001abe0 f   libucrt:87disp.obj
 0001:00019bf0       __tosnan2                  1001abf0 f   libucrt:87disp.obj
 0001:00019c20       __nan2                     1001ac20 f   libucrt:87disp.obj
 0001:00019c60       __rtindfpop                1001ac60 f   libucrt:87disp.obj
 0001:00019c62       __rtindfnpop               1001ac62     libucrt:87disp.obj
 0001:00019c73       __rttosnpopde              1001ac73     libucrt:87disp.obj
 0001:00019c80       __rtatan2inf               1001ac80 f   libucrt:87disp.obj
 0001:00019c9d       __rtchsifneg               1001ac9d     libucrt:87disp.obj
 0001:00019cb0       __twoToTOS                 1001acb0 f   libucrt:common.obj
 0001:00019cc5       __load_CW                  1001acc5 f   libucrt:common.obj
 0001:00019cdc       __convertTOStoQNaN         1001acdc f   libucrt:common.obj
 0001:00019cf5       __fload_withFB             1001acf5 f   libucrt:common.obj
 0001:00019d38       __checkTOS_withFB          1001ad38 f   libucrt:common.obj
 0001:00019d4e       __fast_exit                1001ad4e f   libucrt:common.obj
 0001:00019d5b       __math_exit                1001ad5b f   libucrt:common.obj
 0001:00019d85       __check_overflow_exit      1001ad85 f   libucrt:common.obj
 0001:00019d99       __check_range_exit         1001ad99 f   libucrt:common.obj
 0001:00019e40       __startTwoArgErrorHandling 1001ae40 f   libucrt:genexcep.obj
 0001:00019e57       __startOneArgErrorHandling 1001ae57 f   libucrt:genexcep.obj
 0001:00019e93       ___libm_error_support      1001ae93 f   libucrt:libm_error.obj
 0001:0001a087       __ceil_default             1001b087 f   libucrt:ceil.obj
 0001:0001a145       ___acrt_initialize_fmode   1001b145 f   libucrt:txtmode.obj
 0001:0001a15b       ___set_fpsr_sse2           1001b15b f   libucrt:fpctrl.obj
 0001:0001a1db       __clrfp                    1001b1db f   libucrt:fpctrl.obj
 0001:0001a1ec       __ctrlfp                   1001b1ec f   libucrt:fpctrl.obj
 0001:0001a216       __set_statfp               1001b216 f   libucrt:fpctrl.obj
 0001:0001a26f       __statfp                   1001b26f f   libucrt:fpctrl.obj
 0001:0001a27f       __d_inttype                1001b27f f   libucrt:powhlp.obj
 0001:0001a2e7       __powhlp                   1001b2e7 f   libucrt:powhlp.obj
 0001:0001a412       __87except                 1001b412 f   libucrt:87except.obj
 0001:0001a522       __frnd                     1001b522 f   libucrt:frnd.obj
 0001:0001a536       __errcode                  1001b536 f   libucrt:fpexcept.obj
 0001:0001a56a       __except1                  1001b56a f   libucrt:fpexcept.obj
 0001:0001a638       __handle_exc               1001b638 f   libucrt:fpexcept.obj
 0001:0001a8b8       __raise_exc                1001b8b8 f   libucrt:fpexcept.obj
 0001:0001a8db       __raise_exc_ex             1001b8db f   libucrt:fpexcept.obj
 0001:0001abcc       __set_errno_from_matherr   1001bbcc f   libucrt:fpexcept.obj
 0001:0001abfd       __umatherr                 1001bbfd f   libucrt:fpexcept.obj
 0001:0001ac9d       __decomp                   1001bc9d f   libucrt:util.obj
 0001:0001ad6f       __set_exp                  1001bd6f f   libucrt:util.obj
 0001:0001ad9c       __sptype                   1001bd9c f   libucrt:util.obj
 0001:0001adff       __fpclass                  1001bdff f   libucrt:ieeemisc.obj
 0001:0001aea3       _IsProcessorFeaturePresent@4 1001bea3 f   kernel32:KERNEL32.dll
 0001:0001aeb0       __FindPESection            1001beb0 f   LIBCMT:pesect.obj
 0001:0001af00       __IsNonwritableInCurrentImage 1001bf00 f   LIBCMT:pesect.obj
 0001:0001afc0       __ValidateImageBase        1001bfc0 f   LIBCMT:pesect.obj
 0001:0001aff3       __EH_epilog3               1001bff3 f   LIBCMT:ehprolg3.obj
 0001:0001b008       __EH_prolog3               1001c008 f   LIBCMT:ehprolg3.obj
 0001:0001b03c       __EH_prolog3_catch         1001c03c f   LIBCMT:ehprolg3.obj
 0001:0001b080       __aulldvrm                 1001c080 f   LIBCMT:ulldvrm.obj
 0001:0001b120       __aullrem                  1001c120 f   LIBCMT:ullrem.obj
 0001:0001b1a0       __allmul                   1001c1a0 f   LIBCMT:llmul.obj
 0001:0001b1e0       __alldiv                   1001c1e0 f   LIBCMT:lldiv.obj
 0001:0001b290       __allrem                   1001c290 f   LIBCMT:llrem.obj
 0001:0001b350       __allshl                   1001c350 f   LIBCMT:llshl.obj
 0001:0001b370       __aullshr                  1001c370 f   LIBCMT:ullshr.obj
 0001:0001b390       __ftol2_sse                1001c390 f   LIBCMT:ftol2.obj
 0001:0001b399       __ftol2_pentium4           1001c399 f   LIBCMT:ftol2.obj
 0001:0001b3ac       __ftol2_sse_excpt          1001c3ac f   LIBCMT:ftol2.obj
 0001:0001b3d0       __ftol2                    1001c3d0 f   LIBCMT:ftol2.obj
 0001:0001b450       __alloca_probe_16          1001c450 f   LIBCMT:alloca16.obj
 0001:0001b466       __alloca_probe_8           1001c466     LIBCMT:alloca16.obj
 0001:0001b480       _strrchr                   1001c480 f   libvcruntime:strrchr.obj
 0001:0001b5c0       _strchr                    1001c5c0 f   libvcruntime:strchr.obj
 0001:0001b62e       ___from_strstr_to_strchr   1001c62e     libvcruntime:strchr.obj
 0002:00000000       __imp__GetLastError@0      1001d000     kernel32:KERNEL32.dll
 0002:00000004       __imp__GetSystemTimeAsFileTime@4 1001d004     kernel32:KERNEL32.dll
 0002:00000008       __imp__CloseHandle@4       1001d008     kernel32:KERNEL32.dll
 0002:0000000c       __imp__EnterCriticalSection@4 1001d00c     kernel32:KERNEL32.dll
 0002:00000010       __imp__LeaveCriticalSection@4 1001d010     kernel32:KERNEL32.dll
 0002:00000014       __imp__MapViewOfFile@20    1001d014     kernel32:KERNEL32.dll
 0002:00000018       __imp__UnmapViewOfFile@4   1001d018     kernel32:KERNEL32.dll
 0002:0000001c       __imp__CreateFileMappingA@24 1001d01c     kernel32:KERNEL32.dll
 0002:00000020       __imp__InitializeCriticalSection@4 1001d020     kernel32:KERNEL32.dll
 0002:00000024       __imp__WriteConsoleW@20    1001d024     kernel32:KERNEL32.dll
 0002:00000028       __imp__SetEndOfFile@4      1001d028     kernel32:KERNEL32.dll
 0002:0000002c       __imp__ReadConsoleW@20     1001d02c     kernel32:KERNEL32.dll
 0002:00000030       __imp__ReadFile@20         1001d030     kernel32:KERNEL32.dll
 0002:00000034       __imp__HeapReAlloc@16      1001d034     kernel32:KERNEL32.dll
 0002:00000038       __imp__HeapSize@12         1001d038     kernel32:KERNEL32.dll
 0002:0000003c       __imp__CreateFileW@28      1001d03c     kernel32:KERNEL32.dll
 0002:00000040       __imp__GetStringTypeW@16   1001d040     kernel32:KERNEL32.dll
 0002:00000044       __imp__SetFilePointerEx@20 1001d044     kernel32:KERNEL32.dll
 0002:00000048       __imp__GetFileSizeEx@8     1001d048     kernel32:KERNEL32.dll
 0002:0000004c       __imp__SetStdHandle@8      1001d04c     kernel32:KERNEL32.dll
 0002:00000050       __imp__GetConsoleMode@8    1001d050     kernel32:KERNEL32.dll
 0002:00000054       __imp__GetConsoleOutputCP@0 1001d054     kernel32:KERNEL32.dll
 0002:00000058       __imp__WriteFile@20        1001d058     kernel32:KERNEL32.dll
 0002:0000005c       __imp__UnhandledExceptionFilter@4 1001d05c     kernel32:KERNEL32.dll
 0002:00000060       __imp__SetUnhandledExceptionFilter@4 1001d060     kernel32:KERNEL32.dll
 0002:00000064       __imp__GetCurrentProcess@0 1001d064     kernel32:KERNEL32.dll
 0002:00000068       __imp__TerminateProcess@8  1001d068     kernel32:KERNEL32.dll
 0002:0000006c       __imp__IsProcessorFeaturePresent@4 1001d06c     kernel32:KERNEL32.dll
 0002:00000070       __imp__QueryPerformanceCounter@4 1001d070     kernel32:KERNEL32.dll
 0002:00000074       __imp__GetCurrentProcessId@0 1001d074     kernel32:KERNEL32.dll
 0002:00000078       __imp__GetCurrentThreadId@0 1001d078     kernel32:KERNEL32.dll
 0002:0000007c       __imp__InitializeSListHead@4 1001d07c     kernel32:KERNEL32.dll
 0002:00000080       __imp__IsDebuggerPresent@0 1001d080     kernel32:KERNEL32.dll
 0002:00000084       __imp__GetStartupInfoW@4   1001d084     kernel32:KERNEL32.dll
 0002:00000088       __imp__GetModuleHandleW@4  1001d088     kernel32:KERNEL32.dll
 0002:0000008c       __imp__RaiseException@16   1001d08c     kernel32:KERNEL32.dll
 0002:00000090       __imp__InterlockedFlushSList@4 1001d090     kernel32:KERNEL32.dll
 0002:00000094       __imp__RtlUnwind@16        1001d094     kernel32:KERNEL32.dll
 0002:00000098       __imp__SetLastError@4      1001d098     kernel32:KERNEL32.dll
 0002:0000009c       __imp__DeleteCriticalSection@4 1001d09c     kernel32:KERNEL32.dll
 0002:000000a0       __imp__InitializeCriticalSectionAndSpinCount@8 1001d0a0     kernel32:KERNEL32.dll
 0002:000000a4       __imp__TlsAlloc@0          1001d0a4     kernel32:KERNEL32.dll
 0002:000000a8       __imp__TlsGetValue@4       1001d0a8     kernel32:KERNEL32.dll
 0002:000000ac       __imp__TlsSetValue@8       1001d0ac     kernel32:KERNEL32.dll
 0002:000000b0       __imp__TlsFree@4           1001d0b0     kernel32:KERNEL32.dll
 0002:000000b4       __imp__FreeLibrary@4       1001d0b4     kernel32:KERNEL32.dll
 0002:000000b8       __imp__GetProcAddress@8    1001d0b8     kernel32:KERNEL32.dll
 0002:000000bc       __imp__LoadLibraryExW@12   1001d0bc     kernel32:KERNEL32.dll
 0002:000000c0       __imp__EncodePointer@4     1001d0c0     kernel32:KERNEL32.dll
 0002:000000c4       __imp__ExitProcess@4       1001d0c4     kernel32:KERNEL32.dll
 0002:000000c8       __imp__GetModuleHandleExW@12 1001d0c8     kernel32:KERNEL32.dll
 0002:000000cc       __imp__GetModuleFileNameW@12 1001d0cc     kernel32:KERNEL32.dll
 0002:000000d0       __imp__HeapAlloc@12        1001d0d0     kernel32:KERNEL32.dll
 0002:000000d4       __imp__HeapFree@12         1001d0d4     kernel32:KERNEL32.dll
 0002:000000d8       __imp__CompareStringW@24   1001d0d8     kernel32:KERNEL32.dll
 0002:000000dc       __imp__LCMapStringW@24     1001d0dc     kernel32:KERNEL32.dll
 0002:000000e0       __imp__GetStdHandle@4      1001d0e0     kernel32:KERNEL32.dll
 0002:000000e4       __imp__GetFileType@4       1001d0e4     kernel32:KERNEL32.dll
 0002:000000e8       __imp__FindClose@4         1001d0e8     kernel32:KERNEL32.dll
 0002:000000ec       __imp__FindFirstFileExW@24 1001d0ec     kernel32:KERNEL32.dll
 0002:000000f0       __imp__FindNextFileW@8     1001d0f0     kernel32:KERNEL32.dll
 0002:000000f4       __imp__IsValidCodePage@4   1001d0f4     kernel32:KERNEL32.dll
 0002:000000f8       __imp__GetACP@0            1001d0f8     kernel32:KERNEL32.dll
 0002:000000fc       __imp__GetOEMCP@0          1001d0fc     kernel32:KERNEL32.dll
 0002:00000100       __imp__GetCPInfo@8         1001d100     kernel32:KERNEL32.dll
 0002:00000104       __imp__GetCommandLineA@0   1001d104     kernel32:KERNEL32.dll
 0002:00000108       __imp__GetCommandLineW@0   1001d108     kernel32:KERNEL32.dll
 0002:0000010c       __imp__MultiByteToWideChar@24 1001d10c     kernel32:KERNEL32.dll
 0002:00000110       __imp__WideCharToMultiByte@32 1001d110     kernel32:KERNEL32.dll
 0002:00000114       __imp__GetEnvironmentStringsW@0 1001d114     kernel32:KERNEL32.dll
 0002:00000118       __imp__FreeEnvironmentStringsW@4 1001d118     kernel32:KERNEL32.dll
 0002:0000011c       __imp__SetEnvironmentVariableW@8 1001d11c     kernel32:KERNEL32.dll
 0002:00000120       __imp__GetProcessHeap@0    1001d120     kernel32:KERNEL32.dll
 0002:00000124       __imp__FlushFileBuffers@4  1001d124     kernel32:KERNEL32.dll
 0002:00000128       __imp__DecodePointer@4     1001d128     kernel32:KERNEL32.dll
 0002:0000012c       \177KERNEL32_NULL_THUNK_DATA 1001d12c     kernel32:KERNEL32.dll
 0002:00000130       __imp__CreateDialogParamA@20 1001d130     user32:USER32.dll
 0002:00000134       __imp__ShowWindow@8        1001d134     user32:USER32.dll
 0002:00000138       __imp__DestroyWindow@4     1001d138     user32:USER32.dll
 0002:0000013c       __imp__SendMessageA@16     1001d13c     user32:USER32.dll
 0002:00000140       __imp__GetParent@4         1001d140     user32:USER32.dll
 0002:00000144       __imp__GetWindowLongA@8    1001d144     user32:USER32.dll
 0002:00000148       __imp__IsWindow@4          1001d148     user32:USER32.dll
 0002:0000014c       __imp__RegisterWindowMessageA@4 1001d14c     user32:USER32.dll
 0002:00000150       __imp__SendMessageTimeoutA@28 1001d150     user32:USER32.dll
 0002:00000154       __imp__PostMessageA@16     1001d154     user32:USER32.dll
 0002:00000158       \177USER32_NULL_THUNK_DATA 1001d158     user32:USER32.dll
 0002:0000015c       ___guard_check_icall_fptr  1001d15c     LIBCMT:guard_support.obj
 0002:00000160       ___xc_a                    1001d160     LIBCMT:initializers.obj
 0002:00000164       ___xc_z                    1001d164     LIBCMT:initializers.obj
 0002:00000168       ___xi_a                    1001d168     LIBCMT:initializers.obj
 0002:0000016c       ___acrt_stdio_initializer  1001d16c     libucrt:stdio_initializer.obj
 0002:00000170       ___acrt_multibyte_initializer 1001d170     libucrt:multibyte_initializer.obj
 0002:00000174       ___acrt_tran_sse2_initializer 1001d174     libucrt:sse2_initializer.obj
 0002:00000178       ___acrt_fmode_initializer  1001d178     libucrt:fmode_initializer.obj
 0002:0000017c       ___xi_z                    1001d17c     LIBCMT:initializers.obj
 0002:00000180       ___xp_a                    1001d180     LIBCMT:initializers.obj
 0002:00000184       ___acrt_locale_terminator  1001d184     libucrt:locale_initializer.obj
 0002:00000188       ___dcrt_console_output_terminator 1001d188     libucrt:console_output_initializer.obj
 0002:0000018c       ___acrt_stdio_terminator   1001d18c     libucrt:stdio_initializer.obj
 0002:00000190       ___xp_z                    1001d190     LIBCMT:initializers.obj
 0002:00000194       ___xt_a                    1001d194     LIBCMT:initializers.obj
 0002:00000198       ___xt_z                    1001d198     LIBCMT:initializers.obj
 0002:000001a0       ??_C@_0BJ@FKCDJFDK@JAVA_ACCESSBRIDGE_LOGDIR@ 1001d1a0     AccessBridgeDebug.obj
 0002:000001bc       ??_C@_04FPOLKAEB@?4log@    1001d1bc     AccessBridgeDebug.obj
 0002:000001c4       ??_C@_01NOFIACDB@w@        1001d1c4     AccessBridgeDebug.obj
 0002:000001c8       ??_C@_04EINJHBMM@?6?$CFs?6@ 1001d1c8     AccessBridgeDebug.obj
 0002:000001d0       ??_C@_0BH@PPBGFLKL@Could?5not?5open?5file?5?$CFs@ 1001d1d0     AccessBridgeDebug.obj
 0002:000001e8       ??_C@_07IBOBEFLP@?$FL?$CFllu?$FN?5@ 1001d1e8     AccessBridgeDebug.obj
 0002:000001f0       ??_C@_02PCIJFNDE@?$AN?6@   1001d1f0     AccessBridgeDebug.obj
 0002:000001f4       ??_C@_0BH@BLGOOJIK@AccessBridge?9?$CFp?9?$CFp?4mmf@ 1001d1f4     AccessBridgeJavaVMInstance.obj
 0002:0000020c       ??_C@_03DJNNCAJF@OK?$DP@   1001d20c     AccessBridgeJavaVMInstance.obj
 0002:00000210       ??_C@_03ONJMBPEK@OK?$CB@   1001d210     AccessBridgeJavaVMInstance.obj
 0002:00000214       ??_C@_0CP@JIGBIHFH@?$FLINFO?$FN?3?5In?5AccessBridgeVMInstan@ 1001d214     AccessBridgeJavaVMInstance.obj
 0002:00000244       ??_C@_0CH@KAGNBCII@?$FLINFO?$FN?3?5?5?5?5?5javaAccessBridgeWin@ 1001d244     AccessBridgeJavaVMInstance.obj
 0002:0000026c       ??_C@_0CC@NKGMANMJ@?$FLINFO?$FN?3?5In?5findAccessBridgeWind@ 1001d26c     AccessBridgeJavaVMInstance.obj
 0002:00000290       ??_C@_0CK@NBPNOPCH@?$FLINFO?$FN?3?5In?5findABJavaInstanceFr@ 1001d290     AccessBridgeJavaVMInstance.obj
 0002:000002c0       ??_7exception@std@@6B@     1001d2c0     AccessBridgeMessageQueue.obj
 0002:000002c8       ??_C@_0BC@EOODALEL@Unknown?5exception@ 1001d2c8     AccessBridgeMessageQueue.obj
 0002:000002e0       ??_7bad_alloc@std@@6B@     1001d2e0     AccessBridgeMessageQueue.obj
 0002:000002e8       ??_C@_0P@GHFPNOJB@bad?5allocation@ 1001d2e8     AccessBridgeMessageQueue.obj
 0002:000002f8       ??_C@_0CN@EPCNBBKD@?$FLINFO?$FN?3?5?5?5in?5AccessBridgeMessag@ 1001d2f8     AccessBridgeMessageQueue.obj
 0002:00000328       ??_C@_0BM@FHOEMINC@?$FLINFO?$FN?3?5?5?5?5?5queue?5size?5?$DN?5?$CFd@ 1001d328     AccessBridgeMessageQueue.obj
 0002:00000344       ??_C@_0DF@PKPPNDEN@?$FLWARN?$FN?3?5?5?5?5?5queue?5was?5locked?$DL?5r@ 1001d344     AccessBridgeMessageQueue.obj
 0002:0000037c       ??_C@_0CF@CAPEOLCL@?$FLINFO?$FN?3?5?5?5?5?5adding?5element?5to?5q@ 1001d37c     AccessBridgeMessageQueue.obj
 0002:000003a4       ??_C@_0DL@IILCMNMG@?$FLINFO?$FN?3?5?5?5?5?5returning?5from?5Acce@ 1001d3a4     AccessBridgeMessageQueue.obj
 0002:000003e0       ??_C@_0DA@NHLJEKKG@?$FLINFO?$FN?3?5?5?5in?5AccessBridgeMessag@ 1001d3e0     AccessBridgeMessageQueue.obj
 0002:00000410       ??_C@_0CJ@FBOCEMKO@?$FLINFO?$FN?3?5?5?5?5?5removing?5element?5fr@ 1001d410     AccessBridgeMessageQueue.obj
 0002:0000043c       ??_C@_0DO@NEJIEHGM@?$FLINFO?$FN?3?5?5?5?5?5returning?5from?5Acce@ 1001d43c     AccessBridgeMessageQueue.obj
 0002:0000047c       ??_C@_0BM@BIAOFPJG@AccessBridge?9FromJava?9Hello@ 1001d47c     AccessBridgeMessages.obj
 0002:00000498       ??_C@_0BP@OELHMMDF@AccessBridge?9FromWindows?9Hello@ 1001d498     AccessBridgeMessages.obj
 0002:000004b8       ??_C@_0EC@DLPGLEGA@?$AN?6AccessBridgeWindowsEntryPoint@ 1001d4b8     AccessBridgeWindowsEntryPoints.obj
 0002:000004fc       ??_C@_0BG@GGFIABLO@windows_access_bridge@ 1001d4fc     WinAccessBridge.obj
 0002:00000514       ??_C@_0BL@GLCNGDJJ@?$FLINFO?$FN?3?5DLL_PROCESS_ATTACH@ 1001d514     WinAccessBridge.obj
 0002:00000530       ??_C@_0EG@HHOMJPNP@?$FLINFO?$FN?3?5?$CK?$CK?$CK?5AccessBridgeDialogP@ 1001d530     WinAccessBridge.obj
 0002:00000578       ??_C@_0CP@LHINEKAP@?$FLINFO?$FN?3?5AccessBridgeDialogProc?5@ 1001d578     WinAccessBridge.obj
 0002:000005a8       ??_C@_0EH@MDELPMEJ@?$FLINFO?$FN?3?5AccessBridgeDialogProc?5@ 1001d5a8     WinAccessBridge.obj
 0002:000005f0       ??_C@_0DP@HBEMDAPF@?$FLINFO?$FN?3?5AccessBridgeDialogProc?5@ 1001d5f0     WinAccessBridge.obj
 0002:00000630       ??_C@_0EH@MPLEACPJ@?$FLINFO?$FN?3?5AccessBridgeDialogProc?5@ 1001d630     WinAccessBridge.obj
 0002:00000678       ??_C@_0EG@GGGHDKAD@?$FLINFO?$FN?3?5?$CK?$CK?$CK?$CK?$CK?5AccessBridgeDialo@ 1001d678     WinAccessBridge.obj
 0002:000006c0       ??_C@_0DE@BGNNIIOB@?$FLINFO?$FN?3?5?5?5javaVMs?5chain?5in?5use?0@ 1001d6c0     WinAccessBridge.obj
 0002:000006f4       ??_C@_0CC@NEJJLLGC@?$FLINFO?$FN?3?5?5?5calling?5javaVMDestroy@ 1001d6f4     WinAccessBridge.obj
 0002:00000718       ??_C@_0FG@BHPCMIAO@?$FLINFO?$FN?3?5AccessBridgeDialogProc?5@ 1001d718     WinAccessBridge.obj
 0002:00000770       ??_C@_0BN@FIPGEIKI@?$FLINFO?$FN?3?5WinAccessBridge?5ctor@ 1001d770     WinAccessBridge.obj
 0002:00000790       ??_C@_0DE@JFKNENGC@?$FLINFO?$FN?3?5?$CK?$CK?$CK?$CK?$CKin?5WinAccessBridge@ 1001d790     WinAccessBridge.obj
 0002:000007c4       ??_C@_0CG@EDMKMONP@?$FLINFO?$FN?3?5?5?5telling?5?$CFp?5we?8re?5goin@ 1001d7c4     WinAccessBridge.obj
 0002:000007ec       ??_C@_0DB@CFPLAPDG@?$FLINFO?$FN?3?5?5?5finished?5telling?5JVMs@ 1001d7ec     WinAccessBridge.obj
 0002:00000820       ??_C@_0EE@GBJFCFOA@?$FLINFO?$FN?3?5?5?5finished?5deleting?5eve@ 1001d820     WinAccessBridge.obj
 0002:00000864       ??_C@_0BP@EBFMIPOK@?$FLINFO?$FN?3?5GOODBYE?5CRUEL?5WORLD?4?4?4@ 1001d864     WinAccessBridge.obj
 0002:00000884       ??_C@_0BJ@LMONFDOG@ACCESSBRIDGESTATUSWINDOW@ 1001d884     WinAccessBridge.obj
 0002:000008a0       ??_C@_0DN@NNELAOKC@?$FLINFO?$FN?3?5in?5WinAccessBridge?3?3ren@ 1001d8a0     WinAccessBridge.obj
 0002:000008e0       ??_C@_0CJ@LMLGKPGD@?$FLINFO?$FN?3?5?5?5Setting?5Java?5event?5ma@ 1001d8e0     WinAccessBridge.obj
 0002:0000090c       ??_C@_0DC@IJKHOBEO@?$FLINFO?$FN?3?5?5?5Setting?5Accessibility@ 1001d90c     WinAccessBridge.obj
 0002:00000940       ??_C@_0DN@ECLBFGAO@?$FLERROR?$FN?3?5Failed?5to?5initiate?5IPC@ 1001d940     WinAccessBridge.obj
 0002:00000980       ??_C@_0DG@OEMNKFJP@?$FLINFO?$FN?3?5?5?5Success?$CB?$CB?5?5We?5rendezv@ 1001d980     WinAccessBridge.obj
 0002:000009b8       ??_C@_0DK@BLMJEFJH@?$FLERROR?$FN?3?5sending?5memory?5package@ 1001d9b8     WinAccessBridge.obj
 0002:000009f4       ??_C@_0DC@BABNPCOM@?$FLINFO?$FN?3?5?5in?5WinAccessBridge?3?3qu@ 1001d9f4     WinAccessBridge.obj
 0002:00000a28       ??_C@_0DE@NOAFOCML@?$FLINFO?$FN?3?5in?5WinAccessBridge?3?3rec@ 1001da28     WinAccessBridge.obj
 0002:00000a5c       ??_C@_0BM@KNOOFOHJ@?$FLINFO?$FN?3?5?5dequeueing?5message@ 1001da5c     WinAccessBridge.obj
 0002:00000a78       ??_C@_0CD@GBHFIMOB@?$FLERROR?$FN?3?5Queue?5seems?5to?5be?5brok@ 1001da78     WinAccessBridge.obj
 0002:00000a9c       ??_C@_0CA@LFELFFDM@?$FLINFO?$FN?3?5?5found?5one?$DL?5sending?5it?$CB@ 1001da9c     WinAccessBridge.obj
 0002:00000abc       ??_C@_0BP@ENBFDBDP@?$FLWARN?$FN?3?5?5?5ODD?4?4?4?5element?5?$DN?$DN?50?$CB@ 1001dabc     WinAccessBridge.obj
 0002:00000adc       ??_C@_0CP@OIAJKCPF@?$FLWARN?$FN?3?5?5Queue?5in?5use?0?5will?5try@ 1001dadc     WinAccessBridge.obj
 0002:00000b0c       ??_C@_0DH@KAJCMPPF@?$FLWARN?$FN?3?5?5unable?5to?5dequeue?5mess@ 1001db0c     WinAccessBridge.obj
 0002:00000b44       ??_C@_0CO@KCIANNAF@?$FLINFO?$FN?3?5PreProcessing?5package?5s@ 1001db44     WinAccessBridge.obj
 0002:00000b78       ??_C@_0EF@DFMGOCJF@?$FLERROR?$FN?3?5?5?5processing?5FAILED?$CB?$CB?5@ 1001db78     WinAccessBridge.obj
 0002:00000bc0       ??_C@_0CL@HBCKEPEE@?$FLINFO?$FN?3?5?5?5?5package?5preprocessin@ 1001dbc0     WinAccessBridge.obj
 0002:00000bec       ??_C@_0DM@CCADHAH@?$FLINFO?$FN?3?5WinAccessBridge?3?3Proces@ 1001dbec     WinAccessBridge.obj
 0002:00000c28       ??_C@_0CI@KAACKIJC@?$FLINFO?$FN?3?5?5?5?5type?5?$DN?$DN?5cJavaShutdow@ 1001dc28     WinAccessBridge.obj
 0002:00000c50       ??_C@_0CE@KGDIDFJM@?$FLINFO?$FN?3?5?5?5?5event?5callback?5compl@ 1001dc50     WinAccessBridge.obj
 0002:00000c74       ??_C@_0BI@MGOIGNJM@?$FLINFO?$FN?3?5?5?5?5event?5fired?$CB@ 1001dc74     WinAccessBridge.obj
 0002:00000c90       ??_C@_0EC@JELBKKLB@?$FLERROR?$FN?3?5?5?5?5processing?5FAILED?$CB?$CB@ 1001dc90     WinAccessBridge.obj
 0002:00000cd4       ??_C@_0CM@OIHFPHBP@?$FLINFO?$FN?3?5?5?5?5begin?5callback?5to?5AT@ 1001dcd4     WinAccessBridge.obj
 0002:00000d00       ??_C@_0EB@PCOLNIOI@?$FLERROR?$FN?3?5?5?5processing?5FAILED?$CB?$CB?5@ 1001dd00     WinAccessBridge.obj
 0002:00000d48       ??_C@_0EG@DADDGPDA@?$FLERROR?$FN?3?5?5?5?5processing?5FAILED?$CB?$CB@ 1001dd48     WinAccessBridge.obj
 0002:00000d90       ??_C@_0CI@PMGDCMNI@?$FLINFO?$FN?3?5?5?5?5package?5processing?5c@ 1001dd90     WinAccessBridge.obj
 0002:00000db8       ??_C@_0DD@EDMANGOO@?$FLINFO?$FN?3?5?$CK?$CK?$CK?$CK?$CK?5WinAccessBridge?3?3@ 1001ddb8     WinAccessBridge.obj
 0002:00000dec       ??_C@_0CP@IIHJFGGB@?$FLINFO?$FN?3?5?5?5data?5structures?5succe@ 1001ddec     WinAccessBridge.obj
 0002:00000e1c       ??_C@_0DB@JABMCGEJ@?$FLERROR?$FN?3?5couldn?8t?5find?5matching@ 1001de1c     WinAccessBridge.obj
 0002:00000e50       ??_C@_0DJ@EFGAHBMH@?$FLINFO?$FN?3?5WinAccessBridge?3?3releas@ 1001de50     WinAccessBridge.obj
 0002:00000e8c       ??_C@_0CO@GDCOMIDN@?$FLINFO?$FN?3?5WinAccessBridge?3?3getVer@ 1001de8c     WinAccessBridge.obj
 0002:00000ec0       ??_C@_0IH@JNMBAFNI@?$FLINFO?$FN?3?5?5?5VMversion?3?5?$CFls?6?5?5?5?5?5?5@ 1001dec0     WinAccessBridge.obj
 0002:00000f48       ??_C@_0CJ@MFBANPLF@?$FLINFO?$FN?3?5In?5WinAccessBridge?3?3isJ@ 1001df48     WinAccessBridge.obj
 0002:00000f74       ??_C@_0CK@OIADIKJK@?$FLINFO?$FN?3?5WinAccessBridge?3?3isJava@ 1001df74     WinAccessBridge.obj
 0002:00000fa0       ??_C@_0DJ@GDIICFAI@?$FLINFO?$FN?3?5WinAccessBridge?3?3isSame@ 1001dfa0     WinAccessBridge.obj
 0002:00000fe0       ??_C@_0EF@JHJAECO@?$FLINFO?$FN?3?5?5?5WinAccessBridge?3?3isSa@ 1001dfe0     WinAccessBridge.obj
 0002:00001028       ??_C@_0EL@EGCPHNBB@?$FLINFO?$FN?3?5?5?5WinAccessBridge?3?3isSa@ 1001e028     WinAccessBridge.obj
 0002:00001078       ??_C@_0FE@JNIGOBOL@?$FLERROR?$FN?3?5?5?5WinAccessBridge?3?3isS@ 1001e078     WinAccessBridge.obj
 0002:000010cc       ??_C@_0DM@KHCMPGEG@?$FLINFO?$FN?3?5WinAccessBridge?3?3getAcc@ 1001e0cc     WinAccessBridge.obj
 0002:00001108       ??_C@_0DA@KDJKNLAN@?$FLINFO?$FN?3?5?5?5?5?5current?9?$DOvmID?5?$DN?5?$CFX?0@ 1001e108     WinAccessBridge.obj
 0002:00001138       ??_C@_0CP@IJNFIHAG@?$FLINFO?$FN?3?5?5?5?5?5pkg?9?$DOrAccessibleCon@ 1001e138     WinAccessBridge.obj
 0002:00001168       ??_C@_0DJ@FFBPMFOM@?$FLERROR?$FN?3?5getAccessibleContextFr@ 1001e168     WinAccessBridge.obj
 0002:000011a4       ??_C@_0DO@IIGOCPCC@?$FLERROR?$FN?3?5getAccessibleContextFr@ 1001e1a4     WinAccessBridge.obj
 0002:000011e4       ??_C@_0DL@KEEIEGBJ@?$FLINFO?$FN?3?5?5?5in?5WinAccessBridge?3?3g@ 1001e1e4     WinAccessBridge.obj
 0002:00001220       ??_C@_0EA@HDGDGEMM@?$FLINFO?$FN?3?5WinAccessBridge?3?3getHWN@ 1001e220     WinAccessBridge.obj
 0002:00001260       ??_C@_0EA@FHJPOEHJ@?$FLINFO?$FN?3?5WinAccessBridge?3?3getAcc@ 1001e260     WinAccessBridge.obj
 0002:000012a0       ??_C@_0EB@HKEAOAKG@?$FLINFO?$FN?3?5WinAccessBridge?3?3getAcc@ 1001e2a0     WinAccessBridge.obj
 0002:000012e8       ??_C@_0EC@OFBFCAEJ@?$FLINFO?$FN?3?5WinAccessBridge?3?3getAcc@ 1001e2e8     WinAccessBridge.obj
 0002:00001330       ??_C@_0JA@MODCAACP@?$FLINFO?$FN?3?5?5?5name?3?5?$CFls?6?5?5?5?5?5?5?5?5?5?5d@ 1001e330     WinAccessBridge.obj
 0002:000013c0       ??_C@_0EJ@HLHMECO@?$FLINFO?$FN?3?5WinAccessBridge?3?3getAcc@ 1001e3c0     WinAccessBridge.obj
 0002:00001410       ??_C@_0EA@MDGJLODH@?$FLINFO?$FN?3?5WinAccessBridge?3?3getAcc@ 1001e410     WinAccessBridge.obj
 0002:00001450       ??_C@_0EI@IEEMIFOJ@?$FLINFO?$FN?3?5?$CD?$CD?$CD?$CD?$CD?5WinAccessBridge?3?3@ 1001e450     WinAccessBridge.obj
 0002:00001498       ??_C@_0EC@FNKONEFN@?$FLINFO?$FN?3?5?5?5?$CD?$CD?$CD?$CD?$CD?5WinAccessBridge@ 1001e498     WinAccessBridge.obj
 0002:000014e0       ??_C@_0EA@GPGOILHN@?$FLERROR?$FN?3?5?5?5?$CD?$CD?$CD?$CD?$CD?5WinAccessBridg@ 1001e4e0     WinAccessBridge.obj
 0002:00001520       ??_C@_0EO@GIFIOBJO@?$FLINFO?$FN?3?5?$CD?$CD?$CD?$CD?$CD?5WinAccessBridge?3?3@ 1001e520     WinAccessBridge.obj
 0002:00001570       ??_C@_0DK@FPHEFKPF@?$FLINFO?$FN?3?5?5?5XXXX?5pkg?9?$DOrTableCellI@ 1001e570     WinAccessBridge.obj
 0002:000015b0       ??_C@_0EG@CFNEHAJF@?$FLINFO?$FN?3?5?5?5?$CD?$CD?$CD?$CD?$CD?5WinAccessBridge@ 1001e5b0     WinAccessBridge.obj
 0002:000015f8       ??_C@_0EE@DMEKGPAL@?$FLERROR?$FN?3?5?5?5?$CD?$CD?$CD?$CD?$CD?5WinAccessBridg@ 1001e5f8     WinAccessBridge.obj
 0002:00001640       ??_C@_0EJ@GHNOCBA@?$FLINFO?$FN?3?5?$CD?$CD?$CD?$CD?$CD?5WinAccessBridge?3?3@ 1001e640     WinAccessBridge.obj
 0002:00001690       ??_C@_0EH@MMAIEADN@?$FLINFO?$FN?3?5?5?5?$CD?$CD?$CD?$CD?$CD?5WinAccessBridge@ 1001e690     WinAccessBridge.obj
 0002:000016d8       ??_C@_0EF@IGPDOLOH@?$FLERROR?$FN?3?5?5?5?$CD?$CD?$CD?$CD?$CD?5WinAccessBridg@ 1001e6d8     WinAccessBridge.obj
 0002:00001720       ??_C@_0EM@KLDOANDG@?$FLINFO?$FN?3?5?$CD?$CD?$CD?$CD?$CD?5WinAccessBridge?3?3@ 1001e720     WinAccessBridge.obj
 0002:00001770       ??_C@_0EK@DJMDCCLK@?$FLINFO?$FN?3?5?5?5?$CD?$CD?$CD?$CD?$CD?5WinAccessBridge@ 1001e770     WinAccessBridge.obj
 0002:000017c0       ??_C@_0EI@CELDDCKP@?$FLERROR?$FN?3?5?5?5?$CD?$CD?$CD?$CD?$CD?5WinAccessBridg@ 1001e7c0     WinAccessBridge.obj
 0002:00001808       ??_C@_0FC@BPONCABC@?$FLINFO?$FN?3?5?$CD?$CD?$CD?$CD?$CD?5WinAccessBridge?3?3@ 1001e808     WinAccessBridge.obj
 0002:00001860       ??_C@_0EM@JPIPIDPC@?$FLINFO?$FN?3?5?5?5?$CD?$CD?$CD?$CD?$CD?5WinAccessBridge@ 1001e860     WinAccessBridge.obj
 0002:000018b0       ??_C@_0EK@IGPCFPOI@?$FLERROR?$FN?3?5?5?5?$CD?$CD?$CD?$CD?$CD?5WinAccessBridg@ 1001e8b0     WinAccessBridge.obj
 0002:00001900       ??_C@_0FF@GEJHIBCC@?$FLINFO?$FN?3?5?$CD?$CD?$CD?$CD?$CD?5WinAccessBridge?3?3@ 1001e900     WinAccessBridge.obj
 0002:00001958       ??_C@_0EP@PJFHLMKB@?$FLINFO?$FN?3?5?5?5?$CD?$CD?$CD?$CD?$CD?5WinAccessBridge@ 1001e958     WinAccessBridge.obj
 0002:000019a8       ??_C@_0EN@FJIGOJNI@?$FLERROR?$FN?3?5?5?5?$CD?$CD?$CD?$CD?$CD?5WinAccessBridg@ 1001e9a8     WinAccessBridge.obj
 0002:000019f8       ??_C@_0FB@IPIFJJKK@?$FLINFO?$FN?3?5?$CD?$CD?$CD?$CD?$CD?5WinAccessBridge?3?3@ 1001e9f8     WinAccessBridge.obj
 0002:00001a50       ??_C@_0EP@DHAGNOBO@?$FLINFO?$FN?3?5?5?5?$CD?$CD?$CD?$CD?$CD?5WinAccessBridge@ 1001ea50     WinAccessBridge.obj
 0002:00001aa0       ??_C@_0EN@IFAFODLF@?$FLERROR?$FN?3?5?5?5?$CD?$CD?$CD?$CD?$CD?5WinAccessBridg@ 1001eaa0     WinAccessBridge.obj
 0002:00001af0       ??_C@_0EK@FCAMCNJB@?$FLINFO?$FN?3?5?$CD?$CD?$CD?$CD?$CD?5WinAccessBridge?3?3@ 1001eaf0     WinAccessBridge.obj
 0002:00001b40       ??_C@_0EI@LCHMKLCB@?$FLINFO?$FN?3?5?5?5?$CD?$CD?$CD?$CD?$CD?5WinAccessBridge@ 1001eb40     WinAccessBridge.obj
 0002:00001b88       ??_C@_0EG@PCFFNJPM@?$FLERROR?$FN?3?5?5?5?$CD?$CD?$CD?$CD?$CD?5WinAccessBridg@ 1001eb88     WinAccessBridge.obj
 0002:00001bd0       ??_C@_0EN@MHFLCDEG@?$FLINFO?$FN?3?5?$CD?$CD?$CD?$CD?$CD?5WinAccessBridge?3?3@ 1001ebd0     WinAccessBridge.obj
 0002:00001c20       ??_C@_0EL@HPJEOBAF@?$FLINFO?$FN?3?5?5?5?$CD?$CD?$CD?$CD?$CD?5WinAccessBridge@ 1001ec20     WinAccessBridge.obj
 0002:00001c70       ??_C@_0EJ@EFJNHGOC@?$FLERROR?$FN?3?5?5?5?$CD?$CD?$CD?$CD?$CD?5WinAccessBridg@ 1001ec70     WinAccessBridge.obj
 0002:00001cc0       ??_C@_0FE@EEAPAHGA@?$FLINFO?$FN?3?5?$CD?$CD?$CD?$CD?$CD?5WinAccessBridge?3?3@ 1001ecc0     WinAccessBridge.obj
 0002:00001d18       ??_C@_0FC@IJCKDOEL@?$FLINFO?$FN?3?5?5?5?$CD?$CD?$CD?$CD?$CD?5WinAccessBridge@ 1001ed18     WinAccessBridge.obj
 0002:00001d70       ??_C@_0FA@EEJJLKOB@?$FLERROR?$FN?3?5?5?5?$CD?$CD?$CD?$CD?$CD?5WinAccessBridg@ 1001ed70     WinAccessBridge.obj
 0002:00001dc0       ??_C@_0EN@IKMAMDCJ@?$FLINFO?$FN?3?5?$CD?$CD?$CD?$CD?$CD?5WinAccessBridge?3?3@ 1001edc0     WinAccessBridge.obj
 0002:00001e10       ??_C@_0EL@MCFEFCEP@?$FLINFO?$FN?3?5?5?5?$CD?$CD?$CD?$CD?$CD?5WinAccessBridge@ 1001ee10     WinAccessBridge.obj
 0002:00001e60       ??_C@_0EJ@OEGCIAEN@?$FLERROR?$FN?3?5?5?5?$CD?$CD?$CD?$CD?$CD?5WinAccessBridg@ 1001ee60     WinAccessBridge.obj
 0002:00001eb0       ??_C@_0FB@FBDIFIGA@?$FLERROR?$FN?3?5?$CD?$CD?$CD?$CD?$CD?5WinAccessBridge?3@ 1001eeb0     WinAccessBridge.obj
 0002:00001f08       ??_C@_0EO@KBJAHINP@?$FLINFO?$FN?3?5?5?5?$CD?$CD?$CD?$CD?$CD?5WinAccessBridge@ 1001ef08     WinAccessBridge.obj
 0002:00001f58       ??_C@_0EM@FBMEIFEO@?$FLERROR?$FN?3?5?5?5?$CD?$CD?$CD?$CD?$CD?5WinAccessBridg@ 1001ef58     WinAccessBridge.obj
 0002:00001fa8       ??_C@_0EN@EJPIGDNI@?$FLINFO?$FN?3?5?$CD?$CD?$CD?$CD?$CD?5WinAccessBridge?3?3@ 1001efa8     WinAccessBridge.obj
 0002:00001ff8       ??_C@_0EB@EHNAMLGG@?$FLINFO?$FN?3?5?5?5?$CD?$CD?$CD?$CD?$CD?5WinAccessBridge@ 1001eff8     WinAccessBridge.obj
 0002:0000203c       ??_C@_0DP@JGIKFGJD@?$FLERROR?$FN?3?5?5?5?$CD?$CD?$CD?$CD?$CD?5WinAccessBridg@ 1001f03c     WinAccessBridge.obj
 0002:00002080       ??_C@_0FA@BNCMMHDE@?$FLINFO?$FN?3?5?$CD?$CD?$CD?$CD?$CD?5WinAccessBridge?3?3@ 1001f080     WinAccessBridge.obj
 0002:000020d0       ??_C@_0EE@HJIACDJB@?$FLINFO?$FN?3?5?5?5?$CD?$CD?$CD?$CD?$CD?5WinAccessBridge@ 1001f0d0     WinAccessBridge.obj
 0002:00002118       ??_C@_0EC@HJIAKIIH@?$FLERROR?$FN?3?5?5?5?$CD?$CD?$CD?$CD?$CD?5WinAccessBridg@ 1001f118     WinAccessBridge.obj
 0002:00002160       ??_C@_0FF@NCBHFIIB@?$FLINFO?$FN?3?5?$CD?$CD?$CD?$CD?$CD?5WinAccessBridge?3?3@ 1001f160     WinAccessBridge.obj
 0002:000021b8       ??_C@_0ED@CBAGECAG@?$FLINFO?$FN?3?5?5?5?$CD?$CD?$CD?$CD?$CD?5WinAccessBridge@ 1001f1b8     WinAccessBridge.obj
 0002:00002200       ??_C@_0EB@NLKCNKIL@?$FLERROR?$FN?3?5?5?5?$CD?$CD?$CD?$CD?$CD?5WinAccessBridg@ 1001f200     WinAccessBridge.obj
 0002:00002248       ??_C@_0EK@KPCBMLHL@?$FLINFO?$FN?3?5?$CD?$CD?$CD?$CD?$CD?5WinAccessBridge?3?3@ 1001f248     WinAccessBridge.obj
 0002:00002298       ??_C@_0ED@KBOKJBJ@?$FLINFO?$FN?3?5?5?5?$CD?$CD?$CD?$CD?$CD?5pkg?9?$DOrAccessibl@ 1001f298     WinAccessBridge.obj
 0002:000022e0       ??_C@_0EE@MLCJPFKH@?$FLINFO?$FN?3?5?5?5?$CD?$CD?$CD?$CD?$CD?5WinAccessBridge@ 1001f2e0     WinAccessBridge.obj
 0002:00002328       ??_C@_0EC@ONHLHLKJ@?$FLERROR?$FN?3?5?5?5?$CD?$CD?$CD?$CD?$CD?5WinAccessBridg@ 1001f328     WinAccessBridge.obj
 0002:00002370       ??_C@_0EI@BEINFODC@?$FLINFO?$FN?3?5?$CD?$CD?$CD?$CD?$CD?5WinAccessBridge?3?3@ 1001f370     WinAccessBridge.obj
 0002:000023b8       ??_C@_0CN@CIJKLIHC@?$FLINFO?$FN?3?5?5?5?$CD?$CD?$CD?$CD?$CD?5hypertextInfo?4l@ 1001f3b8     WinAccessBridge.obj
 0002:000023e8       ??_C@_0EC@GJFIBKBJ@?$FLINFO?$FN?3?5?5?5?$CD?$CD?$CD?$CD?$CD?5WinAccessBridge@ 1001f3e8     WinAccessBridge.obj
 0002:00002430       ??_C@_0EA@ENIAHHMF@?$FLERROR?$FN?3?5?5?5?$CD?$CD?$CD?$CD?$CD?5WinAccessBridg@ 1001f430     WinAccessBridge.obj
 0002:00002470       ??_C@_0EI@MFFNFMHA@?$FLINFO?$FN?3?5WinAccessBridge?3?3activa@ 1001f470     WinAccessBridge.obj
 0002:000024b8       ??_C@_0GC@OOPIFCLD@?$FLERROR?$FN?3?5?5WinAccessBridge?3?3acti@ 1001f4b8     WinAccessBridge.obj
 0002:00002520       ??_C@_0EJ@KNECEC@?$FLINFO?$FN?3?5?$CD?$CD?$CD?$CD?$CD?5WinAccessBridge?3?3@ 1001f520     WinAccessBridge.obj
 0002:0000256c       ??_C@_0CJ@CHHBPBDA@?$FLINFO?$FN?3?5?5?5?$CD?$CD?$CD?$CD?$CD?5hypetext?5link?5c@ 1001f56c     WinAccessBridge.obj
 0002:00002598       ??_C@_0EG@OFFPNIFM@?$FLINFO?$FN?3?5?5?$CD?$CD?$CD?$CD?$CD?5WinAccessBridge?3@ 1001f598     WinAccessBridge.obj
 0002:000025e0       ??_C@_0EF@CJEMCIKC@?$FLERROR?$FN?3?5?5?5?$CD?$CD?$CD?$CD?$CD?5WinAccessBridg@ 1001f5e0     WinAccessBridge.obj
 0002:00002628       ??_C@_0EK@KALHBKDC@?$FLINFO?$FN?3?5?$CD?$CD?$CD?$CD?$CD?5WinAccessBridge?3?3@ 1001f628     WinAccessBridge.obj
 0002:00002674       ??_C@_0CD@FAKLHPNN@?$FLINFO?$FN?3?5?5?5?$CD?$CD?$CD?$CD?$CD?5pkg?9?$DOrSuccess?5?$DN@ 1001f674     WinAccessBridge.obj
 0002:00002698       ??_C@_0ED@CLMPFLBE@?$FLERROR?$FN?3?5?5?5?$CD?$CD?$CD?$CD?$CD?5WinAccessBridg@ 1001f698     WinAccessBridge.obj
 0002:000026e0       ??_C@_0EC@DJBOOIDG@?$FLERROR?$FN?3?5?5?$CD?$CD?$CD?$CD?$CD?5WinAccessBridge@ 1001f6e0     WinAccessBridge.obj
 0002:00002728       ??_C@_0EN@IMDNGAME@?$FLINFO?$FN?3?5?$CD?$CD?$CD?$CD?$CD?5WinAccessBridge?3?3@ 1001f728     WinAccessBridge.obj
 0002:00002778       ??_C@_0CJ@LGNOCJK@?$FLINFO?$FN?3?5?5?5?$CD?$CD?$CD?$CD?$CD?5hypetext?5link?5i@ 1001f778     WinAccessBridge.obj
 0002:000027a8       ??_C@_0EM@KCINDCOI@?$FLINFO?$FN?3?5?5?5?$CD?$CD?$CD?$CD?$CD?5WinAccessBridge@ 1001f7a8     WinAccessBridge.obj
 0002:000027f8       ??_C@_0EI@IEJDJKBK@?$FLERROR?$FN?5?5?$CD?$CD?$CD?$CD?$CD?5WinAccessBridge?3@ 1001f7f8     WinAccessBridge.obj
 0002:00002840       ??_C@_0EI@OHHKPFCO@?$FLINFO?$FN?3?5?$CD?$CD?$CD?$CD?$CD?5WinAccessBridge?3?3@ 1001f840     WinAccessBridge.obj
 0002:00002888       ??_C@_0EK@CIOPKHEJ@?$FLINFO?$FN?3?5?$CD?$CD?$CD?$CD?$CD?5WinAccessBridge?3?3@ 1001f888     WinAccessBridge.obj
 0002:000028d4       ??_C@_0DC@GOKFJHHA@?$FLINFO?$FN?3?5?5?5?$CD?$CD?$CD?$CD?$CD?5keyBindings?4key@ 1001f8d4     WinAccessBridge.obj
 0002:00002908       ??_C@_0KM@PICKCJIM@?$FLINFO?$FN?3?5?5?5Key?5Binding?5?$CD?5?$CFd?5?5?5?5?5@ 1001f908     WinAccessBridge.obj
 0002:000029b8       ??_C@_0EE@LGIDNFJF@?$FLINFO?$FN?3?5?5?5?$CD?$CD?$CD?$CD?$CD?5WinAccessBridge@ 1001f9b8     WinAccessBridge.obj
 0002:00002a00       ??_C@_0EB@PIGLELIJ@?$FLINFO?$FN?3?5?5?5?$CD?$CD?$CD?$CD?$CD?5WinAccessBridge@ 1001fa00     WinAccessBridge.obj
 0002:00002a48       ??_C@_0EE@KBJHDGDB@?$FLINFO?$FN?3?5?$CD?$CD?$CD?$CD?$CD?5WinAccessBridge?3?3@ 1001fa48     WinAccessBridge.obj
 0002:00002a8c       ??_C@_0CG@JNBKIMJN@?$FLINFO?$FN?3?5?5?5?$CD?$CD?$CD?$CD?$CD?5icons?4iconsCoun@ 1001fa8c     WinAccessBridge.obj
 0002:00002ab4       ??_C@_0DO@JGGAAEEG@?$FLINFO?$FN?3?5?5?5?$CD?$CD?$CD?$CD?$CD?5WinAccessBridge@ 1001fab4     WinAccessBridge.obj
 0002:00002af4       ??_C@_0DM@PHFGBDGG@?$FLERROR?$FN?3?5?5?5?$CD?$CD?$CD?$CD?$CD?5WinAccessBridg@ 1001faf4     WinAccessBridge.obj
 0002:00002b30       ??_C@_0EG@EKEEJFO@?$FLINFO?$FN?3?5?$CD?$CD?$CD?$CD?$CD?5WinAccessBridge?3?3@ 1001fb30     WinAccessBridge.obj
 0002:00002b78       ??_C@_0CK@COBILBN@?$FLINFO?$FN?3?5?5?5?$CD?$CD?$CD?$CD?$CD?5actions?4actions@ 1001fb78     WinAccessBridge.obj
 0002:00002ba8       ??_C@_0EA@EKDNLNJA@?$FLINFO?$FN?3?5?5?5?$CD?$CD?$CD?$CD?$CD?5WinAccessBridge@ 1001fba8     WinAccessBridge.obj
 0002:00002be8       ??_C@_0DO@HNCGODDL@?$FLERROR?$FN?3?5?5?5?$CD?$CD?$CD?$CD?$CD?5WinAccessBridg@ 1001fbe8     WinAccessBridge.obj
 0002:00002c28       ??_C@_0EH@IJHNMJPE@?$FLINFO?$FN?3?5WinAccessBridge?3?3doAcce@ 1001fc28     WinAccessBridge.obj
 0002:00002c70       ??_C@_0FL@LJNDNJAB@?$FLERROR?$FN?3?5?5?5WinAccessBridge?3?3doA@ 1001fc70     WinAccessBridge.obj
 0002:00002ccc       ??_C@_0DF@LBCGPHPD@?$FLINFO?$FN?3?5WinAccessBridge?3?3setTex@ 1001fccc     WinAccessBridge.obj
 0002:00002d04       ??_C@_0DJ@BDMKEGCI@?$FLINFO?$FN?3?5WinAccessBridge?3?3getPar@ 1001fd04     WinAccessBridge.obj
 0002:00002d40       ??_C@_0FE@FILBCBC@?$FLINFO?$FN?3?5?5?5pkg?9?$DOvmID?3?5?$CFX?5?5?5?5?5?5?5?5@ 1001fd40     WinAccessBridge.obj
 0002:00002d94       ??_C@_0CG@EPJKPFNH@?$FLINFO?$FN?3?5?5?5pkg?9?$DOrAccessibleConte@ 1001fd94     WinAccessBridge.obj
 0002:00002dbc       ??_C@_0DJ@LMOBJNAA@?$FLINFO?$FN?3?5WinAccessBridge?3?3getTop@ 1001fdbc     WinAccessBridge.obj
 0002:00002df8       ??_C@_0EB@EGNBJNPN@?$FLINFO?$FN?3?5WinAccessBridge?3?3getPar@ 1001fdf8     WinAccessBridge.obj
 0002:00002e3c       ??_C@_0DG@HMAMEAHE@?$FLINFO?$FN?3?5WinAccessBridge?3?3getObj@ 1001fe3c     WinAccessBridge.obj
 0002:00002e74       ??_C@_0DL@DIELJEEF@?$FLINFO?$FN?3?5WinAccessBridge?3?3getAct@ 1001fe74     WinAccessBridge.obj
 0002:00002eb0       ??_C@_0EA@KKNJCPIF@?$FLINFO?$FN?3?5WinAccessBridge?3?3getVir@ 1001feb0     WinAccessBridge.obj
 0002:00002ef0       ??_C@_0EK@LJJEDFEG@?$FLINFO?$FN?3?5?5?5?5?5WinAccessBridge?3?3ge@ 1001fef0     WinAccessBridge.obj
 0002:00002f3c       ??_C@_0DE@NGCOAPLI@?$FLINFO?$FN?3?5WinAccessBridge?3?3reques@ 1001ff3c     WinAccessBridge.obj
 0002:00002f70       ??_C@_0EB@LDKGCIL@?$FLINFO?$FN?3?5?5?5?5?5WinAccessBridge?3?3se@ 1001ff70     WinAccessBridge.obj
 0002:00002fb8       ??_C@_0EK@FKPJFOFL@?$FLINFO?$FN?3?5?5?5?5?5WinAccessBridge?3?3ge@ 1001ffb8     WinAccessBridge.obj
 0002:00003004       ??_C@_0DP@PHLAPJAH@?$FLINFO?$FN?3?5WinAccessBridge?3?3getVis@ 10020004     WinAccessBridge.obj
 0002:00003044       ??_C@_0DK@FFJLHNNJ@?$FLINFO?$FN?3?5WinAccessBridge?3?3getVis@ 10020044     WinAccessBridge.obj
 0002:00003080       ??_C@_0DM@MCJMMMCP@?$FLINFO?$FN?3?5WinAccessBridge?3?3setCar@ 10020080     WinAccessBridge.obj
 0002:000030c0       ??_C@_0EJ@FBPIKPOJ@?$FLINFO?$FN?3?5WinAccessBridge?3?3getAcc@ 100200c0     WinAccessBridge.obj
 0002:00003110       ??_C@_0EK@DNDDFNHD@?$FLINFO?$FN?3?5?5?5charCount?3?5?$CFd?5?5?5?5?5?5?5?5@ 10020110     WinAccessBridge.obj
 0002:00003160       ??_C@_0EG@BGFOEIHE@?$FLINFO?$FN?3?5WinAccessBridge?3?3getAcc@ 10020160     WinAccessBridge.obj
 0002:000031a8       ??_C@_0EK@KLCBPNFL@?$FLINFO?$FN?3?5WinAccessBridge?3?3getAcc@ 100201a8     WinAccessBridge.obj
 0002:000031f8       ??_C@_0EL@MJHEEFIF@?$FLINFO?$FN?3?5WinAccessBridge?3?3getAcc@ 100201f8     WinAccessBridge.obj
 0002:00003248       ??_C@_0EF@MMEINAI@?$FLINFO?$FN?3?5WinAccessBridge?3?3getAcc@ 10020248     WinAccessBridge.obj
 0002:00003290       ??_C@_0EA@GJMJEHDC@?$FLINFO?$FN?3?5WinAccessBridge?3?3getCar@ 10020290     WinAccessBridge.obj
 0002:000032d0       ??_C@_0EJ@BCHIKCEF@?$FLINFO?$FN?3?5WinAccessBridge?3?3getAcc@ 100202d0     WinAccessBridge.obj
 0002:00003320       ??_C@_0EI@LCFAOBKP@?$FLINFO?$FN?3?5WinAccessBridge?3?3getAcc@ 10020320     WinAccessBridge.obj
 0002:00003368       ??_C@_0DM@NFGOCJPM@?$FLINFO?$FN?3?5WinAccessBridge?3?3addJav@ 10020368     WinAccessBridge.obj
 0002:000033a4       ??_C@_0DP@PIGNLFHB@?$FLINFO?$FN?3?5?5?5?9?$DOpkgType?5?$DN?5?$CFX?0?5event@ 100203a4     WinAccessBridge.obj
 0002:000033e8       ??_C@_0EC@OKCIJGM@?$FLINFO?$FN?3?5in?5WinAccessBridge?3?3rem@ 100203e8     WinAccessBridge.obj
 0002:00003430       ??_C@_0EI@HMKIAPB@?$FLINFO?$FN?3?5in?5WinAccessBridge?3?3add@ 10020430     WinAccessBridge.obj
 0002:00003478       ??_C@_0DP@KFDABLNL@?$FLINFO?$FN?3?5?5?5?9?$DOpkgType?5?$DN?5?$CFX?0?5event@ 10020478     WinAccessBridge.obj
 0002:000034b8       ??_C@_0EL@BFCCGHFN@?$FLINFO?$FN?3?5in?5WinAccessBridge?3?3rem@ 100204b8     WinAccessBridge.obj
 0002:00003508       ??_7type_info@@6B@         10020508     LIBCMT:std_type_info_static.obj
 0002:0000350c       __pDefaultRawDllMain       1002050c     LIBCMT:dll_dllmain.obj
 0002:0000350c       __pRawDllMain              1002050c     LIBCMT:dll_dllmain.obj
 0002:0000351c       ??_7bad_array_new_length@std@@6B@ 1002051c     LIBCMT:throw_bad_alloc.obj
 0002:00003524       ??_C@_0BF@KINCDENJ@bad?5array?5new?5length@ 10020524     LIBCMT:throw_bad_alloc.obj
 0002:000036fc       ??_C@_08EHJDFFNH@__based?$CI@ 100206fc     libvcruntime:undname.obj
 0002:00003708       ??_C@_07KOLFKCDI@__cdecl@  10020708     libvcruntime:undname.obj
 0002:00003710       ??_C@_08GHMPAG@__pascal@   10020710     libvcruntime:undname.obj
 0002:0000371c       ??_C@_09IFJBGAPI@__stdcall@ 1002071c     libvcruntime:undname.obj
 0002:00003728       ??_C@_0L@NPHFGOKO@__thiscall@ 10020728     libvcruntime:undname.obj
 0002:00003734       ??_C@_0L@JMKHOMEK@__fastcall@ 10020734     libvcruntime:undname.obj
 0002:00003740       ??_C@_0N@BCKKPABJ@__vectorcall@ 10020740     libvcruntime:undname.obj
 0002:00003750       ??_C@_09HIJEGCPM@__clrcall@ 10020750     libvcruntime:undname.obj
 0002:0000375c       ??_C@_06GHPCKEAG@__eabi@   1002075c     libvcruntime:undname.obj
 0002:00003764       ??_C@_09IOPIDJLG@__swift_1@ 10020764     libvcruntime:undname.obj
 0002:00003770       ??_C@_09KFNFGKHF@__swift_2@ 10020770     libvcruntime:undname.obj
 0002:0000377c       ??_C@_07JOMMBBKO@__ptr64@  1002077c     libvcruntime:undname.obj
 0002:00003784       ??_C@_0L@PILCLIHE@__restrict@ 10020784     libvcruntime:undname.obj
 0002:00003790       ??_C@_0M@GFIIJFMG@__unaligned@ 10020790     libvcruntime:undname.obj
 0002:0000379c       ??_C@_09DHDLOLLB@restrict?$CI@ 1002079c     libvcruntime:undname.obj
 0002:000037a6       ??_C@_00CNPNBAHC@@         100207a6     libvcruntime:undname.obj
 0002:000037a8       ??_C@_04NIHEBCM@?5new@     100207a8     libvcruntime:undname.obj
 0002:000037b0       ??_C@_07FPCDHGMM@?5delete@ 100207b0     libvcruntime:undname.obj
 0002:000037b8       ??_C@_01NEMOKFLO@?$DN@     100207b8     libvcruntime:undname.obj
 0002:000037bc       ??_C@_02GPIOPFAK@?$DO?$DO@ 100207bc     libvcruntime:undname.obj
 0002:000037c0       ??_C@_02FODMEDOG@?$DM?$DM@ 100207c0     libvcruntime:undname.obj
 0002:000037c4       ??_C@_01DCLJPIOD@?$CB@     100207c4     libvcruntime:undname.obj
 0002:000037c8       ??_C@_02EGOFBIJA@?$DN?$DN@ 100207c8     libvcruntime:undname.obj
 0002:000037cc       ??_C@_02FDNJECIE@?$CB?$DN@ 100207cc     libvcruntime:undname.obj
 0002:000037d0       ??_C@_02GPECMEKF@?$FL?$FN@ 100207d0     libvcruntime:undname.obj
 0002:000037d4       ??_C@_08LHJFAFGD@operator@ 100207d4     libvcruntime:undname.obj
 0002:000037e0       ??_C@_02HBOOOICD@?9?$DO@   100207e0     libvcruntime:undname.obj
 0002:000037e4       ??_C@_01NBENCBCI@?$CK@     100207e4     libvcruntime:undname.obj
 0002:000037e8       ??_C@_02ECNGHCIF@?$CL?$CL@ 100207e8     libvcruntime:undname.obj
 0002:000037ec       ??_C@_02BAABKJLB@?9?9@     100207ec     libvcruntime:undname.obj
 0002:000037f0       ??_C@_01JOAMLHOP@?9@       100207f0     libvcruntime:undname.obj
 0002:000037f4       ??_C@_01MIFGBAGJ@?$CL@     100207f4     libvcruntime:undname.obj
 0002:000037f8       ??_C@_01HNPIGOCE@?$CG@     100207f8     libvcruntime:undname.obj
 0002:000037fc       ??_C@_03MNHNFDLC@?9?$DO?$CK@ 100207fc     libvcruntime:undname.obj
 0002:00003800       ??_C@_01KMDKNFGN@?1@       10020800     libvcruntime:undname.obj
 0002:00003804       ??_C@_01FGNFDNOH@?$CF@     10020804     libvcruntime:undname.obj
 0002:00003808       ??_C@_01MNNFJEPP@?$DM@     10020808     libvcruntime:undname.obj
 0002:0000380c       ??_C@_02EHCHHCKH@?$DM?$DN@ 1002080c     libvcruntime:undname.obj
 0002:00003810       ??_C@_01PPODPGHN@?$DO@     10020810     libvcruntime:undname.obj
 0002:00003814       ??_C@_02EEKDKGMJ@?$DO?$DN@ 10020814     libvcruntime:undname.obj
 0002:00003818       ??_C@_01IHBHIGKO@?0@       10020818     libvcruntime:undname.obj
 0002:0000381c       ??_C@_02HCKGKOFO@?$CI?$CJ@ 1002081c     libvcruntime:undname.obj
 0002:00003820       ??_C@_01PJKLJHI@?$HO@      10020820     libvcruntime:undname.obj
 0002:00003824       ??_C@_01JKBOJNNK@?$FO@     10020824     libvcruntime:undname.obj
 0002:00003828       ??_C@_01DNKMNLPK@?$HM@     10020828     libvcruntime:undname.obj
 0002:0000382c       ??_C@_02PPKAJPJL@?$CG?$CG@ 1002082c     libvcruntime:undname.obj
 0002:00003830       ??_C@_02NONPIBCD@?$HM?$HM@ 10020830     libvcruntime:undname.obj
 0002:00003834       ??_C@_02FPIMKNGF@?$CK?$DN@ 10020834     libvcruntime:undname.obj
 0002:00003838       ??_C@_02FOEOMHFC@?$CL?$DN@ 10020838     libvcruntime:undname.obj
 0002:0000383c       ??_C@_02FKMDLLOA@?9?$DN@   1002083c     libvcruntime:undname.obj
 0002:00003840       ??_C@_02FJEHGPIO@?1?$DN@   10020840     libvcruntime:undname.obj
 0002:00003844       ??_C@_02FENAOKFI@?$CF?$DN@ 10020844     libvcruntime:undname.obj
 0002:00003848       ??_C@_03IKFCCPFF@?$DO?$DO?$DN@ 10020848     libvcruntime:undname.obj
 0002:0000384c       ??_C@_03CDNPDDLA@?$DM?$DM?$DN@ 1002084c     libvcruntime:undname.obj
 0002:00003850       ??_C@_02FGJGFEAB@?$CG?$DN@ 10020850     libvcruntime:undname.obj
 0002:00003854       ??_C@_02DHLNPPGH@?$HM?$DN@ 10020854     libvcruntime:undname.obj
 0002:00003858       ??_C@_02MHEGNOJ@?$FO?$DN@  10020858     libvcruntime:undname.obj
 0002:0000385c       ??_C@_09IFPLHPGF@?$GAvftable?8@ 1002085c     libvcruntime:undname.obj
 0002:00003868       ??_C@_09BLBHBJP@?$GAvbtable?8@ 10020868     libvcruntime:undname.obj
 0002:00003874       ??_C@_07FEEIOKP@?$GAvcall?8@ 10020874     libvcruntime:undname.obj
 0002:0000387c       ??_C@_08LLFFHHDJ@?$GAtypeof?8@ 1002087c     libvcruntime:undname.obj
 0002:00003888       ??_C@_0BF@KDPPACIK@?$GAlocal?5static?5guard?8@ 10020888     libvcruntime:undname.obj
 0002:000038a0       ??_C@_08OBABFOLI@?$GAstring?8@ 100208a0     libvcruntime:undname.obj
 0002:000038ac       ??_C@_0BD@JDLKDPAB@?$GAvbase?5destructor?8@ 100208ac     libvcruntime:undname.obj
 0002:000038c0       ??_C@_0BN@DEGPLNFK@?$GAvector?5deleting?5destructor?8@ 100208c0     libvcruntime:undname.obj
 0002:000038e0       ??_C@_0BO@OBMKPJIG@?$GAdefault?5constructor?5closure?8@ 100208e0     libvcruntime:undname.obj
 0002:00003900       ??_C@_0BN@IMDCHIKM@?$GAscalar?5deleting?5destructor?8@ 10020900     libvcruntime:undname.obj
 0002:00003920       ??_C@_0BO@PFGOCPJJ@?$GAvector?5constructor?5iterator?8@ 10020920     libvcruntime:undname.obj
 0002:00003940       ??_C@_0BN@LFPFMEDL@?$GAvector?5destructor?5iterator?8@ 10020940     libvcruntime:undname.obj
 0002:00003960       ??_C@_0CE@IKBNEHA@?$GAvector?5vbase?5constructor?5itera@ 10020960     libvcruntime:undname.obj
 0002:00003984       ??_C@_0BL@NILFHHPC@?$GAvirtual?5displacement?5map?8@ 10020984     libvcruntime:undname.obj
 0002:000039a0       ??_C@_0CB@JONCMFFK@?$GAeh?5vector?5constructor?5iterator@ 100209a0     libvcruntime:undname.obj
 0002:000039c4       ??_C@_0CA@GCEOPDGL@?$GAeh?5vector?5destructor?5iterator?8@ 100209c4     libvcruntime:undname.obj
 0002:000039e4       ??_C@_0CH@OOJPLCPH@?$GAeh?5vector?5vbase?5constructor?5it@ 100209e4     libvcruntime:undname.obj
 0002:00003a0c       ??_C@_0BL@LLKPOHJI@?$GAcopy?5constructor?5closure?8@ 10020a0c     libvcruntime:undname.obj
 0002:00003a28       ??_C@_0BA@KBCDOMBN@?$GAudt?5returning?8@ 10020a28     libvcruntime:undname.obj
 0002:00003a38       ??_C@_03KLGMFNMG@?$GAEH@   10020a38     libvcruntime:undname.obj
 0002:00003a3c       ??_C@_05KHLCHHI@?$GARTTI@  10020a3c     libvcruntime:undname.obj
 0002:00003a44       ??_C@_0BA@KKLDJDLB@?$GAlocal?5vftable?8@ 10020a44     libvcruntime:undname.obj
 0002:00003a54       ??_C@_0CE@IIHCMGGL@?$GAlocal?5vftable?5constructor?5clos@ 10020a54     libvcruntime:undname.obj
 0002:00003a78       ??_C@_06FHBGPFGH@?5new?$FL?$FN@ 10020a78     libvcruntime:undname.obj
 0002:00003a80       ??_C@_09LBNFPBCA@?5delete?$FL?$FN@ 10020a80     libvcruntime:undname.obj
 0002:00003a8c       ??_C@_0P@HJKNJFNN@?$GAomni?5callsig?8@ 10020a8c     libvcruntime:undname.obj
 0002:00003a9c       ??_C@_0BL@CNOONJFP@?$GAplacement?5delete?5closure?8@ 10020a9c     libvcruntime:undname.obj
 0002:00003ab8       ??_C@_0BN@CKNJLHMB@?$GAplacement?5delete?$FL?$FN?5closure?8@ 10020ab8     libvcruntime:undname.obj
 0002:00003ad8       ??_C@_0CG@CFDHKGGD@?$GAmanaged?5vector?5constructor?5ite@ 10020ad8     libvcruntime:undname.obj
 0002:00003b00       ??_C@_0CF@IMGKMJNO@?$GAmanaged?5vector?5destructor?5iter@ 10020b00     libvcruntime:undname.obj
 0002:00003b28       ??_C@_0CG@HLDDJMAG@?$GAeh?5vector?5copy?5constructor?5ite@ 10020b28     libvcruntime:undname.obj
 0002:00003b50       ??_C@_0CM@FCBBDIGB@?$GAeh?5vector?5vbase?5copy?5construct@ 10020b50     libvcruntime:undname.obj
 0002:00003b7c       ??_C@_0BL@CLIPGLGB@?$GAdynamic?5initializer?5for?5?8@ 10020b7c     libvcruntime:undname.obj
 0002:00003b98       ??_C@_0CB@PDBIFEP@?$GAdynamic?5atexit?5destructor?5for?5@ 10020b98     libvcruntime:undname.obj
 0002:00003bbc       ??_C@_0CD@CGAJBKEJ@?$GAvector?5copy?5constructor?5iterat@ 10020bbc     libvcruntime:undname.obj
 0002:00003be0       ??_C@_0CJ@GJELGAMM@?$GAvector?5vbase?5copy?5constructor?5@ 10020be0     libvcruntime:undname.obj
 0002:00003c0c       ??_C@_0CL@FGIJHLCE@?$GAmanaged?5vector?5copy?5constructo@ 10020c0c     libvcruntime:undname.obj
 0002:00003c38       ??_C@_0BM@PMGGMLDN@?$GAlocal?5static?5thread?5guard?8@ 10020c38     libvcruntime:undname.obj
 0002:00003c54       ??_C@_0N@BDNMDMOL@operator?5?$CC?$CC?5@ 10020c54     libvcruntime:undname.obj
 0002:00003c64       ??_C@_0BC@GGEBGALA@operator?5co_await@ 10020c64     libvcruntime:undname.obj
 0002:00003c78       ??_C@_0BC@DAFEJGAK@?5Type?5Descriptor?8@ 10020c78     libvcruntime:undname.obj
 0002:00003c8c       ??_C@_0BM@LDKODKLH@?5Base?5Class?5Descriptor?5at?5?$CI@ 10020c8c     libvcruntime:undname.obj
 0002:00003ca8       ??_C@_0BD@LGICGFMM@?5Base?5Class?5Array?8@ 10020ca8     libvcruntime:undname.obj
 0002:00003cbc       ??_C@_0BN@MECKDCOJ@?5Class?5Hierarchy?5Descriptor?8@ 10020cbc     libvcruntime:undname.obj
 0002:00003cdc       ??_C@_0BK@CFCOFLF@?5Complete?5Object?5Locator?8@ 10020cdc     libvcruntime:undname.obj
 0002:00003d04       ??_C@_1DM@KHCHBNEB@?$AAa?$AAp?$AAi?$AA?9?$AAm?$AAs?$AA?9?$AAw?$AAi?$AAn?$AA?9?$AAc?$AAo?$AAr?$AAe@ 10020d04     libvcruntime:winapi_downlevel.obj
 0002:00003d40       ??_C@_1DK@LPPGFMPP@?$AAa?$AAp?$AAi?$AA?9?$AAm?$AAs?$AA?9?$AAw?$AAi?$AAn?$AA?9?$AAc?$AAo?$AAr?$AAe@ 10020d40     libvcruntime:winapi_downlevel.obj
 0002:00003d7c       ??_C@_1BC@GDMECMAK@?$AAk?$AAe?$AAr?$AAn?$AAe?$AAl?$AA3?$AA2@ 10020d7c     libvcruntime:winapi_downlevel.obj
 0002:00003d90       ??_C@_1BA@PFFKHIOG@?$AAa?$AAp?$AAi?$AA?9?$AAm?$AAs?$AA?9@ 10020d90     libvcruntime:winapi_downlevel.obj
 0002:00003da0       ??_C@_1BA@IAIFMGEF@?$AAe?$AAx?$AAt?$AA?9?$AAm?$AAs?$AA?9@ 10020da0     libvcruntime:winapi_downlevel.obj
 0002:00003db8       ??_C@_08KNHFBNJ@FlsAlloc@  10020db8     libvcruntime:winapi_downlevel.obj
 0002:00003dcc       ??_C@_07PEJMOBNF@FlsFree@  10020dcc     libvcruntime:winapi_downlevel.obj
 0002:00003ddc       ??_C@_0M@GDNOONDI@FlsGetValue@ 10020ddc     libvcruntime:winapi_downlevel.obj
 0002:00003df0       ??_C@_0M@JCPCPOEF@FlsSetValue@ 10020df0     libvcruntime:winapi_downlevel.obj
 0002:00003e04       ??_C@_0BM@HCFOFFN@InitializeCriticalSectionEx@ 10020e04     libvcruntime:winapi_downlevel.obj
 0002:00003e24       ??_7bad_exception@std@@6B@ 10020e24     libvcruntime:frame.obj
 0002:00003e2c       ??_C@_0O@DPKOEFFH@bad?5exception@ 10020e2c     libvcruntime:frame.obj
 0002:00003e3c       __pDestructExceptionObject 10020e3c     libvcruntime:ehhelpers.obj
 0002:00003e40       ?standard_lookup_table_spectre@__crt_stdio_output@@3V?$spectre_mitigated_lookup_table@Ustate_transition_pair@__crt_stdio_output@@$0IA@@1@B 10020e40     libucrt:output.obj
 0002:00003f40       ??_C@_1O@CEDCILHN@?$AA?$CI?$AAn?$AAu?$AAl?$AAl?$AA?$CJ@ 10020f40     libucrt:output.obj
 0002:00003f50       ??_C@_06OJHGLDPL@?$CInull?$CJ@ 10020f50     libucrt:output.obj
 0002:00003f58       ___acrt_exception_action_table 10020f58     libucrt:exception_filter.obj
 0002:00003fe8       ___acrt_signal_action_table_count 10020fe8     libucrt:exception_filter.obj
 0002:00003fec       ___acrt_signal_action_first_fpe_index 10020fec     libucrt:exception_filter.obj
 0002:00003ff0       ___acrt_signal_action_fpe_count 10020ff0     libucrt:exception_filter.obj
 0002:00003ff4       ??_C@_1BI@BGOHAHKC@?$AAm?$AAs?$AAc?$AAo?$AAr?$AAe?$AAe?$AA?4?$AAd?$AAl?$AAl@ 10020ff4     libucrt:exit.obj
 0002:0000400c       ??_C@_0P@MIGLKIOC@CorExitProcess@ 1002100c     libucrt:exit.obj
 0002:00004260       ??_C@_1EA@JGEFHKEI@?$AAa?$AAp?$AAi?$AA?9?$AAm?$AAs?$AA?9?$AAw?$AAi?$AAn?$AA?9?$AAc?$AAo?$AAr?$AAe@ 10021260     libucrt:winapi_thunks.obj
 0002:000042a0       ??_C@_1DI@KMEPCBPN@?$AAa?$AAp?$AAi?$AA?9?$AAm?$AAs?$AA?9?$AAw?$AAi?$AAn?$AA?9?$AAc?$AAo?$AAr?$AAe@ 100212a0     libucrt:winapi_thunks.obj
 0002:000042d8       ??_C@_1DI@IJCEHOCB@?$AAa?$AAp?$AAi?$AA?9?$AAm?$AAs?$AA?9?$AAw?$AAi?$AAn?$AA?9?$AAc?$AAo?$AAr?$AAe@ 100212d8     libucrt:winapi_thunks.obj
 0002:00004310       ??_C@_1EI@MPIAOHOC@?$AAa?$AAp?$AAi?$AA?9?$AAm?$AAs?$AA?9?$AAw?$AAi?$AAn?$AA?9?$AAc?$AAo?$AAr?$AAe@ 10021310     libucrt:winapi_thunks.obj
 0002:00004358       ??_C@_1FK@FPHCKFIE@?$AAa?$AAp?$AAi?$AA?9?$AAm?$AAs?$AA?9?$AAw?$AAi?$AAn?$AA?9?$AAc?$AAo?$AAr?$AAe@ 10021358     libucrt:winapi_thunks.obj
 0002:000043b8       ??_C@_1EM@DILCGIIO@?$AAa?$AAp?$AAi?$AA?9?$AAm?$AAs?$AA?9?$AAw?$AAi?$AAn?$AA?9?$AAc?$AAo?$AAr?$AAe@ 100213b8     libucrt:winapi_thunks.obj
 0002:00004404       ??_C@_1DM@LNCGDDPN@?$AAa?$AAp?$AAi?$AA?9?$AAm?$AAs?$AA?9?$AAw?$AAi?$AAn?$AA?9?$AAc?$AAo?$AAr?$AAe@ 10021404     libucrt:winapi_thunks.obj
 0002:00004440       ??_C@_1DO@FPAPJEMD@?$AAa?$AAp?$AAi?$AA?9?$AAm?$AAs?$AA?9?$AAw?$AAi?$AAn?$AA?9?$AAc?$AAo?$AAr?$AAe@ 10021440     libucrt:winapi_thunks.obj
 0002:00004480       ??_C@_1DK@NDHNAHIO@?$AAa?$AAp?$AAi?$AA?9?$AAm?$AAs?$AA?9?$AAw?$AAi?$AAn?$AA?9?$AAc?$AAo?$AAr?$AAe@ 10021480     libucrt:winapi_thunks.obj
 0002:000044bc       ??_C@_1DM@KGHDGBCM@?$AAa?$AAp?$AAi?$AA?9?$AAm?$AAs?$AA?9?$AAw?$AAi?$AAn?$AA?9?$AAc?$AAo?$AAr?$AAe@ 100214bc     libucrt:winapi_thunks.obj
 0002:000044f8       ??_C@_1EO@IJIOEFOH@?$AAa?$AAp?$AAi?$AA?9?$AAm?$AAs?$AA?9?$AAw?$AAi?$AAn?$AA?9?$AAr?$AAt?$AAc?$AAo@ 100214f8     libucrt:winapi_thunks.obj
 0002:00004548       ??_C@_1FG@HHGEKANL@?$AAa?$AAp?$AAi?$AA?9?$AAm?$AAs?$AA?9?$AAw?$AAi?$AAn?$AA?9?$AAs?$AAe?$AAc?$AAu@ 10021548     libucrt:winapi_thunks.obj
 0002:000045a0       ??_C@_1EG@DBIOJECG@?$AAe?$AAx?$AAt?$AA?9?$AAm?$AAs?$AA?9?$AAw?$AAi?$AAn?$AA?9?$AAn?$AAt?$AAu?$AAs@ 100215a0     libucrt:winapi_thunks.obj
 0002:000045e8       ??_C@_1EO@FIHMJCLF@?$AAe?$AAx?$AAt?$AA?9?$AAm?$AAs?$AA?9?$AAw?$AAi?$AAn?$AA?9?$AAn?$AAt?$AAu?$AAs@ 100215e8     libucrt:winapi_thunks.obj
 0002:00004638       ??_C@_1BC@DNHGCMLG@?$AAa?$AAd?$AAv?$AAa?$AAp?$AAi?$AA3?$AA2@ 10021638     libucrt:winapi_thunks.obj
 0002:0000464c       ??_C@_1BG@CJPGBMEF@?$AAk?$AAe?$AAr?$AAn?$AAe?$AAl?$AAb?$AAa?$AAs?$AAe@ 1002164c     libucrt:winapi_thunks.obj
 0002:00004664       ??_C@_1M@OAIMIKLP@?$AAn?$AAt?$AAd?$AAl?$AAl@ 10021664     libucrt:winapi_thunks.obj
 0002:00004670       ??_C@_1EG@DPGNFKGC@?$AAa?$AAp?$AAi?$AA?9?$AAm?$AAs?$AA?9?$AAw?$AAi?$AAn?$AA?9?$AAa?$AAp?$AAp?$AAm@ 10021670     libucrt:winapi_thunks.obj
 0002:000046b8       ??_C@_1O@BCCLBEOE@?$AAu?$AAs?$AAe?$AAr?$AA3?$AA2@ 100216b8     libucrt:winapi_thunks.obj
 0002:000046c8       ??_C@_1DM@BPJLHKCE@?$AAa?$AAp?$AAi?$AA?9?$AAm?$AAs?$AA?9?$AAw?$AAi?$AAn?$AA?9?$AAc?$AAo?$AAr?$AAe@ 100216c8     libucrt:winapi_thunks.obj
 0002:00004708       ??_C@_0BA@FHFNEAED@AreFileApisANSI@ 10021708     libucrt:winapi_thunks.obj
 0002:00004720       ??_C@_0BA@IHGNDAEB@CompareStringEx@ 10021720     libucrt:winapi_thunks.obj
 0002:00004740       ??_C@_0O@KKBNKAPF@LCMapStringEx@ 10021740     libucrt:winapi_thunks.obj
 0002:00004758       ??_C@_0BB@HBDEELFH@LocaleNameToLCID@ 10021758     libucrt:winapi_thunks.obj
 0002:00004770       ??_C@_0CF@OJOFEIGO@AppPolicyGetProcessTerminationM@ 10021770     libucrt:winapi_thunks.obj
 0002:000047f8       ??_C@_03OEIAHPBN@INF@      100217f8     libucrt:cvt.obj
 0002:000047fc       ??_C@_03OJHLLCGB@inf@      100217fc     libucrt:cvt.obj
 0002:00004800       ??_C@_03LKNCIKJB@NAN@      10021800     libucrt:cvt.obj
 0002:00004804       ??_C@_03LHCJEHON@nan@      10021804     libucrt:cvt.obj
 0002:00004808       ??_C@_09OFJJIMPC@NAN?$CISNAN?$CJ@ 10021808     libucrt:cvt.obj
 0002:00004814       ??_C@_09IPFBKMDL@nan?$CIsnan?$CJ@ 10021814     libucrt:cvt.obj
 0002:00004820       ??_C@_08IKHNHAJ@NAN?$CIIND?$CJ@ 10021820     libucrt:cvt.obj
 0002:0000482c       ??_C@_08OFCDMILK@nan?$CIind?$CJ@ 1002182c     libucrt:cvt.obj
 0002:00004838       ??_C@_05KLBDPFGC@e?$CL000@ 10021838     libucrt:cvt.obj
 0002:00004840       ___lc_time_c               10021840     libucrt:nlsdata.obj
 0002:000049a4       ??_C@_03KOEHGMDN@Sun@      100219a4     libucrt:nlsdata.obj
 0002:000049a8       ??_C@_03PDAGKDH@Mon@       100219a8     libucrt:nlsdata.obj
 0002:000049ac       ??_C@_03NAGEINEP@Tue@      100219ac     libucrt:nlsdata.obj
 0002:000049b0       ??_C@_03MHOMLAJA@Wed@      100219b0     libucrt:nlsdata.obj
 0002:000049b4       ??_C@_03IOFIKPDN@Thu@      100219b4     libucrt:nlsdata.obj
 0002:000049b8       ??_C@_03IDIOELNC@Fri@      100219b8     libucrt:nlsdata.obj
 0002:000049bc       ??_C@_03FEFJNEK@Sat@       100219bc     libucrt:nlsdata.obj
 0002:000049c0       ??_C@_06OOPIFAJ@Sunday@    100219c0     libucrt:nlsdata.obj
 0002:000049c8       ??_C@_06JLEDEDGH@Monday@   100219c8     libucrt:nlsdata.obj
 0002:000049d0       ??_C@_07BAAGCFCM@Tuesday@  100219d0     libucrt:nlsdata.obj
 0002:000049d8       ??_C@_09DLIGFAKA@Wednesday@ 100219d8     libucrt:nlsdata.obj
 0002:000049e4       ??_C@_08HACCIKIA@Thursday@ 100219e4     libucrt:nlsdata.obj
 0002:000049f0       ??_C@_06JECMNKMI@Friday@   100219f0     libucrt:nlsdata.obj
 0002:000049f8       ??_C@_08INBOOONO@Saturday@ 100219f8     libucrt:nlsdata.obj
 0002:00004a04       ??_C@_03JIHJHPIE@Jan@      10021a04     libucrt:nlsdata.obj
 0002:00004a08       ??_C@_03HJBDCHOM@Feb@      10021a08     libucrt:nlsdata.obj
 0002:00004a0c       ??_C@_03ODNJBKGA@Mar@      10021a0c     libucrt:nlsdata.obj
 0002:00004a10       ??_C@_03LEOLGMJP@Apr@      10021a10     libucrt:nlsdata.obj
 0002:00004a14       ??_C@_03CNMDKL@May@        10021a14     libucrt:nlsdata.obj
 0002:00004a18       ??_C@_03IDFGHECI@Jun@      10021a18     libucrt:nlsdata.obj
 0002:00004a1c       ??_C@_03LBGABGKK@Jul@      10021a1c     libucrt:nlsdata.obj
 0002:00004a20       ??_C@_03IFJFEIGA@Aug@      10021a20     libucrt:nlsdata.obj
 0002:00004a24       ??_C@_03GGCAPAJC@Sep@      10021a24     libucrt:nlsdata.obj
 0002:00004a28       ??_C@_03BMAOKBAD@Oct@      10021a28     libucrt:nlsdata.obj
 0002:00004a2c       ??_C@_03JPJOFNIA@Nov@      10021a2c     libucrt:nlsdata.obj
 0002:00004a30       ??_C@_03MKABNOCG@Dec@      10021a30     libucrt:nlsdata.obj
 0002:00004a34       ??_C@_07CGJPFGJA@January@  10021a34     libucrt:nlsdata.obj
 0002:00004a3c       ??_C@_08GNJGEPFN@February@ 10021a3c     libucrt:nlsdata.obj
 0002:00004a48       ??_C@_05HPCKOFNC@March@    10021a48     libucrt:nlsdata.obj
 0002:00004a50       ??_C@_05DMJDNLEJ@April@    10021a50     libucrt:nlsdata.obj
 0002:00004a58       ??_C@_04CNLMGBGM@June@     10021a58     libucrt:nlsdata.obj
 0002:00004a60       ??_C@_04MIEPOIFP@July@     10021a60     libucrt:nlsdata.obj
 0002:00004a68       ??_C@_06LBBHFDDG@August@   10021a68     libucrt:nlsdata.obj
 0002:00004a70       ??_C@_09BHHEALKD@September@ 10021a70     libucrt:nlsdata.obj
 0002:00004a7c       ??_C@_07JJNFCEND@October@  10021a7c     libucrt:nlsdata.obj
 0002:00004a84       ??_C@_08HCHEGEOA@November@ 10021a84     libucrt:nlsdata.obj
 0002:00004a90       ??_C@_08EDHMEBNP@December@ 10021a90     libucrt:nlsdata.obj
 0002:00004a9c       ??_C@_02DEDBPAFC@AM@       10021a9c     libucrt:nlsdata.obj
 0002:00004aa0       ??_C@_02CJNFDJBF@PM@       10021aa0     libucrt:nlsdata.obj
 0002:00004aa4       ??_C@_08BPBNCDIB@MM?1dd?1yy@ 10021aa4     libucrt:nlsdata.obj
 0002:00004ab0       ??_C@_0BE@CKGJFCPC@dddd?0?5MMMM?5dd?0?5yyyy@ 10021ab0     libucrt:nlsdata.obj
 0002:00004ac4       ??_C@_08JCCMCCIL@HH?3mm?3ss@ 10021ac4     libucrt:nlsdata.obj
 0002:00004ad0       ??_C@_17MBGCMIPB@?$AAS?$AAu?$AAn@ 10021ad0     libucrt:nlsdata.obj
 0002:00004ad8       ??_C@_17KBOMKBF@?$AAM?$AAo?$AAn@ 10021ad8     libucrt:nlsdata.obj
 0002:00004ae0       ??_C@_17BMKGEGOJ@?$AAT?$AAu?$AAe@ 10021ae0     libucrt:nlsdata.obj
 0002:00004ae8       ??_C@_17CJEDCEPE@?$AAW?$AAe?$AAd@ 10021ae8     libucrt:nlsdata.obj
 0002:00004af0       ??_C@_17PDPHAADD@?$AAT?$AAh?$AAu@ 10021af0     libucrt:nlsdata.obj
 0002:00004af8       ??_C@_17HFOLPPLP@?$AAF?$AAr?$AAi@ 10021af8     libucrt:nlsdata.obj
 0002:00004b00       ??_C@_17GGIBDPIH@?$AAS?$AAa?$AAt@ 10021b00     libucrt:nlsdata.obj
 0002:00004b08       ??_C@_1O@IHNHDHPB@?$AAS?$AAu?$AAn?$AAd?$AAa?$AAy@ 10021b08     libucrt:nlsdata.obj
 0002:00004b18       ??_C@_1O@MMNBFLIA@?$AAM?$AAo?$AAn?$AAd?$AAa?$AAy@ 10021b18     libucrt:nlsdata.obj
 0002:00004b28       ??_C@_1BA@ENFBFFEK@?$AAT?$AAu?$AAe?$AAs?$AAd?$AAa?$AAy@ 10021b28     libucrt:nlsdata.obj
 0002:00004b38       ??_C@_1BE@EBOGMDOH@?$AAW?$AAe?$AAd?$AAn?$AAe?$AAs?$AAd?$AAa?$AAy@ 10021b38     libucrt:nlsdata.obj
 0002:00004b4c       ??_C@_1BC@HHMNLIHE@?$AAT?$AAh?$AAu?$AAr?$AAs?$AAd?$AAa?$AAy@ 10021b4c     libucrt:nlsdata.obj
 0002:00004b60       ??_C@_1O@PDICJHAG@?$AAF?$AAr?$AAi?$AAd?$AAa?$AAy@ 10021b60     libucrt:nlsdata.obj
 0002:00004b70       ??_C@_1BC@ENMNNPAJ@?$AAS?$AAa?$AAt?$AAu?$AAr?$AAd?$AAa?$AAy@ 10021b70     libucrt:nlsdata.obj
 0002:00004b84       ??_C@_17DKNBKCHM@?$AAJ?$AAa?$AAn@ 10021b84     libucrt:nlsdata.obj
 0002:00004b8c       ??_C@_17LMDJEKJN@?$AAF?$AAe?$AAb@ 10021b8c     libucrt:nlsdata.obj
 0002:00004b94       ??_C@_17CKNLEDEC@?$AAM?$AAa?$AAr@ 10021b94     libucrt:nlsdata.obj
 0002:00004b9c       ??_C@_17LFPOIHDD@?$AAA?$AAp?$AAr@ 10021b9c     libucrt:nlsdata.obj
 0002:00004ba4       ??_C@_17PNNKMEED@?$AAM?$AAa?$AAy@ 10021ba4     libucrt:nlsdata.obj
 0002:00004bac       ??_C@_17KCJGOCPB@?$AAJ?$AAu?$AAn@ 10021bac     libucrt:nlsdata.obj
 0002:00004bb4       ??_C@_17IJPCKHK@?$AAJ?$AAu?$AAl@ 10021bb4     libucrt:nlsdata.obj
 0002:00004bbc       ??_C@_17ICPELBCN@?$AAA?$AAu?$AAg@ 10021bbc     libucrt:nlsdata.obj
 0002:00004bc4       ??_C@_17HCHCOKMG@?$AAS?$AAe?$AAp@ 10021bc4     libucrt:nlsdata.obj
 0002:00004bcc       ??_C@_17FNLKOI@?$AAO?$AAc?$AAt@ 10021bcc     libucrt:nlsdata.obj
 0002:00004bd4       ??_C@_17BBDMLCIG@?$AAN?$AAo?$AAv@ 10021bd4     libucrt:nlsdata.obj
 0002:00004bdc       ??_C@_17EGKACKIF@?$AAD?$AAe?$AAc@ 10021bdc     libucrt:nlsdata.obj
 0002:00004be4       ??_C@_1BA@EFMEIEBA@?$AAJ?$AAa?$AAn?$AAu?$AAa?$AAr?$AAy@ 10021be4     libucrt:nlsdata.obj
 0002:00004bf4       ??_C@_1BC@JGDDFFAM@?$AAF?$AAe?$AAb?$AAr?$AAu?$AAa?$AAr?$AAy@ 10021bf4     libucrt:nlsdata.obj
 0002:00004c08       ??_C@_1M@IKEENEDF@?$AAM?$AAa?$AAr?$AAc?$AAh@ 10021c08     libucrt:nlsdata.obj
 0002:00004c14       ??_C@_1M@GJNLMHFD@?$AAA?$AAp?$AAr?$AAi?$AAl@ 10021c14     libucrt:nlsdata.obj
 0002:00004c20       ??_C@_19EPFLPGAP@?$AAJ?$AAu?$AAn?$AAe@ 10021c20     libucrt:nlsdata.obj
 0002:00004c2c       ??_C@_19BIFMLPCD@?$AAJ?$AAu?$AAl?$AAy@ 10021c2c     libucrt:nlsdata.obj
 0002:00004c38       ??_C@_1O@PAHLKOAC@?$AAA?$AAu?$AAg?$AAu?$AAs?$AAt@ 10021c38     libucrt:nlsdata.obj
 0002:00004c48       ??_C@_1BE@DKAAMBJL@?$AAS?$AAe?$AAp?$AAt?$AAe?$AAm?$AAb?$AAe?$AAr@ 10021c48     libucrt:nlsdata.obj
 0002:00004c5c       ??_C@_1BA@EPANDLNG@?$AAO?$AAc?$AAt?$AAo?$AAb?$AAe?$AAr@ 10021c5c     libucrt:nlsdata.obj
 0002:00004c6c       ??_C@_1BC@BGLIFPF@?$AAN?$AAo?$AAv?$AAe?$AAm?$AAb?$AAe?$AAr@ 10021c6c     libucrt:nlsdata.obj
 0002:00004c80       ??_C@_1BC@FEMKIFH@?$AAD?$AAe?$AAc?$AAe?$AAm?$AAb?$AAe?$AAr@ 10021c80     libucrt:nlsdata.obj
 0002:00004c94       ??_C@_15ODEHAHHF@?$AAA?$AAM@ 10021c94     libucrt:nlsdata.obj
 0002:00004c9c       ??_C@_15CLMNNGEL@?$AAP?$AAM@ 10021c9c     libucrt:nlsdata.obj
 0002:00004ca4       ??_C@_1BC@IEBCMHCM@?$AAM?$AAM?$AA?1?$AAd?$AAd?$AA?1?$AAy?$AAy@ 10021ca4     libucrt:nlsdata.obj
 0002:00004cb8       ??_C@_1CI@KNAKOEBC@?$AAd?$AAd?$AAd?$AAd?$AA?0?$AA?5?$AAM?$AAM?$AAM?$AAM?$AA?5?$AAd?$AAd?$AA?0?$AA?5@ 10021cb8     libucrt:nlsdata.obj
 0002:00004ce0       ??_C@_1BC@GDGBMEMK@?$AAH?$AAH?$AA?3?$AAm?$AAm?$AA?3?$AAs?$AAs@ 10021ce0     libucrt:nlsdata.obj
 0002:00004cf4       ??_C@_1M@BMHNFIME@?$AAe?$AAn?$AA?9?$AAU?$AAS@ 10021cf4     libucrt:nlsdata.obj
 0002:00004d00       ?ccs@?1???$__acrt_stdio_parse_mode@D@@YA?AU__acrt_stdio_stream_mode@@QBD@Z@4QBDB 10021d00     libucrt:openfile.obj
 0002:00004d04       ?utf8_encoding@?1???$__acrt_stdio_parse_mode@D@@YA?AU__acrt_stdio_stream_mode@@QBD@Z@4QBDB 10021d04     libucrt:openfile.obj
 0002:00004d0c       ?utf16_encoding@?1???$__acrt_stdio_parse_mode@D@@YA?AU__acrt_stdio_stream_mode@@QBD@Z@4QBDB 10021d0c     libucrt:openfile.obj
 0002:00004d14       ?unicode_encoding@?1???$__acrt_stdio_parse_mode@D@@YA?AU__acrt_stdio_stream_mode@@QBD@Z@4QBDB 10021d14     libucrt:openfile.obj
 0002:00004d2c       ??_C@_1M@HPNHIDJI@?$AAj?$AAa?$AA?9?$AAJ?$AAP@ 10021d2c     libucrt:mbctype.obj
 0002:00004d38       ??_C@_1M@BIBDDEMK@?$AAz?$AAh?$AA?9?$AAC?$AAN@ 10021d38     libucrt:mbctype.obj
 0002:00004d44       ??_C@_1M@JLOOOEGK@?$AAk?$AAo?$AA?9?$AAK?$AAR@ 10021d44     libucrt:mbctype.obj
 0002:00004d50       ??_C@_1M@CLNBBOPM@?$AAz?$AAh?$AA?9?$AAT?$AAW@ 10021d50     libucrt:mbctype.obj
 0002:00004d60       ___newctype                10021d60     libucrt:ctype.obj
 0002:00005060       ___newclmap                10022060     libucrt:ctype.obj
 0002:000051e0       ___newcumap                100221e0     libucrt:ctype.obj
 0002:00005a80       ??_C@_15EMKDOKLE@?$AAa?$AAr@ 10022a80     libucrt:lcidtoname_downlevel.obj
 0002:00005a88       ??_C@_15KNPADPLH@?$AAb?$AAg@ 10022a88     libucrt:lcidtoname_downlevel.obj
 0002:00005a90       ??_C@_15EDMHLDMO@?$AAc?$AAa@ 10022a90     libucrt:lcidtoname_downlevel.obj
 0002:00005a98       ??_C@_1O@BPEAJADD@?$AAz?$AAh?$AA?9?$AAC?$AAH?$AAS@ 10022a98     libucrt:lcidtoname_downlevel.obj
 0002:00005aa8       ??_C@_15LJNHCMNK@?$AAc?$AAs@ 10022aa8     libucrt:lcidtoname_downlevel.obj
 0002:00005ab0       ??_C@_15FOMCIDHG@?$AAd?$AAa@ 10022ab0     libucrt:lcidtoname_downlevel.obj
 0002:00005ab8       ??_C@_15NBKABECB@?$AAd?$AAe@ 10022ab8     libucrt:lcidtoname_downlevel.obj
 0002:00005ac0       ??_C@_15GHPEIIAO@?$AAe?$AAl@ 10022ac0     libucrt:lcidtoname_downlevel.obj
 0002:00005ac8       ??_C@_15MNPNEAIF@?$AAe?$AAn@ 10022ac8     libucrt:lcidtoname_downlevel.obj
 0002:00005ad0       ??_C@_15GPIOMPMH@?$AAe?$AAs@ 10022ad0     libucrt:lcidtoname_downlevel.obj
 0002:00005ad8       ??_C@_15NGLOAKJC@?$AAf?$AAi@ 10022ad8     libucrt:lcidtoname_downlevel.obj
 0002:00005ae0       ??_C@_15FBKGNKAM@?$AAf?$AAr@ 10022ae0     libucrt:lcidtoname_downlevel.obj
 0002:00005ae8       ??_C@_15KGGCNEFK@?$AAh?$AAe@ 10022ae8     libucrt:lcidtoname_downlevel.obj
 0002:00005af0       ??_C@_15PGHLIDMF@?$AAh?$AAu@ 10022af0     libucrt:lcidtoname_downlevel.obj
 0002:00005af8       ??_C@_15BIEMAPLM@?$AAi?$AAs@ 10022af8     libucrt:lcidtoname_downlevel.obj
 0002:00005b00       ??_C@_15IFJLDHAF@?$AAi?$AAt@ 10022b00     libucrt:lcidtoname_downlevel.obj
 0002:00005b08       ??_C@_15GEMIOCAG@?$AAj?$AAa@ 10022b08     libucrt:lcidtoname_downlevel.obj
 0002:00005b10       ??_C@_15EPELEGJA@?$AAk?$AAo@ 10022b10     libucrt:lcidtoname_downlevel.obj
 0002:00005b18       ??_C@_15NDDHIMN@?$AAn?$AAl@ 10022b18     libucrt:lcidtoname_downlevel.obj
 0002:00005b20       ??_C@_15BPIGNHCD@?$AAn?$AAo@ 10022b20     libucrt:lcidtoname_downlevel.obj
 0002:00005b28       ??_C@_15DEOPBLCG@?$AAp?$AAl@ 10022b28     libucrt:lcidtoname_downlevel.obj
 0002:00005b30       ??_C@_15KBECGEFG@?$AAp?$AAt@ 10022b30     libucrt:lcidtoname_downlevel.obj
 0002:00005b38       ??_C@_15GLJCBFMD@?$AAr?$AAo@ 10022b38     libucrt:lcidtoname_downlevel.obj
 0002:00005b40       ??_C@_15FEDGKCDI@?$AAr?$AAu@ 10022b40     libucrt:lcidtoname_downlevel.obj
 0002:00005b48       ??_C@_15GLKMLLHM@?$AAh?$AAr@ 10022b48     libucrt:lcidtoname_downlevel.obj
 0002:00005b50       ??_C@_15CPKMFBDB@?$AAs?$AAk@ 10022b50     libucrt:lcidtoname_downlevel.obj
 0002:00005b58       ??_C@_15BAAIOGMK@?$AAs?$AAq@ 10022b58     libucrt:lcidtoname_downlevel.obj
 0002:00005b60       ??_C@_15INNPNOHD@?$AAs?$AAv@ 10022b60     libucrt:lcidtoname_downlevel.obj
 0002:00005b68       ??_C@_15CABMMOGH@?$AAt?$AAh@ 10022b68     libucrt:lcidtoname_downlevel.obj
 0002:00005b70       ??_C@_15BPLIHJJM@?$AAt?$AAr@ 10022b70     libucrt:lcidtoname_downlevel.obj
 0002:00005b78       ??_C@_15NEOEKKDJ@?$AAu?$AAr@ 10022b78     libucrt:lcidtoname_downlevel.obj
 0002:00005b80       ??_C@_15NFICGAJK@?$AAi?$AAd@ 10022b80     libucrt:lcidtoname_downlevel.obj
 0002:00005b88       ??_C@_15PJPFLCCM@?$AAu?$AAk@ 10022b88     libucrt:lcidtoname_downlevel.obj
 0002:00005b90       ??_C@_15HPJPHDM@?$AAb?$AAe@ 10022b90     libucrt:lcidtoname_downlevel.obj
 0002:00005b98       ??_C@_15LCHLGJII@?$AAs?$AAl@ 10022b98     libucrt:lcidtoname_downlevel.obj
 0002:00005ba0       ??_C@_15PCFJPHHO@?$AAe?$AAt@ 10022ba0     libucrt:lcidtoname_downlevel.obj
 0002:00005ba8       ??_C@_15HPFPGODN@?$AAl?$AAv@ 10022ba8     libucrt:lcidtoname_downlevel.obj
 0002:00005bb0       ??_C@_15NFFGKGLG@?$AAl?$AAt@ 10022bb0     libucrt:lcidtoname_downlevel.obj
 0002:00005bb8       ??_C@_15BDAKCCHN@?$AAf?$AAa@ 10022bb8     libucrt:lcidtoname_downlevel.obj
 0002:00005bc0       ??_C@_15NFGIAIAJ@?$AAv?$AAi@ 10022bc0     libucrt:lcidtoname_downlevel.obj
 0002:00005bc8       ??_C@_15LMKNDMHN@?$AAh?$AAy@ 10022bc8     libucrt:lcidtoname_downlevel.obj
 0002:00005bd0       ??_C@_15IJBHMCFL@?$AAa?$AAz@ 10022bd0     libucrt:lcidtoname_downlevel.obj
 0002:00005bd8       ??_C@_15EKOFJABL@?$AAe?$AAu@ 10022bd8     libucrt:lcidtoname_downlevel.obj
 0002:00005be0       ??_C@_15BGHADCNK@?$AAm?$AAk@ 10022be0     libucrt:lcidtoname_downlevel.obj
 0002:00005be8       ??_C@_15JDNICKHM@?$AAa?$AAf@ 10022be8     libucrt:lcidtoname_downlevel.obj
 0002:00005bf0       ??_C@_15KPJEDBKD@?$AAk?$AAa@ 10022bf0     libucrt:lcidtoname_downlevel.obj
 0002:00005bf8       ??_C@_15PDNFFFEO@?$AAf?$AAo@ 10022bf8     libucrt:lcidtoname_downlevel.obj
 0002:00005c00       ??_C@_15OMLEGLOC@?$AAh?$AAi@ 10022c00     libucrt:lcidtoname_downlevel.obj
 0002:00005c08       ??_C@_15IDNNENKK@?$AAm?$AAs@ 10022c08     libucrt:lcidtoname_downlevel.obj
 0002:00005c10       ??_C@_15MACJNBMH@?$AAk?$AAk@ 10022c10     libucrt:lcidtoname_downlevel.obj
 0002:00005c18       ??_C@_15DKDJEOND@?$AAk?$AAy@ 10022c18     libucrt:lcidtoname_downlevel.obj
 0002:00005c20       ??_C@_15DFGDLJBG@?$AAs?$AAw@ 10022c20     libucrt:lcidtoname_downlevel.obj
 0002:00005c28       ??_C@_15BBFAICNG@?$AAu?$AAz@ 10022c28     libucrt:lcidtoname_downlevel.obj
 0002:00005c30       ??_C@_15DKNDCGEA@?$AAt?$AAt@ 10022c30     libucrt:lcidtoname_downlevel.obj
 0002:00005c38       ??_C@_15MGIFMDPL@?$AAp?$AAa@ 10022c38     libucrt:lcidtoname_downlevel.obj
 0002:00005c40       ??_C@_15HCNDBBA@?$AAg?$AAu@ 10022c40     libucrt:lcidtoname_downlevel.obj
 0002:00005c48       ??_C@_15FNBEIBON@?$AAt?$AAa@ 10022c48     libucrt:lcidtoname_downlevel.obj
 0002:00005c50       ??_C@_15NCHGBGLK@?$AAt?$AAe@ 10022c50     libucrt:lcidtoname_downlevel.obj
 0002:00005c58       ??_C@_15PHPHCBPF@?$AAk?$AAn@ 10022c58     libucrt:lcidtoname_downlevel.obj
 0002:00005c60       ??_C@_15DLGBCKMP@?$AAm?$AAr@ 10022c60     libucrt:lcidtoname_downlevel.obj
 0002:00005c68       ??_C@_15EABBLBFF@?$AAs?$AAa@ 10022c68     libucrt:lcidtoname_downlevel.obj
 0002:00005c70       ??_C@_15CBKOMCOI@?$AAm?$AAn@ 10022c70     libucrt:lcidtoname_downlevel.obj
 0002:00005c78       ??_C@_15CKDMCJAF@?$AAg?$AAl@ 10022c78     libucrt:lcidtoname_downlevel.obj
 0002:00005c80       ??_C@_17CNJFBPG@?$AAk?$AAo?$AAk@ 10022c80     libucrt:lcidtoname_downlevel.obj
 0002:00005c88       ??_C@_17FFBJICPL@?$AAs?$AAy?$AAr@ 10022c88     libucrt:lcidtoname_downlevel.obj
 0002:00005c90       ??_C@_17KPNDCPAF@?$AAd?$AAi?$AAv@ 10022c90     libucrt:lcidtoname_downlevel.obj
 0002:00005c98       ??_C@_11LOCGONAA@@         10022c98     libucrt:lcidtoname_downlevel.obj
 0002:00005c9c       ??_C@_1M@OKAHONE@?$AAa?$AAr?$AA?9?$AAS?$AAA@ 10022c9c     libucrt:lcidtoname_downlevel.obj
 0002:00005ca8       ??_C@_1M@FFFIGIGK@?$AAb?$AAg?$AA?9?$AAB?$AAG@ 10022ca8     libucrt:lcidtoname_downlevel.obj
 0002:00005cb4       ??_C@_1M@BJNKEDC@?$AAc?$AAa?$AA?9?$AAE?$AAS@ 10022cb4     libucrt:lcidtoname_downlevel.obj
 0002:00005cc0       ??_C@_1M@IJJHFJHA@?$AAc?$AAs?$AA?9?$AAC?$AAZ@ 10022cc0     libucrt:lcidtoname_downlevel.obj
 0002:00005ccc       ??_C@_1M@CLPEOBGI@?$AAd?$AAa?$AA?9?$AAD?$AAK@ 10022ccc     libucrt:lcidtoname_downlevel.obj
 0002:00005cd8       ??_C@_1M@MCMADGCB@?$AAd?$AAe?$AA?9?$AAD?$AAE@ 10022cd8     libucrt:lcidtoname_downlevel.obj
 0002:00005ce4       ??_C@_1M@OOCKEMAM@?$AAe?$AAl?$AA?9?$AAG?$AAR@ 10022ce4     libucrt:lcidtoname_downlevel.obj
 0002:00005cf0       ??_C@_1M@DDNJFGID@?$AAf?$AAi?$AA?9?$AAF?$AAI@ 10022cf0     libucrt:lcidtoname_downlevel.obj
 0002:00005cfc       ??_C@_1M@GLIPPMAC@?$AAf?$AAr?$AA?9?$AAF?$AAR@ 10022cfc     libucrt:lcidtoname_downlevel.obj
 0002:00005d08       ??_C@_1M@GFMCHPE@?$AAh?$AAe?$AA?9?$AAI?$AAL@ 10022d08     libucrt:lcidtoname_downlevel.obj
 0002:00005d14       ??_C@_1M@MHLPGNKM@?$AAh?$AAu?$AA?9?$AAH?$AAU@ 10022d14     libucrt:lcidtoname_downlevel.obj
 0002:00005d20       ??_C@_1M@LPDDNNPN@?$AAi?$AAs?$AA?9?$AAI?$AAS@ 10022d20     libucrt:lcidtoname_downlevel.obj
 0002:00005d2c       ??_C@_1M@MADIPODN@?$AAi?$AAt?$AA?9?$AAI?$AAT@ 10022d2c     libucrt:lcidtoname_downlevel.obj
 0002:00005d38       ??_C@_1M@IHBJJGG@?$AAn?$AAl?$AA?9?$AAN?$AAL@ 10022d38     libucrt:lcidtoname_downlevel.obj
 0002:00005d44       ??_C@_1M@EANAGDL@?$AAn?$AAb?$AA?9?$AAN?$AAO@ 10022d44     libucrt:lcidtoname_downlevel.obj
 0002:00005d50       ??_C@_1M@NEIEMEGP@?$AAp?$AAl?$AA?9?$AAP?$AAL@ 10022d50     libucrt:lcidtoname_downlevel.obj
 0002:00005d5c       ??_C@_1M@BOCFIGEP@?$AAp?$AAt?$AA?9?$AAB?$AAR@ 10022d5c     libucrt:lcidtoname_downlevel.obj
 0002:00005d68       ??_C@_1M@IMPFOPBG@?$AAr?$AAo?$AA?9?$AAR?$AAO@ 10022d68     libucrt:lcidtoname_downlevel.obj
 0002:00005d74       ??_C@_1M@IDNNEJMM@?$AAr?$AAu?$AA?9?$AAR?$AAU@ 10022d74     libucrt:lcidtoname_downlevel.obj
 0002:00005d80       ??_C@_1M@LILEEOGM@?$AAh?$AAr?$AA?9?$AAH?$AAR@ 10022d80     libucrt:lcidtoname_downlevel.obj
 0002:00005d8c       ??_C@_1M@FKIFEHPB@?$AAs?$AAk?$AA?9?$AAS?$AAK@ 10022d8c     libucrt:lcidtoname_downlevel.obj
 0002:00005d98       ??_C@_1M@LJMAMNPJ@?$AAs?$AAq?$AA?9?$AAA?$AAL@ 10022d98     libucrt:lcidtoname_downlevel.obj
 0002:00005da4       ??_C@_1M@GIAKDKJK@?$AAs?$AAv?$AA?9?$AAS?$AAE@ 10022da4     libucrt:lcidtoname_downlevel.obj
 0002:00005db0       ??_C@_1M@MKJKIKCL@?$AAt?$AAh?$AA?9?$AAT?$AAH@ 10022db0     libucrt:lcidtoname_downlevel.obj
 0002:00005dbc       ??_C@_1M@MFLCCMPB@?$AAt?$AAr?$AA?9?$AAT?$AAR@ 10022dbc     libucrt:lcidtoname_downlevel.obj
 0002:00005dc8       ??_C@_1M@OIJHDKJN@?$AAu?$AAr?$AA?9?$AAP?$AAK@ 10022dc8     libucrt:lcidtoname_downlevel.obj
 0002:00005dd4       ??_C@_1M@LHIPCIEK@?$AAi?$AAd?$AA?9?$AAI?$AAD@ 10022dd4     libucrt:lcidtoname_downlevel.obj
 0002:00005de0       ??_C@_1M@MFMOBGI@?$AAu?$AAk?$AA?9?$AAU?$AAA@ 10022de0     libucrt:lcidtoname_downlevel.obj
 0002:00005dec       ??_C@_1M@OBGLJIPL@?$AAb?$AAe?$AA?9?$AAB?$AAY@ 10022dec     libucrt:lcidtoname_downlevel.obj
 0002:00005df8       ??_C@_1M@BCFAJEAD@?$AAs?$AAl?$AA?9?$AAS?$AAI@ 10022df8     libucrt:lcidtoname_downlevel.obj
 0002:00005e04       ??_C@_1M@FKFFEDDN@?$AAe?$AAt?$AA?9?$AAE?$AAE@ 10022e04     libucrt:lcidtoname_downlevel.obj
 0002:00005e10       ??_C@_1M@KGKKAACI@?$AAl?$AAv?$AA?9?$AAL?$AAV@ 10022e10     libucrt:lcidtoname_downlevel.obj
 0002:00005e1c       ??_C@_1M@IFGBIJO@?$AAl?$AAt?$AA?9?$AAL?$AAT@ 10022e1c     libucrt:lcidtoname_downlevel.obj
 0002:00005e28       ??_C@_1M@FGEAHEDM@?$AAf?$AAa?$AA?9?$AAI?$AAR@ 10022e28     libucrt:lcidtoname_downlevel.obj
 0002:00005e34       ??_C@_1M@KBMAIBFN@?$AAv?$AAi?$AA?9?$AAV?$AAN@ 10022e34     libucrt:lcidtoname_downlevel.obj
 0002:00005e40       ??_C@_1M@GPCBKDJK@?$AAh?$AAy?$AA?9?$AAA?$AAM@ 10022e40     libucrt:lcidtoname_downlevel.obj
 0002:00005e4c       ??_C@_1BG@BECMDDJB@?$AAa?$AAz?$AA?9?$AAA?$AAZ?$AA?9?$AAL?$AAa?$AAt?$AAn@ 10022e4c     libucrt:lcidtoname_downlevel.obj
 0002:00005e64       ??_C@_1M@MAOFCAEA@?$AAe?$AAu?$AA?9?$AAE?$AAS@ 10022e64     libucrt:lcidtoname_downlevel.obj
 0002:00005e70       ??_C@_1M@IGHABKPI@?$AAm?$AAk?$AA?9?$AAM?$AAK@ 10022e70     libucrt:lcidtoname_downlevel.obj
 0002:00005e7c       ??_C@_1M@IAIGNEJG@?$AAt?$AAn?$AA?9?$AAZ?$AAA@ 10022e7c     libucrt:lcidtoname_downlevel.obj
 0002:00005e88       ??_C@_1M@IIJCOJFA@?$AAx?$AAh?$AA?9?$AAZ?$AAA@ 10022e88     libucrt:lcidtoname_downlevel.obj
 0002:00005e94       ??_C@_1M@LGPJHNJH@?$AAz?$AAu?$AA?9?$AAZ?$AAA@ 10022e94     libucrt:lcidtoname_downlevel.obj
 0002:00005ea0       ??_C@_1M@HOKAOIO@?$AAa?$AAf?$AA?9?$AAZ?$AAA@ 10022ea0     libucrt:lcidtoname_downlevel.obj
 0002:00005eac       ??_C@_1M@DPCLHLIE@?$AAk?$AAa?$AA?9?$AAG?$AAE@ 10022eac     libucrt:lcidtoname_downlevel.obj
 0002:00005eb8       ??_C@_1M@BLKMHJBI@?$AAf?$AAo?$AA?9?$AAF?$AAO@ 10022eb8     libucrt:lcidtoname_downlevel.obj
 0002:00005ec4       ??_C@_1M@LGGJAPPB@?$AAh?$AAi?$AA?9?$AAI?$AAN@ 10022ec4     libucrt:lcidtoname_downlevel.obj
 0002:00005ed0       ??_C@_1M@FIKPIHFE@?$AAm?$AAt?$AA?9?$AAM?$AAT@ 10022ed0     libucrt:lcidtoname_downlevel.obj
 0002:00005edc       ??_C@_1M@HEGGPBFA@?$AAs?$AAe?$AA?9?$AAN?$AAO@ 10022edc     libucrt:lcidtoname_downlevel.obj
 0002:00005ee8       ??_C@_1M@EIBJEEPA@?$AAm?$AAs?$AA?9?$AAM?$AAY@ 10022ee8     libucrt:lcidtoname_downlevel.obj
 0002:00005ef4       ??_C@_1M@FHLBGMPP@?$AAk?$AAk?$AA?9?$AAK?$AAZ@ 10022ef4     libucrt:lcidtoname_downlevel.obj
 0002:00005f00       ??_C@_1M@NGJJLCGI@?$AAk?$AAy?$AA?9?$AAK?$AAG@ 10022f00     libucrt:lcidtoname_downlevel.obj
 0002:00005f0c       ??_C@_1M@GIENNBFC@?$AAs?$AAw?$AA?9?$AAK?$AAE@ 10022f0c     libucrt:lcidtoname_downlevel.obj
 0002:00005f18       ??_C@_1BG@NDGMJIMJ@?$AAu?$AAz?$AA?9?$AAU?$AAZ?$AA?9?$AAL?$AAa?$AAt?$AAn@ 10022f18     libucrt:lcidtoname_downlevel.obj
 0002:00005f30       ??_C@_1M@IDCCIHBC@?$AAt?$AAt?$AA?9?$AAR?$AAU@ 10022f30     libucrt:lcidtoname_downlevel.obj
 0002:00005f3c       ??_C@_1M@LOICPMOJ@?$AAb?$AAn?$AA?9?$AAI?$AAN@ 10022f3c     libucrt:lcidtoname_downlevel.obj
 0002:00005f48       ??_C@_1M@KPKKNEAH@?$AAp?$AAa?$AA?9?$AAI?$AAN@ 10022f48     libucrt:lcidtoname_downlevel.obj
 0002:00005f54       ??_C@_1M@PJGPPBOG@?$AAg?$AAu?$AA?9?$AAI?$AAN@ 10022f54     libucrt:lcidtoname_downlevel.obj
 0002:00005f60       ??_C@_1M@KMKMOPHI@?$AAt?$AAa?$AA?9?$AAI?$AAN@ 10022f60     libucrt:lcidtoname_downlevel.obj
 0002:00005f6c       ??_C@_1M@KFEHEPAC@?$AAt?$AAe?$AA?9?$AAI?$AAN@ 10022f6c     libucrt:lcidtoname_downlevel.obj
 0002:00005f78       ??_C@_1M@CDCLMGHI@?$AAk?$AAn?$AA?9?$AAI?$AAN@ 10022f78     libucrt:lcidtoname_downlevel.obj
 0002:00005f84       ??_C@_1M@MIODLDKF@?$AAm?$AAl?$AA?9?$AAI?$AAN@ 10022f84     libucrt:lcidtoname_downlevel.obj
 0002:00005f90       ??_C@_1M@PBIEACPO@?$AAm?$AAr?$AA?9?$AAI?$AAN@ 10022f90     libucrt:lcidtoname_downlevel.obj
 0002:00005f9c       ??_C@_1M@NIDEAGPH@?$AAs?$AAa?$AA?9?$AAI?$AAN@ 10022f9c     libucrt:lcidtoname_downlevel.obj
 0002:00005fa8       ??_C@_1M@FHIHCBIO@?$AAm?$AAn?$AA?9?$AAM?$AAN@ 10022fa8     libucrt:lcidtoname_downlevel.obj
 0002:00005fb4       ??_C@_1M@JAIJPENP@?$AAc?$AAy?$AA?9?$AAG?$AAB@ 10022fb4     libucrt:lcidtoname_downlevel.obj
 0002:00005fc0       ??_C@_1M@PHGFBEPN@?$AAg?$AAl?$AA?9?$AAE?$AAS@ 10022fc0     libucrt:lcidtoname_downlevel.obj
 0002:00005fcc       ??_C@_1O@KPIPDNCP@?$AAk?$AAo?$AAk?$AA?9?$AAI?$AAN@ 10022fcc     libucrt:lcidtoname_downlevel.obj
 0002:00005fdc       ??_C@_1O@KNHJLDJA@?$AAs?$AAy?$AAr?$AA?9?$AAS?$AAY@ 10022fdc     libucrt:lcidtoname_downlevel.obj
 0002:00005fec       ??_C@_1O@MKEKBLAH@?$AAd?$AAi?$AAv?$AA?9?$AAM?$AAV@ 10022fec     libucrt:lcidtoname_downlevel.obj
 0002:00005ffc       ??_C@_1O@OHDCKDDF@?$AAq?$AAu?$AAz?$AA?9?$AAB?$AAO@ 10022ffc     libucrt:lcidtoname_downlevel.obj
 0002:0000600c       ??_C@_1M@LEPJNLFD@?$AAn?$AAs?$AA?9?$AAZ?$AAA@ 1002300c     libucrt:lcidtoname_downlevel.obj
 0002:00006018       ??_C@_1M@OMLEIIJB@?$AAm?$AAi?$AA?9?$AAN?$AAZ@ 10023018     libucrt:lcidtoname_downlevel.obj
 0002:00006024       ??_C@_1M@PMPEAILG@?$AAa?$AAr?$AA?9?$AAI?$AAQ@ 10023024     libucrt:lcidtoname_downlevel.obj
 0002:00006030       ??_C@_1M@CNKPNOEE@?$AAd?$AAe?$AA?9?$AAC?$AAH@ 10023030     libucrt:lcidtoname_downlevel.obj
 0002:0000603c       ??_C@_1M@LKMGMLKO@?$AAe?$AAn?$AA?9?$AAG?$AAB@ 1002303c     libucrt:lcidtoname_downlevel.obj
 0002:00006048       ??_C@_1M@PGKJFFGL@?$AAe?$AAs?$AA?9?$AAM?$AAX@ 10023048     libucrt:lcidtoname_downlevel.obj
 0002:00006054       ??_C@_1M@DNNANBDC@?$AAf?$AAr?$AA?9?$AAB?$AAE@ 10023054     libucrt:lcidtoname_downlevel.obj
 0002:00006060       ??_C@_1M@HLGMDFHM@?$AAi?$AAt?$AA?9?$AAC?$AAH@ 10023060     libucrt:lcidtoname_downlevel.obj
 0002:0000606c       ??_C@_1M@CLLBGJH@?$AAn?$AAl?$AA?9?$AAB?$AAE@ 1002306c     libucrt:lcidtoname_downlevel.obj
 0002:00006078       ??_C@_1M@BODBOGLF@?$AAn?$AAn?$AA?9?$AAN?$AAO@ 10023078     libucrt:lcidtoname_downlevel.obj
 0002:00006084       ??_C@_1M@HFFAHKAD@?$AAp?$AAt?$AA?9?$AAP?$AAT@ 10023084     libucrt:lcidtoname_downlevel.obj
 0002:00006090       ??_C@_1BG@LNOAKHIE@?$AAs?$AAr?$AA?9?$AAS?$AAP?$AA?9?$AAL?$AAa?$AAt?$AAn@ 10023090     libucrt:lcidtoname_downlevel.obj
 0002:000060a8       ??_C@_1M@HBMHBGAK@?$AAs?$AAv?$AA?9?$AAF?$AAI@ 100230a8     libucrt:lcidtoname_downlevel.obj
 0002:000060b4       ??_C@_1BG@DGCJGJBE@?$AAa?$AAz?$AA?9?$AAA?$AAZ?$AA?9?$AAC?$AAy?$AAr?$AAl@ 100230b4     libucrt:lcidtoname_downlevel.obj
 0002:000060cc       ??_C@_1M@KEJDAAHB@?$AAs?$AAe?$AA?9?$AAS?$AAE@ 100230cc     libucrt:lcidtoname_downlevel.obj
 0002:000060d8       ??_C@_1M@HEIBJJAD@?$AAm?$AAs?$AA?9?$AAB?$AAN@ 100230d8     libucrt:lcidtoname_downlevel.obj
 0002:000060e4       ??_C@_1BG@PBGJMCEM@?$AAu?$AAz?$AA?9?$AAU?$AAZ?$AA?9?$AAC?$AAy?$AAr?$AAl@ 100230e4     libucrt:lcidtoname_downlevel.obj
 0002:000060fc       ??_C@_1O@LAOBCMDF@?$AAq?$AAu?$AAz?$AA?9?$AAE?$AAC@ 100230fc     libucrt:lcidtoname_downlevel.obj
 0002:0000610c       ??_C@_1M@POEEMAIO@?$AAa?$AAr?$AA?9?$AAE?$AAG@ 1002310c     libucrt:lcidtoname_downlevel.obj
 0002:00006118       ??_C@_1M@EFAKDEDL@?$AAz?$AAh?$AA?9?$AAH?$AAK@ 10023118     libucrt:lcidtoname_downlevel.obj
 0002:00006124       ??_C@_1M@HKKIJHGI@?$AAd?$AAe?$AA?9?$AAA?$AAT@ 10023124     libucrt:lcidtoname_downlevel.obj
 0002:00006130       ??_C@_1M@KBFBEHJF@?$AAe?$AAn?$AA?9?$AAA?$AAU@ 10023130     libucrt:lcidtoname_downlevel.obj
 0002:0000613c       ??_C@_1M@MNPLFAAH@?$AAe?$AAs?$AA?9?$AAE?$AAS@ 1002313c     libucrt:lcidtoname_downlevel.obj
 0002:00006148       ??_C@_1M@HJOOJFMA@?$AAf?$AAr?$AA?9?$AAC?$AAA@ 10023148     libucrt:lcidtoname_downlevel.obj
 0002:00006154       ??_C@_1BG@JPOFPNAB@?$AAs?$AAr?$AA?9?$AAS?$AAP?$AA?9?$AAC?$AAy?$AAr?$AAl@ 10023154     libucrt:lcidtoname_downlevel.obj
 0002:0000616c       ??_C@_1M@LNFOCMOB@?$AAs?$AAe?$AA?9?$AAF?$AAI@ 1002316c     libucrt:lcidtoname_downlevel.obj
 0002:00006178       ??_C@_1O@MGJBOAMB@?$AAq?$AAu?$AAz?$AA?9?$AAP?$AAE@ 10023178     libucrt:lcidtoname_downlevel.obj
 0002:00006188       ??_C@_1M@GJINLBOK@?$AAa?$AAr?$AA?9?$AAL?$AAY@ 10023188     libucrt:lcidtoname_downlevel.obj
 0002:00006194       ??_C@_1M@GGMNHJNL@?$AAz?$AAh?$AA?9?$AAS?$AAG@ 10023194     libucrt:lcidtoname_downlevel.obj
 0002:000061a0       ??_C@_1M@HOIKODND@?$AAd?$AAe?$AA?9?$AAL?$AAU@ 100231a0     libucrt:lcidtoname_downlevel.obj
 0002:000061ac       ??_C@_1M@DDOCCGFG@?$AAe?$AAn?$AA?9?$AAC?$AAA@ 100231ac     libucrt:lcidtoname_downlevel.obj
 0002:000061b8       ??_C@_1M@BNOEMJLF@?$AAe?$AAs?$AA?9?$AAG?$AAT@ 100231b8     libucrt:lcidtoname_downlevel.obj
 0002:000061c4       ??_C@_1M@EOGNKEK@?$AAf?$AAr?$AA?9?$AAC?$AAH@ 100231c4     libucrt:lcidtoname_downlevel.obj
 0002:000061d0       ??_C@_1M@FLIDJFHL@?$AAh?$AAr?$AA?9?$AAB?$AAA@ 100231d0     libucrt:lcidtoname_downlevel.obj
 0002:000061dc       ??_C@_1O@FMCELNAJ@?$AAs?$AAm?$AAj?$AA?9?$AAN?$AAO@ 100231dc     libucrt:lcidtoname_downlevel.obj
 0002:000061ec       ??_C@_1M@JHGLJMGJ@?$AAa?$AAr?$AA?9?$AAD?$AAZ@ 100231ec     libucrt:lcidtoname_downlevel.obj
 0002:000061f8       ??_C@_1M@JKKFDCNP@?$AAz?$AAh?$AA?9?$AAM?$AAO@ 100231f8     libucrt:lcidtoname_downlevel.obj
 0002:00006204       ??_C@_1M@GEEFALPE@?$AAd?$AAe?$AA?9?$AAL?$AAI@ 10023204     libucrt:lcidtoname_downlevel.obj
 0002:00006210       ??_C@_1M@IGEOFBG@?$AAe?$AAn?$AA?9?$AAN?$AAZ@ 10023210     libucrt:lcidtoname_downlevel.obj
 0002:0000621c       ??_C@_1M@KDBONEHP@?$AAe?$AAs?$AA?9?$AAC?$AAR@ 1002321c     libucrt:lcidtoname_downlevel.obj
 0002:00006228       ??_C@_1M@FHMDOHNN@?$AAf?$AAr?$AA?9?$AAL?$AAU@ 10023228     libucrt:lcidtoname_downlevel.obj
 0002:00006234       ??_C@_1BG@NFKKMAFG@?$AAb?$AAs?$AA?9?$AAB?$AAA?$AA?9?$AAL?$AAa?$AAt?$AAn@ 10023234     libucrt:lcidtoname_downlevel.obj
 0002:0000624c       ??_C@_1O@IMNBEMCI@?$AAs?$AAm?$AAj?$AA?9?$AAS?$AAE@ 1002324c     libucrt:lcidtoname_downlevel.obj
 0002:0000625c       ??_C@_1M@DHHMBNDP@?$AAa?$AAr?$AA?9?$AAM?$AAA@ 1002325c     libucrt:lcidtoname_downlevel.obj
 0002:00006268       ??_C@_1M@BNBLJCGH@?$AAe?$AAn?$AA?9?$AAI?$AAE@ 10023268     libucrt:lcidtoname_downlevel.obj
 0002:00006274       ??_C@_1M@GEPAFMDL@?$AAe?$AAs?$AA?9?$AAP?$AAA@ 10023274     libucrt:lcidtoname_downlevel.obj
 0002:00006280       ??_C@_1M@OJONDMDL@?$AAf?$AAr?$AA?9?$AAM?$AAC@ 10023280     libucrt:lcidtoname_downlevel.obj
 0002:0000628c       ??_C@_1BG@OBCNFJB@?$AAs?$AAr?$AA?9?$AAB?$AAA?$AA?9?$AAL?$AAa?$AAt?$AAn@ 1002328c     libucrt:lcidtoname_downlevel.obj
 0002:000062a4       ??_C@_1O@KEMEEGPO@?$AAs?$AAm?$AAa?$AA?9?$AAN?$AAO@ 100232a4     libucrt:lcidtoname_downlevel.obj
 0002:000062b4       ??_C@_1M@ELMGFODK@?$AAa?$AAr?$AA?9?$AAT?$AAN@ 100232b4     libucrt:lcidtoname_downlevel.obj
 0002:000062c0       ??_C@_1M@BHDLHFAF@?$AAe?$AAn?$AA?9?$AAZ?$AAA@ 100232c0     libucrt:lcidtoname_downlevel.obj
 0002:000062cc       ??_C@_1M@BMGIGLIF@?$AAe?$AAs?$AA?9?$AAD?$AAO@ 100232cc     libucrt:lcidtoname_downlevel.obj
 0002:000062d8       ??_C@_1BG@CMBHIPBE@?$AAs?$AAr?$AA?9?$AAB?$AAA?$AA?9?$AAC?$AAy?$AAr?$AAl@ 100232d8     libucrt:lcidtoname_downlevel.obj
 0002:000062f0       ??_C@_1O@HEDBLHNP@?$AAs?$AAm?$AAa?$AA?9?$AAS?$AAE@ 100232f0     libucrt:lcidtoname_downlevel.obj
 0002:00006300       ??_C@_1M@DAGCADIM@?$AAa?$AAr?$AA?9?$AAO?$AAM@ 10023300     libucrt:lcidtoname_downlevel.obj
 0002:0000630c       ??_C@_1M@FODLMICG@?$AAe?$AAn?$AA?9?$AAJ?$AAM@ 1002330c     libucrt:lcidtoname_downlevel.obj
 0002:00006318       ??_C@_1M@DNMLCIHB@?$AAe?$AAs?$AA?9?$AAV?$AAE@ 10023318     libucrt:lcidtoname_downlevel.obj
 0002:00006324       ??_C@_1O@EOKHMKJK@?$AAs?$AAm?$AAs?$AA?9?$AAF?$AAI@ 10023324     libucrt:lcidtoname_downlevel.obj
 0002:00006334       ??_C@_1M@CAFJMKOF@?$AAa?$AAr?$AA?9?$AAY?$AAE@ 10023334     libucrt:lcidtoname_downlevel.obj
 0002:00006340       ??_C@_1M@CBFHIJLI@?$AAe?$AAn?$AA?9?$AAC?$AAB@ 10023340     libucrt:lcidtoname_downlevel.obj
 0002:0000634c       ??_C@_1M@BGNFLDN@?$AAe?$AAs?$AA?9?$AAC?$AAO@ 1002334c     libucrt:lcidtoname_downlevel.obj
 0002:00006358       ??_C@_1O@JMPHMAMC@?$AAs?$AAm?$AAn?$AA?9?$AAF?$AAI@ 10023358     libucrt:lcidtoname_downlevel.obj
 0002:00006368       ??_C@_1M@JLANABKE@?$AAa?$AAr?$AA?9?$AAS?$AAY@ 10023368     libucrt:lcidtoname_downlevel.obj
 0002:00006374       ??_C@_1M@HPKGCFGN@?$AAe?$AAn?$AA?9?$AAB?$AAZ@ 10023374     libucrt:lcidtoname_downlevel.obj
 0002:00006380       ??_C@_1M@OLJCMLGM@?$AAe?$AAs?$AA?9?$AAP?$AAE@ 10023380     libucrt:lcidtoname_downlevel.obj
 0002:0000638c       ??_C@_1M@MKKGFKLE@?$AAa?$AAr?$AA?9?$AAJ?$AAO@ 1002338c     libucrt:lcidtoname_downlevel.obj
 0002:00006398       ??_C@_1M@EKPGLDNI@?$AAe?$AAn?$AA?9?$AAT?$AAT@ 10023398     libucrt:lcidtoname_downlevel.obj
 0002:000063a4       ??_C@_1M@OONGHFHE@?$AAe?$AAs?$AA?9?$AAA?$AAR@ 100233a4     libucrt:lcidtoname_downlevel.obj
 0002:000063b0       ??_C@_1M@OOJFGBHE@?$AAa?$AAr?$AA?9?$AAL?$AAB@ 100233b0     libucrt:lcidtoname_downlevel.obj
 0002:000063bc       ??_C@_1M@GCEJHNEG@?$AAe?$AAn?$AA?9?$AAZ?$AAW@ 100233bc     libucrt:lcidtoname_downlevel.obj
 0002:000063c8       ??_C@_1M@JNOCAHJI@?$AAe?$AAs?$AA?9?$AAE?$AAC@ 100233c8     libucrt:lcidtoname_downlevel.obj
 0002:000063d4       ??_C@_1M@JEFHPGGB@?$AAa?$AAr?$AA?9?$AAK?$AAW@ 100233d4     libucrt:lcidtoname_downlevel.obj
 0002:000063e0       ??_C@_1M@MLKIBJOJ@?$AAe?$AAn?$AA?9?$AAP?$AAH@ 100233e0     libucrt:lcidtoname_downlevel.obj
 0002:000063ec       ??_C@_1M@BDNIPEND@?$AAe?$AAs?$AA?9?$AAC?$AAL@ 100233ec     libucrt:lcidtoname_downlevel.obj
 0002:000063f8       ??_C@_1M@MPNMEKBD@?$AAa?$AAr?$AA?9?$AAA?$AAE@ 100233f8     libucrt:lcidtoname_downlevel.obj
 0002:00006404       ??_C@_1M@KBJALCPI@?$AAe?$AAs?$AA?9?$AAU?$AAY@ 10023404     libucrt:lcidtoname_downlevel.obj
 0002:00006410       ??_C@_1M@LLCCOAGA@?$AAa?$AAr?$AA?9?$AAB?$AAH@ 10023410     libucrt:lcidtoname_downlevel.obj
 0002:0000641c       ??_C@_1M@PBFNCDEL@?$AAe?$AAs?$AA?9?$AAP?$AAY@ 1002341c     libucrt:lcidtoname_downlevel.obj
 0002:00006428       ??_C@_1M@EDGINPNP@?$AAa?$AAr?$AA?9?$AAQ?$AAA@ 10023428     libucrt:lcidtoname_downlevel.obj
 0002:00006434       ??_C@_1M@MKDBIIJI@?$AAe?$AAs?$AA?9?$AAB?$AAO@ 10023434     libucrt:lcidtoname_downlevel.obj
 0002:00006440       ??_C@_1M@CPKKEBLD@?$AAe?$AAs?$AA?9?$AAS?$AAV@ 10023440     libucrt:lcidtoname_downlevel.obj
 0002:0000644c       ??_C@_1M@NDBGMMJL@?$AAe?$AAs?$AA?9?$AAH?$AAN@ 1002344c     libucrt:lcidtoname_downlevel.obj
 0002:00006458       ??_C@_1M@JIJIBHDP@?$AAe?$AAs?$AA?9?$AAN?$AAI@ 10023458     libucrt:lcidtoname_downlevel.obj
 0002:00006464       ??_C@_1M@CGFMKEEK@?$AAe?$AAs?$AA?9?$AAP?$AAR@ 10023464     libucrt:lcidtoname_downlevel.obj
 0002:00006470       ??_C@_1O@ICJHKIIK@?$AAz?$AAh?$AA?9?$AAC?$AAH?$AAT@ 10023470     libucrt:lcidtoname_downlevel.obj
 0002:00006480       ??_C@_15CLNEJCE@?$AAs?$AAr@ 10023480     libucrt:lcidtoname_downlevel.obj
 0002:00006ba8       ??_C@_1M@KAHEKEIG@?$AAa?$AAf?$AA?9?$AAz?$AAa@ 10023ba8     libucrt:lcidtoname_downlevel.obj
 0002:00006bb4       ??_C@_1M@GIECOABL@?$AAa?$AAr?$AA?9?$AAa?$AAe@ 10023bb4     libucrt:lcidtoname_downlevel.obj
 0002:00006bc0       ??_C@_1M@BMLMEKGI@?$AAa?$AAr?$AA?9?$AAb?$AAh@ 10023bc0     libucrt:lcidtoname_downlevel.obj
 0002:00006bcc       ??_C@_1M@DAPFDGGB@?$AAa?$AAr?$AA?9?$AAd?$AAz@ 10023bcc     libucrt:lcidtoname_downlevel.obj
 0002:00006bd8       ??_C@_1M@FJNKGKIG@?$AAa?$AAr?$AA?9?$AAe?$AAg@ 10023bd8     libucrt:lcidtoname_downlevel.obj
 0002:00006be4       ??_C@_1M@FLGKKCLO@?$AAa?$AAr?$AA?9?$AAi?$AAq@ 10023be4     libucrt:lcidtoname_downlevel.obj
 0002:00006bf0       ??_C@_1M@GNDIPALM@?$AAa?$AAr?$AA?9?$AAj?$AAo@ 10023bf0     libucrt:lcidtoname_downlevel.obj
 0002:00006bfc       ??_C@_1M@DDMJFMGJ@?$AAa?$AAr?$AA?9?$AAk?$AAw@ 10023bfc     libucrt:lcidtoname_downlevel.obj
 0002:00006c08       ??_C@_1M@EJALMLHM@?$AAa?$AAr?$AA?9?$AAl?$AAb@ 10023c08     libucrt:lcidtoname_downlevel.obj
 0002:00006c14       ??_C@_1M@MOBDBLOC@?$AAa?$AAr?$AA?9?$AAl?$AAy@ 10023c14     libucrt:lcidtoname_downlevel.obj
 0002:00006c20       ??_C@_1M@JAOCLHDH@?$AAa?$AAr?$AA?9?$AAm?$AAa@ 10023c20     libucrt:lcidtoname_downlevel.obj
 0002:00006c2c       ??_C@_1M@JHPMKJIE@?$AAa?$AAr?$AA?9?$AAo?$AAm@ 10023c2c     libucrt:lcidtoname_downlevel.obj
 0002:00006c38       ??_C@_1M@OEPGHFNH@?$AAa?$AAr?$AA?9?$AAq?$AAa@ 10023c38     libucrt:lcidtoname_downlevel.obj
 0002:00006c44       ??_C@_1M@KJDONENM@?$AAa?$AAr?$AA?9?$AAs?$AAa@ 10023c44     libucrt:lcidtoname_downlevel.obj
 0002:00006c50       ??_C@_1M@DMJDKLKM@?$AAa?$AAr?$AA?9?$AAs?$AAy@ 10023c50     libucrt:lcidtoname_downlevel.obj
 0002:00006c5c       ??_C@_1M@OMFIPEDC@?$AAa?$AAr?$AA?9?$AAt?$AAn@ 10023c5c     libucrt:lcidtoname_downlevel.obj
 0002:00006c68       ??_C@_1M@IHMHGAON@?$AAa?$AAr?$AA?9?$AAy?$AAe@ 10023c68     libucrt:lcidtoname_downlevel.obj
 0002:00006c74       ??_C@_1BG@KDCPGJGB@?$AAa?$AAz?$AA?9?$AAa?$AAz?$AA?9?$AAc?$AAy?$AAr?$AAl@ 10023c74     libucrt:lcidtoname_downlevel.obj
 0002:00006c8c       ??_C@_1BG@IBCKDDOE@?$AAa?$AAz?$AA?9?$AAa?$AAz?$AA?9?$AAl?$AAa?$AAt?$AAn@ 10023c8c     libucrt:lcidtoname_downlevel.obj
 0002:00006ca4       ??_C@_1M@EGPFDCPD@?$AAb?$AAe?$AA?9?$AAb?$AAy@ 10023ca4     libucrt:lcidtoname_downlevel.obj
 0002:00006cb0       ??_C@_1M@PCMGMCGC@?$AAb?$AAg?$AA?9?$AAb?$AAg@ 10023cb0     libucrt:lcidtoname_downlevel.obj
 0002:00006cbc       ??_C@_1M@BJBMFGOB@?$AAb?$AAn?$AA?9?$AAi?$AAn@ 10023cbc     libucrt:lcidtoname_downlevel.obj
 0002:00006cc8       ??_C@_1BG@EAKMMACD@?$AAb?$AAs?$AA?9?$AAb?$AAa?$AA?9?$AAl?$AAa?$AAt?$AAn@ 10023cc8     libucrt:lcidtoname_downlevel.obj
 0002:00006ce0       ??_C@_1M@KGADAODK@?$AAc?$AAa?$AA?9?$AAe?$AAs@ 10023ce0     libucrt:lcidtoname_downlevel.obj
 0002:00006cec       ??_C@_1M@COAJPDHI@?$AAc?$AAs?$AA?9?$AAc?$AAz@ 10023cec     libucrt:lcidtoname_downlevel.obj
 0002:00006cf8       ??_C@_1M@DHBHFONH@?$AAc?$AAy?$AA?9?$AAg?$AAb@ 10023cf8     libucrt:lcidtoname_downlevel.obj
 0002:00006d04       ??_C@_1M@IMGKELGA@?$AAd?$AAa?$AA?9?$AAd?$AAk@ 10023d04     libucrt:lcidtoname_downlevel.obj
 0002:00006d10       ??_C@_1M@NNDGDNGA@?$AAd?$AAe?$AA?9?$AAa?$AAt@ 10023d10     libucrt:lcidtoname_downlevel.obj
 0002:00006d1c       ??_C@_1M@IKDBHEEM@?$AAd?$AAe?$AA?9?$AAc?$AAh@ 10023d1c     libucrt:lcidtoname_downlevel.obj
 0002:00006d28       ??_C@_1M@GFFOJMCJ@?$AAd?$AAe?$AA?9?$AAd?$AAe@ 10023d28     libucrt:lcidtoname_downlevel.obj
 0002:00006d34       ??_C@_1M@MDNLKBPM@?$AAd?$AAe?$AA?9?$AAl?$AAi@ 10023d34     libucrt:lcidtoname_downlevel.obj
 0002:00006d40       ??_C@_1M@NJBEEJNL@?$AAd?$AAe?$AA?9?$AAl?$AAu@ 10023d40     libucrt:lcidtoname_downlevel.obj
 0002:00006d4c       ??_C@_1O@GNNELBAP@?$AAd?$AAi?$AAv?$AA?9?$AAm?$AAv@ 10023d4c     libucrt:lcidtoname_downlevel.obj
 0002:00006d5c       ??_C@_1M@EJLEOGAE@?$AAe?$AAl?$AA?9?$AAg?$AAr@ 10023d5c     libucrt:lcidtoname_downlevel.obj
 0002:00006d68       ??_C@_1M@GMPONJN@?$AAe?$AAn?$AA?9?$AAa?$AAu@ 10023d68     libucrt:lcidtoname_downlevel.obj
 0002:00006d74       ??_C@_1M@NIDIIPGF@?$AAe?$AAn?$AA?9?$AAb?$AAz@ 10023d74     libucrt:lcidtoname_downlevel.obj
 0002:00006d80       ??_C@_1M@JEHMIMFO@?$AAe?$AAn?$AA?9?$AAc?$AAa@ 10023d80     libucrt:lcidtoname_downlevel.obj
 0002:00006d8c       ??_C@_1M@IGMJCDLA@?$AAe?$AAn?$AA?9?$AAc?$AAb@ 10023d8c     libucrt:lcidtoname_downlevel.obj
 0002:00006d98       ??_C@_1M@BNFIGBKG@?$AAe?$AAn?$AA?9?$AAg?$AAb@ 10023d98     libucrt:lcidtoname_downlevel.obj
 0002:00006da4       ??_C@_1M@LKIFDIGP@?$AAe?$AAn?$AA?9?$AAi?$AAe@ 10023da4     libucrt:lcidtoname_downlevel.obj
 0002:00006db0       ??_C@_1M@PJKFGCCO@?$AAe?$AAn?$AA?9?$AAj?$AAm@ 10023db0     libucrt:lcidtoname_downlevel.obj
 0002:00006dbc       ??_C@_1M@KPPKEPBO@?$AAe?$AAn?$AA?9?$AAn?$AAz@ 10023dbc     libucrt:lcidtoname_downlevel.obj
 0002:00006dc8       ??_C@_1M@GMDGLDOB@?$AAe?$AAn?$AA?9?$AAp?$AAh@ 10023dc8     libucrt:lcidtoname_downlevel.obj
 0002:00006dd4       ??_C@_1M@ONGIBJNA@?$AAe?$AAn?$AA?9?$AAt?$AAt@ 10023dd4     libucrt:lcidtoname_downlevel.obj
 0002:00006de0       ??_C@_1M@LLODPCMM@?$AAe?$AAn?$AA?9?$AAu?$AAs@ 10023de0     libucrt:lcidtoname_downlevel.obj
 0002:00006dec       ??_C@_1M@LAKFNPAN@?$AAe?$AAn?$AA?9?$AAz?$AAa@ 10023dec     libucrt:lcidtoname_downlevel.obj
 0002:00006df8       ??_C@_1M@MFNHNHEO@?$AAe?$AAn?$AA?9?$AAz?$AAw@ 10023df8     libucrt:lcidtoname_downlevel.obj
 0002:00006e04       ??_C@_1M@EJEINPHM@?$AAe?$AAs?$AA?9?$AAa?$AAr@ 10023e04     libucrt:lcidtoname_downlevel.obj
 0002:00006e10       ??_C@_1M@GNKPCCJA@?$AAe?$AAs?$AA?9?$AAb?$AAo@ 10023e10     libucrt:lcidtoname_downlevel.obj
 0002:00006e1c       ??_C@_1M@LEEGFONL@?$AAe?$AAs?$AA?9?$AAc?$AAl@ 10023e1c     libucrt:lcidtoname_downlevel.obj
 0002:00006e28       ??_C@_1M@KGPDPBDF@?$AAe?$AAs?$AA?9?$AAc?$AAo@ 10023e28     libucrt:lcidtoname_downlevel.obj
 0002:00006e34       ??_C@_1M@EIAHOHH@?$AAe?$AAs?$AA?9?$AAc?$AAr@ 10023e34     libucrt:lcidtoname_downlevel.obj
 0002:00006e40       ??_C@_1M@LLPGMBIN@?$AAe?$AAs?$AA?9?$AAd?$AAo@ 10023e40     libucrt:lcidtoname_downlevel.obj
 0002:00006e4c       ??_C@_1M@DKHMKNJA@?$AAe?$AAs?$AA?9?$AAe?$AAc@ 10023e4c     libucrt:lcidtoname_downlevel.obj
 0002:00006e58       ??_C@_1M@GKGFPKAP@?$AAe?$AAs?$AA?9?$AAe?$AAs@ 10023e58     libucrt:lcidtoname_downlevel.obj
 0002:00006e64       ??_C@_1M@LKHKGDLN@?$AAe?$AAs?$AA?9?$AAg?$AAt@ 10023e64     libucrt:lcidtoname_downlevel.obj
 0002:00006e70       ??_C@_1M@HEIIGGJD@?$AAe?$AAs?$AA?9?$AAh?$AAn@ 10023e70     libucrt:lcidtoname_downlevel.obj
 0002:00006e7c       ??_C@_1M@FBDHPPGD@?$AAe?$AAs?$AA?9?$AAm?$AAx@ 10023e7c     libucrt:lcidtoname_downlevel.obj
 0002:00006e88       ??_C@_1M@DPAGLNDH@?$AAe?$AAs?$AA?9?$AAn?$AAi@ 10023e88     libucrt:lcidtoname_downlevel.obj
 0002:00006e94       ??_C@_1M@MDGOPGDD@?$AAe?$AAs?$AA?9?$AAp?$AAa@ 10023e94     libucrt:lcidtoname_downlevel.obj
 0002:00006ea0       ??_C@_1M@EMAMGBGE@?$AAe?$AAs?$AA?9?$AAp?$AAe@ 10023ea0     libucrt:lcidtoname_downlevel.obj
 0002:00006eac       ??_C@_1M@IBMCAOEC@?$AAe?$AAs?$AA?9?$AAp?$AAr@ 10023eac     libucrt:lcidtoname_downlevel.obj
 0002:00006eb8       ??_C@_1M@FGMDIJED@?$AAe?$AAs?$AA?9?$AAp?$AAy@ 10023eb8     libucrt:lcidtoname_downlevel.obj
 0002:00006ec4       ??_C@_1M@IIDEOLLL@?$AAe?$AAs?$AA?9?$AAs?$AAv@ 10023ec4     libucrt:lcidtoname_downlevel.obj
 0002:00006ed0       ??_C@_1M@GAOBIPA@?$AAe?$AAs?$AA?9?$AAu?$AAy@ 10023ed0     libucrt:lcidtoname_downlevel.obj
 0002:00006edc       ??_C@_1M@JKFFICHJ@?$AAe?$AAs?$AA?9?$AAv?$AAe@ 10023edc     libucrt:lcidtoname_downlevel.obj
 0002:00006ee8       ??_C@_1M@PNMLOJDF@?$AAe?$AAt?$AA?9?$AAe?$AAe@ 10023ee8     libucrt:lcidtoname_downlevel.obj
 0002:00006ef4       ??_C@_1M@GHHLIKEI@?$AAe?$AAu?$AA?9?$AAe?$AAs@ 10023ef4     libucrt:lcidtoname_downlevel.obj
 0002:00006f00       ??_C@_1M@PBNONODE@?$AAf?$AAa?$AA?9?$AAi?$AAr@ 10023f00     libucrt:lcidtoname_downlevel.obj
 0002:00006f0c       ??_C@_1M@JEEHPMIL@?$AAf?$AAi?$AA?9?$AAf?$AAi@ 10023f0c     libucrt:lcidtoname_downlevel.obj
 0002:00006f18       ??_C@_1M@LMDCNDBA@?$AAf?$AAo?$AA?9?$AAf?$AAo@ 10023f18     libucrt:lcidtoname_downlevel.obj
 0002:00006f24       ??_C@_1M@JKEOHLDK@?$AAf?$AAr?$AA?9?$AAb?$AAe@ 10023f24     libucrt:lcidtoname_downlevel.obj
 0002:00006f30       ??_C@_1M@NOHADPMI@?$AAf?$AAr?$AA?9?$AAc?$AAa@ 10023f30     libucrt:lcidtoname_downlevel.obj
 0002:00006f3c       ??_C@_1M@KDHIHAEC@?$AAf?$AAr?$AA?9?$AAc?$AAh@ 10023f3c     libucrt:lcidtoname_downlevel.obj
 0002:00006f48       ??_C@_1M@MMBBFGAK@?$AAf?$AAr?$AA?9?$AAf?$AAr@ 10023f48     libucrt:lcidtoname_downlevel.obj
 0002:00006f54       ??_C@_1M@PAFNENNF@?$AAf?$AAr?$AA?9?$AAl?$AAu@ 10023f54     libucrt:lcidtoname_downlevel.obj
 0002:00006f60       ??_C@_1M@EOHDJGDD@?$AAf?$AAr?$AA?9?$AAm?$AAc@ 10023f60     libucrt:lcidtoname_downlevel.obj
 0002:00006f6c       ??_C@_1M@FAPLLOPF@?$AAg?$AAl?$AA?9?$AAe?$AAs@ 10023f6c     libucrt:lcidtoname_downlevel.obj
 0002:00006f78       ??_C@_1M@FOPBFLOO@?$AAg?$AAu?$AA?9?$AAi?$AAn@ 10023f78     libucrt:lcidtoname_downlevel.obj
 0002:00006f84       ??_C@_1M@KBMCINPM@?$AAh?$AAe?$AA?9?$AAi?$AAl@ 10023f84     libucrt:lcidtoname_downlevel.obj
 0002:00006f90       ??_C@_1M@BBPHKFPJ@?$AAh?$AAi?$AA?9?$AAi?$AAn@ 10023f90     libucrt:lcidtoname_downlevel.obj
 0002:00006f9c       ??_C@_1M@PMBNDPHD@?$AAh?$AAr?$AA?9?$AAb?$AAa@ 10023f9c     libucrt:lcidtoname_downlevel.obj
 0002:00006fa8       ??_C@_1M@BPCKOEGE@?$AAh?$AAr?$AA?9?$AAh?$AAr@ 10023fa8     libucrt:lcidtoname_downlevel.obj
 0002:00006fb4       ??_C@_1M@GACBMHKE@?$AAh?$AAu?$AA?9?$AAh?$AAu@ 10023fb4     libucrt:lcidtoname_downlevel.obj
 0002:00006fc0       ??_C@_1M@MILPAJJC@?$AAh?$AAy?$AA?9?$AAa?$AAm@ 10023fc0     libucrt:lcidtoname_downlevel.obj
 0002:00006fcc       ??_C@_1M@BABBICEC@?$AAi?$AAd?$AA?9?$AAi?$AAd@ 10023fcc     libucrt:lcidtoname_downlevel.obj
 0002:00006fd8       ??_C@_1M@BIKNHHPF@?$AAi?$AAs?$AA?9?$AAi?$AAs@ 10023fd8     libucrt:lcidtoname_downlevel.obj
 0002:00006fe4       ??_C@_1M@NMPCJPHE@?$AAi?$AAt?$AA?9?$AAc?$AAh@ 10023fe4     libucrt:lcidtoname_downlevel.obj
 0002:00006ff0       ??_C@_1M@GHKGFEDF@?$AAi?$AAt?$AA?9?$AAi?$AAt@ 10023ff0     libucrt:lcidtoname_downlevel.obj
 0002:00006ffc       ??_C@_1M@NIEJCJJA@?$AAj?$AAa?$AA?9?$AAj?$AAp@ 10023ffc     libucrt:lcidtoname_downlevel.obj
 0002:00007008       ??_C@_1M@JILFNBIM@?$AAk?$AAa?$AA?9?$AAg?$AAe@ 10024008     libucrt:lcidtoname_downlevel.obj
 0002:00007014       ??_C@_1M@PACPMGPH@?$AAk?$AAk?$AA?9?$AAk?$AAz@ 10024014     libucrt:lcidtoname_downlevel.obj
 0002:00007020       ??_C@_1M@IELFGMHA@?$AAk?$AAn?$AA?9?$AAi?$AAn@ 10024020     libucrt:lcidtoname_downlevel.obj
 0002:0000702c       ??_C@_1O@IBBJHCH@?$AAk?$AAo?$AAk?$AA?9?$AAi?$AAn@ 1002402c     libucrt:lcidtoname_downlevel.obj
 0002:0000703c       ??_C@_1M@DMHAEOGC@?$AAk?$AAo?$AA?9?$AAk?$AAr@ 1002403c     libucrt:lcidtoname_downlevel.obj
 0002:00007048       ??_C@_1M@HBAHBIGA@?$AAk?$AAy?$AA?9?$AAk?$AAg@ 10024048     libucrt:lcidtoname_downlevel.obj
 0002:00007054       ??_C@_1M@KPMILCJG@?$AAl?$AAt?$AA?9?$AAl?$AAt@ 10024054     libucrt:lcidtoname_downlevel.obj
 0002:00007060       ??_C@_1M@BDEKKCA@?$AAl?$AAv?$AA?9?$AAl?$AAv@ 10024060     libucrt:lcidtoname_downlevel.obj
 0002:0000706c       ??_C@_1M@ELCKCCJJ@?$AAm?$AAi?$AA?9?$AAn?$AAz@ 1002406c     libucrt:lcidtoname_downlevel.obj
 0002:00007078       ??_C@_1M@CBOOLAPA@?$AAm?$AAk?$AA?9?$AAm?$AAk@ 10024078     libucrt:lcidtoname_downlevel.obj
 0002:00007084       ??_C@_1M@GPHNBJKN@?$AAm?$AAl?$AA?9?$AAi?$AAn@ 10024084     libucrt:lcidtoname_downlevel.obj
 0002:00007090       ??_C@_1M@PABJILIG@?$AAm?$AAn?$AA?9?$AAm?$AAn@ 10024090     libucrt:lcidtoname_downlevel.obj
 0002:0000709c       ??_C@_1M@FGBKKIPG@?$AAm?$AAr?$AA?9?$AAi?$AAn@ 1002409c     libucrt:lcidtoname_downlevel.obj
 0002:000070a8       ??_C@_1M@NDBPDDAL@?$AAm?$AAs?$AA?9?$AAb?$AAn@ 100240a8     libucrt:lcidtoname_downlevel.obj
 0002:000070b4       ??_C@_1M@OPIHOOPI@?$AAm?$AAs?$AA?9?$AAm?$AAy@ 100240b4     libucrt:lcidtoname_downlevel.obj
 0002:000070c0       ??_C@_1M@PPDBCNFM@?$AAm?$AAt?$AA?9?$AAm?$AAt@ 100240c0     libucrt:lcidtoname_downlevel.obj
 0002:000070cc       ??_C@_1M@KDJDKMDD@?$AAn?$AAb?$AA?9?$AAn?$AAo@ 100240cc     libucrt:lcidtoname_downlevel.obj
 0002:000070d8       ??_C@_1M@KFCFLMJP@?$AAn?$AAl?$AA?9?$AAb?$AAe@ 100240d8     libucrt:lcidtoname_downlevel.obj
 0002:000070e4       ??_C@_1M@KPOPDDGO@?$AAn?$AAl?$AA?9?$AAn?$AAl@ 100240e4     libucrt:lcidtoname_downlevel.obj
 0002:000070f0       ??_C@_1M@LJKPEMLN@?$AAn?$AAn?$AA?9?$AAn?$AAo@ 100240f0     libucrt:lcidtoname_downlevel.obj
 0002:000070fc       ??_C@_1M@BDGHHBFL@?$AAn?$AAs?$AA?9?$AAz?$AAa@ 100240fc     libucrt:lcidtoname_downlevel.obj
 0002:00007108       ??_C@_1M@IDEHOAP@?$AAp?$AAa?$AA?9?$AAi?$AAn@ 10024108     libucrt:lcidtoname_downlevel.obj
 0002:00007114       ??_C@_1M@HDBKGOGH@?$AAp?$AAl?$AA?9?$AAp?$AAl@ 10024114     libucrt:lcidtoname_downlevel.obj
 0002:00007120       ??_C@_1M@LJLLCMEH@?$AAp?$AAt?$AA?9?$AAb?$AAr@ 10024120     libucrt:lcidtoname_downlevel.obj
 0002:0000712c       ??_C@_1M@NCMONAAL@?$AAp?$AAt?$AA?9?$AAp?$AAt@ 1002412c     libucrt:lcidtoname_downlevel.obj
 0002:00007138       ??_C@_1O@EAKMAJDN@?$AAq?$AAu?$AAz?$AA?9?$AAb?$AAo@ 10024138     libucrt:lcidtoname_downlevel.obj
 0002:00007148       ??_C@_1O@BHHPIGDN@?$AAq?$AAu?$AAz?$AA?9?$AAe?$AAc@ 10024148     libucrt:lcidtoname_downlevel.obj
 0002:00007158       ??_C@_1O@GBAPEKMJ@?$AAq?$AAu?$AAz?$AA?9?$AAp?$AAe@ 10024158     libucrt:lcidtoname_downlevel.obj
 0002:00007168       ??_C@_1M@CLGLEFBO@?$AAr?$AAo?$AA?9?$AAr?$AAo@ 10024168     libucrt:lcidtoname_downlevel.obj
 0002:00007174       ??_C@_1M@CEEDODME@?$AAr?$AAu?$AA?9?$AAr?$AAu@ 10024174     libucrt:lcidtoname_downlevel.obj
 0002:00007180       ??_C@_1M@HPKKKMPP@?$AAs?$AAa?$AA?9?$AAi?$AAn@ 10024180     libucrt:lcidtoname_downlevel.obj
 0002:0000718c       ??_C@_1M@BKMAIGOJ@?$AAs?$AAe?$AA?9?$AAf?$AAi@ 1002418c     libucrt:lcidtoname_downlevel.obj
 0002:00007198       ??_C@_1M@NDPIFLFI@?$AAs?$AAe?$AA?9?$AAn?$AAo@ 10024198     libucrt:lcidtoname_downlevel.obj
 0002:000071a4       ??_C@_1M@DANKKHJ@?$AAs?$AAe?$AA?9?$AAs?$AAe@ 100241a4     libucrt:lcidtoname_downlevel.obj
 0002:000071b0       ??_C@_1M@PNBLONPJ@?$AAs?$AAk?$AA?9?$AAs?$AAk@ 100241b0     libucrt:lcidtoname_downlevel.obj
 0002:000071bc       ??_C@_1M@LFMODOAL@?$AAs?$AAl?$AA?9?$AAs?$AAi@ 100241bc     libucrt:lcidtoname_downlevel.obj
 0002:000071c8       ??_C@_1O@DFKOMPG@?$AAs?$AAm?$AAa?$AA?9?$AAn?$AAo@ 100241c8     libucrt:lcidtoname_downlevel.obj
 0002:000071d8       ??_C@_1O@NDKPBNNH@?$AAs?$AAm?$AAa?$AA?9?$AAs?$AAe@ 100241d8     libucrt:lcidtoname_downlevel.obj
 0002:000071e8       ??_C@_1O@PLLKBHAB@?$AAs?$AAm?$AAj?$AA?9?$AAn?$AAo@ 100241e8     libucrt:lcidtoname_downlevel.obj
 0002:000071f8       ??_C@_1O@CLEPOGCA@?$AAs?$AAm?$AAj?$AA?9?$AAs?$AAe@ 100241f8     libucrt:lcidtoname_downlevel.obj
 0002:00007208       ??_C@_1O@DLGJGKMK@?$AAs?$AAm?$AAn?$AA?9?$AAf?$AAi@ 10024208     libucrt:lcidtoname_downlevel.obj
 0002:00007218       ??_C@_1O@OJDJGAJC@?$AAs?$AAm?$AAs?$AA?9?$AAf?$AAi@ 10024218     libucrt:lcidtoname_downlevel.obj
 0002:00007228       ??_C@_1M@BOFOGHPB@?$AAs?$AAq?$AA?9?$AAa?$AAl@ 10024228     libucrt:lcidtoname_downlevel.obj
 0002:00007234       ??_C@_1BG@LJBBIPGB@?$AAs?$AAr?$AA?9?$AAb?$AAa?$AA?9?$AAc?$AAy?$AAr?$AAl@ 10024234     libucrt:lcidtoname_downlevel.obj
 0002:0000724c       ??_C@_1BG@JLBENFOE@?$AAs?$AAr?$AA?9?$AAb?$AAa?$AA?9?$AAl?$AAa?$AAt?$AAn@ 1002424c     libucrt:lcidtoname_downlevel.obj
 0002:00007264       ??_C@_1BG@KODPNHE@?$AAs?$AAr?$AA?9?$AAs?$AAp?$AA?9?$AAc?$AAy?$AAr?$AAl@ 10024264     libucrt:lcidtoname_downlevel.obj
 0002:0000727c       ??_C@_1BG@CIOGKHPB@?$AAs?$AAr?$AA?9?$AAs?$AAp?$AA?9?$AAl?$AAa?$AAt?$AAn@ 1002427c     libucrt:lcidtoname_downlevel.obj
 0002:00007294       ??_C@_1M@NGFJLMAC@?$AAs?$AAv?$AA?9?$AAf?$AAi@ 10024294     libucrt:lcidtoname_downlevel.obj
 0002:000072a0       ??_C@_1M@MPJEJAJC@?$AAs?$AAv?$AA?9?$AAs?$AAe@ 100242a0     libucrt:lcidtoname_downlevel.obj
 0002:000072ac       ??_C@_1M@MPNDHLFK@?$AAs?$AAw?$AA?9?$AAk?$AAe@ 100242ac     libucrt:lcidtoname_downlevel.obj
 0002:000072b8       ??_C@_1O@KOHBJJI@?$AAs?$AAy?$AAr?$AA?9?$AAs?$AAy@ 100242b8     libucrt:lcidtoname_downlevel.obj
 0002:000072c8       ??_C@_1M@LDCEFHA@?$AAt?$AAa?$AA?9?$AAi?$AAn@ 100242c8     libucrt:lcidtoname_downlevel.obj
 0002:000072d4       ??_C@_1M@CNJOFAK@?$AAt?$AAe?$AA?9?$AAi?$AAn@ 100242d4     libucrt:lcidtoname_downlevel.obj
 0002:000072e0       ??_C@_1M@GNAECACD@?$AAt?$AAh?$AA?9?$AAt?$AAh@ 100242e0     libucrt:lcidtoname_downlevel.obj
 0002:000072ec       ??_C@_1M@CHBIHOJO@?$AAt?$AAn?$AA?9?$AAz?$AAa@ 100242ec     libucrt:lcidtoname_downlevel.obj
 0002:000072f8       ??_C@_1M@GCCMIGPJ@?$AAt?$AAr?$AA?9?$AAt?$AAr@ 100242f8     libucrt:lcidtoname_downlevel.obj
 0002:00007304       ??_C@_1M@CELMCNBK@?$AAt?$AAt?$AA?9?$AAr?$AAu@ 10024304     libucrt:lcidtoname_downlevel.obj
 0002:00007310       ??_C@_1M@KLMCELGA@?$AAu?$AAk?$AA?9?$AAu?$AAa@ 10024310     libucrt:lcidtoname_downlevel.obj
 0002:0000731c       ??_C@_1M@EPAJJAJF@?$AAu?$AAr?$AA?9?$AAp?$AAk@ 1002431c     libucrt:lcidtoname_downlevel.obj
 0002:00007328       ??_C@_1BG@GEGPMCDJ@?$AAu?$AAz?$AA?9?$AAu?$AAz?$AA?9?$AAc?$AAy?$AAr?$AAl@ 10024328     libucrt:lcidtoname_downlevel.obj
 0002:00007340       ??_C@_1BG@EGGKJILM@?$AAu?$AAz?$AA?9?$AAu?$AAz?$AA?9?$AAl?$AAa?$AAt?$AAn@ 10024340     libucrt:lcidtoname_downlevel.obj
 0002:00007358       ??_C@_1M@GFOCLFF@?$AAv?$AAi?$AA?9?$AAv?$AAn@ 10024358     libucrt:lcidtoname_downlevel.obj
 0002:00007364       ??_C@_1M@CPAMEDFI@?$AAx?$AAh?$AA?9?$AAz?$AAa@ 10024364     libucrt:lcidtoname_downlevel.obj
 0002:00007370       ??_C@_1O@EBKIFIGN@?$AAz?$AAh?$AA?9?$AAc?$AAh?$AAs@ 10024370     libucrt:lcidtoname_downlevel.obj
 0002:00007380       ??_C@_1O@NMHPGANE@?$AAz?$AAh?$AA?9?$AAc?$AAh?$AAt@ 10024380     libucrt:lcidtoname_downlevel.obj
 0002:00007390       ??_C@_1M@LPINJOMC@?$AAz?$AAh?$AA?9?$AAc?$AAn@ 10024390     libucrt:lcidtoname_downlevel.obj
 0002:0000739c       ??_C@_1M@OCJEJODD@?$AAz?$AAh?$AA?9?$AAh?$AAk@ 1002439c     libucrt:lcidtoname_downlevel.obj
 0002:000073a8       ??_C@_1M@DNDLJINH@?$AAz?$AAh?$AA?9?$AAm?$AAo@ 100243a8     libucrt:lcidtoname_downlevel.obj
 0002:000073b4       ??_C@_1M@MBFDNDND@?$AAz?$AAh?$AA?9?$AAs?$AAg@ 100243b4     libucrt:lcidtoname_downlevel.obj
 0002:000073c0       ??_C@_1M@IMEPLEPE@?$AAz?$AAh?$AA?9?$AAt?$AAw@ 100243c0     libucrt:lcidtoname_downlevel.obj
 0002:000073cc       ??_C@_1M@BBGHNHJP@?$AAz?$AAu?$AA?9?$AAz?$AAa@ 100243cc     libucrt:lcidtoname_downlevel.obj
 0002:000073d8       ?large_power_data@?1??multiply_by_power_of_ten@__crt_strtox@@YA_NAAUbig_integer@2@I@Z@4QBIB 100243d8     libucrt:cfout.obj
 0002:00007ce0       ?large_power_indices@?1??multiply_by_power_of_ten@__crt_strtox@@YA_NAAUbig_integer@2@I@Z@4QBUunpack_index@?1??12@YA_N0I@Z@B 10024ce0     libucrt:cfout.obj
 0002:00007d78       ?small_powers_of_ten@?1??multiply_by_power_of_ten@__crt_strtox@@YA_NAAUbig_integer@2@I@Z@4QBIB 10024d78     libucrt:cfout.obj
 0002:00007d9c       ??_C@_01GBGANLPD@0@        10024d9c     libucrt:cfout.obj
 0002:00007da0       ??_C@_05DNEBIAHO@1?$CDINF@ 10024da0     libucrt:cfout.obj
 0002:00007da8       ??_C@_06IMKFLFPG@1?$CDQNAN@ 10024da8     libucrt:cfout.obj
 0002:00007db0       ??_C@_06PGGFOGJG@1?$CDSNAN@ 10024db0     libucrt:cfout.obj
 0002:00007db8       ??_C@_05PHHOCPM@1?$CDIND@  10024db8     libucrt:cfout.obj
 0002:00007e18       ??_C@_1BA@BALFACEM@?$AAC?$AAO?$AAN?$AAO?$AAU?$AAT?$AA$@ 10024e18     libucrt:initcon.obj
 0002:00007f30       __infinity                 10024f30     libucrt:87tran.obj
 0002:00007f3a       __minfinity                10024f3a     libucrt:87tran.obj
 0002:00007f44       __logemax                  10024f44     libucrt:87tran.obj
 0002:00007f6a       __OP_EXPjmptab             10024f6a     libucrt:87tran.obj
 0002:00007f90       __indefinite               10024f90     libucrt:87disp.obj
 0002:00007f9a       __piby2                    10024f9a     libucrt:87disp.obj
 0002:00007fa4       __piby4                    10024fa4     libucrt:87disp.obj
 0002:00007fd8       __DEFAULT_CW_in_mem        10024fd8     libucrt:common.obj
 0002:00007fda       __pi_by_2_to_61            10024fda     libucrt:common.obj
 0002:00008014       ??_C@_03MGHMBJCF@log@      10025014     libucrt:libm_error.obj
 0002:00008018       ??_C@_05HGHHAHAP@log10@    10025018     libucrt:libm_error.obj
 0002:00008020       ??_C@_03KHJOGHMM@exp@      10025020     libucrt:libm_error.obj
 0002:00008024       ??_C@_03JGHBODFD@pow@      10025024     libucrt:libm_error.obj
 0002:00008028       ??_C@_04FIHNOPOL@asin@     10025028     libucrt:libm_error.obj
 0002:00008030       ??_C@_04PDIFKINK@acos@     10025030     libucrt:libm_error.obj
 0002:00008038       ??_C@_04EIAKFFMI@sqrt@     10025038     libucrt:libm_error.obj
 0002:00008040       __real@3ff0000000000000    10025040     libucrt:libm_error.obj
 0002:00008060       ___acrt_log10_table_t      10025060     libucrt:log10_tables.obj
 0002:00008470       ___acrt_log10_table_cb     10025470     libucrt:log10_tables.obj
 0002:00008880       __real@3fe0000000000000    10025880     libucrt:powhlp.obj
 0002:00008970       ??_C@_04COOMCNPB@sinh@     10025970     libucrt:fpexcept.obj
 0002:00008978       ??_C@_04HPJJNFIM@cosh@     10025978     libucrt:fpexcept.obj
 0002:00008980       ??_C@_04FJHINJAO@tanh@     10025980     libucrt:fpexcept.obj
 0002:00008988       ??_C@_04MLLJIGOK@atan@     10025988     libucrt:fpexcept.obj
 0002:00008990       ??_C@_05KNGEOGJB@atan2@    10025990     libucrt:fpexcept.obj
 0002:00008998       ??_C@_03BLEJJJBH@sin@      10025998     libucrt:fpexcept.obj
 0002:0000899c       ??_C@_03LALBNOCG@cos@      1002599c     libucrt:fpexcept.obj
 0002:000089a0       ??_C@_03IIINPABG@tan@      100259a0     libucrt:fpexcept.obj
 0002:000089a4       ??_C@_04GFPJNGEK@ceil@     100259a4     libucrt:fpexcept.obj
 0002:000089ac       ??_C@_05PBJFFIGL@floor@    100259ac     libucrt:fpexcept.obj
 0002:000089b4       ??_C@_04ODHECPBC@fabs@     100259b4     libucrt:fpexcept.obj
 0002:000089bc       ??_C@_04EHEDPDJG@modf@     100259bc     libucrt:fpexcept.obj
 0002:000089c4       ??_C@_05CEJMAHNP@ldexp@    100259c4     libucrt:fpexcept.obj
 0002:000089cc       ??_C@_05KBKMEMPO@_cabs@    100259cc     libucrt:fpexcept.obj
 0002:000089d4       ??_C@_06MEIMCGCF@_hypot@   100259d4     libucrt:fpexcept.obj
 0002:000089dc       ??_C@_04KEPJIHGP@fmod@     100259dc     libucrt:fpexcept.obj
 0002:000089e4       ??_C@_05GKKHEGJL@frexp@    100259e4     libucrt:fpexcept.obj
 0002:000089ec       ??_C@_03MJLDFKDL@_y0@      100259ec     libucrt:fpexcept.obj
 0002:000089f0       ??_C@_03NAKIGLHK@_y1@      100259f0     libucrt:fpexcept.obj
 0002:000089f4       ??_C@_03ONILCKOB@_yn@      100259f4     libucrt:fpexcept.obj
 0002:000089f8       ??_C@_05JGDBENOH@_logb@    100259f8     libucrt:fpexcept.obj
 0002:00008a00       ??_C@_0L@KDOEJCKC@_nextafter@ 10025a00     libucrt:fpexcept.obj
 0002:00008a10       __d_inf                    10025a10     libucrt:util.obj
 0002:00008a18       __d_max                    10025a18     libucrt:util.obj
 0002:00008a20       __d_mzero                  10025a20     libucrt:util.obj
 0002:00008aa0       __load_config_used         10025aa0     LIBCMT:loadcfg.obj
 0002:00008b40       ??_R4exception@std@@6B@    10025b40     AccessBridgeMessageQueue.obj
 0002:00008b54       ??_R3exception@std@@8      10025b54     AccessBridgeMessageQueue.obj
 0002:00008b64       ??_R2exception@std@@8      10025b64     AccessBridgeMessageQueue.obj
 0002:00008b6c       ??_R1A@?0A@EA@exception@std@@8 10025b6c     AccessBridgeMessageQueue.obj
 0002:00008b88       ??_R4bad_alloc@std@@6B@    10025b88     AccessBridgeMessageQueue.obj
 0002:00008b9c       ??_R3bad_alloc@std@@8      10025b9c     AccessBridgeMessageQueue.obj
 0002:00008bac       ??_R2bad_alloc@std@@8      10025bac     AccessBridgeMessageQueue.obj
 0002:00008bb8       ??_R1A@?0A@EA@bad_alloc@std@@8 10025bb8     AccessBridgeMessageQueue.obj
 0002:00008bd4       ??_R4type_info@@6B@        10025bd4     LIBCMT:std_type_info_static.obj
 0002:00008be8       ??_R3type_info@@8          10025be8     LIBCMT:std_type_info_static.obj
 0002:00008bf8       ??_R2type_info@@8          10025bf8     LIBCMT:std_type_info_static.obj
 0002:00008c00       ??_R1A@?0A@EA@type_info@@8 10025c00     LIBCMT:std_type_info_static.obj
 0002:00008c1c       ??_R4bad_array_new_length@std@@6B@ 10025c1c     LIBCMT:throw_bad_alloc.obj
 0002:00008c30       ??_R3bad_array_new_length@std@@8 10025c30     LIBCMT:throw_bad_alloc.obj
 0002:00008c40       ??_R2bad_array_new_length@std@@8 10025c40     LIBCMT:throw_bad_alloc.obj
 0002:00008c50       ??_R1A@?0A@EA@bad_array_new_length@std@@8 10025c50     LIBCMT:throw_bad_alloc.obj
 0002:00008c6c       ??_R4bad_exception@std@@6B@ 10025c6c     libvcruntime:frame.obj
 0002:00008c80       ??_R3bad_exception@std@@8  10025c80     libvcruntime:frame.obj
 0002:00008c90       ??_R2bad_exception@std@@8  10025c90     libvcruntime:frame.obj
 0002:00008c9c       ??_R1A@?0A@EA@bad_exception@std@@8 10025c9c     libvcruntime:frame.obj
 0002:00008cc0       ___safe_se_handler_table   10025cc0     <linker-defined>
 0002:00008ff0       ___rtc_iaa                 10025ff0     LIBCMT:initsect.obj
 0002:00008ff4       ___rtc_izz                 10025ff4     LIBCMT:initsect.obj
 0002:00008ff8       ___rtc_taa                 10025ff8     LIBCMT:initsect.obj
 0002:00008ffc       ___rtc_tzz                 10025ffc     LIBCMT:initsect.obj
 0002:00009000       __TI2?AVbad_alloc@std@@    10026000     AccessBridgeMessageQueue.obj
 0002:00009010       __CTA2?AVbad_alloc@std@@   10026010     AccessBridgeMessageQueue.obj
 0002:0000901c       __CT??_R0?AVbad_alloc@std@@@8??0bad_alloc@std@@QAE@ABV01@@Z12 1002601c     AccessBridgeMessageQueue.obj
 0002:00009038       __CT??_R0?AVexception@std@@@8??0exception@std@@QAE@ABV01@@Z12 10026038     AccessBridgeMessageQueue.obj
 0002:000090b4       __TI3?AVbad_array_new_length@std@@ 100260b4     LIBCMT:throw_bad_alloc.obj
 0002:000090c4       __CTA3?AVbad_array_new_length@std@@ 100260c4     LIBCMT:throw_bad_alloc.obj
 0002:000090d4       __CT??_R0?AVbad_array_new_length@std@@@8??0bad_array_new_length@std@@QAE@ABV01@@Z12 100260d4     LIBCMT:throw_bad_alloc.obj
 0002:000091f4       __TI2?AVbad_exception@std@@ 100261f4     libvcruntime:frame.obj
 0002:00009204       __CTA2?AVbad_exception@std@@ 10026204     libvcruntime:frame.obj
 0002:00009210       __CT??_R0?AVbad_exception@std@@@8??0bad_exception@std@@QAE@ABV01@@Z12 10026210     libvcruntime:frame.obj
 0002:0000a564       __IMPORT_DESCRIPTOR_KERNEL32 10027564     kernel32:KERNEL32.dll
 0002:0000a578       __IMPORT_DESCRIPTOR_USER32 10027578     user32:USER32.dll
 0002:0000a58c       __NULL_IMPORT_DESCRIPTOR   1002758c     kernel32:KERNEL32.dll
 0003:00000000       ___security_cookie_complement 10028000     LIBCMT:gs_cookie.obj
 0003:00000004       ___security_cookie         10028004     LIBCMT:gs_cookie.obj
 0003:00000010       ___scrt_native_dllmain_reason 10028010     LIBCMT:utility.obj
 0003:00000020       ___isa_enabled             10028020     LIBCMT:cpu_disp.obj
 0003:00000040       __NLG_Destination          10028040     libvcruntime:exsup.obj
 0003:00000050       __iob                      10028050     libucrt:_file.obj
 0003:00000100       ___abort_behavior          10028100     libucrt:abort.obj
 0003:00000110       ___badioinfo               10028110     libucrt:ioinit.obj
 0003:00000150       ___acrt_initial_locale_data 10028150     libucrt:nlsdata.obj
 0003:00000208       ___acrt_initial_locale_pointers 10028208     libucrt:nlsdata.obj
 0003:00000210       ___acrt_wide_c_locale_string 10028210     libucrt:nlsdata.obj
 0003:00000218       ___acrt_initial_multibyte_data 10028218     libucrt:mbctype.obj
 0003:00000738       ___globallocalestatus      10028738     libucrt:glstatus.obj
 0003:00000740       ___acrt_lconv_c            10028740     libucrt:localeconv.obj
 0003:00000790       ___acrt_lconv_static_decimal 10028790     libucrt:localeconv.obj
 0003:00000794       ___acrt_lconv_static_W_decimal 10028794     libucrt:localeconv.obj
 0003:000007a0       __lookuptrailbytes         100287a0     libucrt:read.obj
 0003:000008c0       __fltused                  100288c0     LIBCMT:fltused.obj
 0003:000008d0       ??_R0?AVbad_alloc@std@@@8  100288d0     AccessBridgeMessageQueue.obj
 0003:000008ec       ??_R0?AVexception@std@@@8  100288ec     AccessBridgeMessageQueue.obj
 0003:00000908       ??_R0?AVtype_info@@@8      10028908     LIBCMT:std_type_info_static.obj
 0003:00000920       ??_R0?AVbad_array_new_length@std@@@8 10028920     LIBCMT:throw_bad_alloc.obj
 0003:00000948       ??_R0?AVbad_exception@std@@@8 10028948     libvcruntime:frame.obj
 0003:00000968       ?_OptionsStorage@?1??__local_stdio_printf_options@@9@4_KA 10028968     AccessBridgeDebug.obj
 0003:00000974       ?theFromJavaHelloMsgID@@3IA 10028974     AccessBridgeMessages.obj
 0003:00000978       ?theFromWindowsHelloMsgID@@3IA 10028978     AccessBridgeMessages.obj
 0003:0000097c       ?sendMemoryIPCLock@@3U_RTL_CRITICAL_SECTION@@A 1002897c     WinAccessBridge.obj
 0003:00000994       ?newJVMs@@3PAPADA          10028994     WinAccessBridge.obj
 0003:00000998       ?theWindowsAccessBridge@@3PAVWinAccessBridge@@A 10028998     WinAccessBridge.obj
 0003:0000099c       ?theDialogWindow@@3PAUHWND__@@A 1002899c     WinAccessBridge.obj
 0003:000009a0       ?isVMInstanceChainInUse@@3_NA 100289a0     WinAccessBridge.obj
 0003:00000cc8       ?__type_info_root_node@@3U__type_info_node@@A 10028cc8     LIBCMT:tncleanup.obj
 0003:00000cd0       ?_OptionsStorage@?1??__local_stdio_scanf_options@@9@4_KA 10028cd0     LIBCMT:default_local_stdio_options.obj
 0003:00000cd8       ___scrt_current_native_startup_state 10028cd8     LIBCMT:utility.obj
 0003:00000cdc       ___scrt_native_startup_lock 10028cdc     LIBCMT:utility.obj
 0003:00000cfc       ___scrt_debugger_hook_flag 10028cfc     LIBCMT:utility_desktop.obj
 0003:00000d00       ___isa_available           10028d00     LIBCMT:cpu_disp.obj
 0003:00000d04       ___favor                   10028d04     LIBCMT:cpu_disp.obj
 0003:00000d08       ?pArgList@UnDecorator@@0PAVReplicator@@A 10028d08     libvcruntime:undname.obj
 0003:00000d0c       ?pZNameList@UnDecorator@@0PAVReplicator@@A 10028d0c     libvcruntime:undname.obj
 0003:00000d10       ?pTemplateArgList@UnDecorator@@0PAVReplicator@@A 10028d10     libvcruntime:undname.obj
 0003:00000d14       ?gName@UnDecorator@@0PBDB  10028d14     libvcruntime:undname.obj
 0003:00000d18       ?name@UnDecorator@@0PBDB   10028d18     libvcruntime:undname.obj
 0003:00000d1c       ?disableFlags@UnDecorator@@0KA 10028d1c     libvcruntime:undname.obj
 0003:00000d20       ?fExplicitTemplateParams@UnDecorator@@0_NA 10028d20     libvcruntime:undname.obj
 0003:00000d21       ?fGetTemplateArgumentList@UnDecorator@@0_NA 10028d21     libvcruntime:undname.obj
 0003:00000d24       ?m_pGetParameter@UnDecorator@@0P6APADJ@ZA 10028d24     libvcruntime:undname.obj
 0003:00000d28       ?m_CHPENameOffset@UnDecorator@@0KA 10028d28     libvcruntime:undname.obj
 0003:00000d2c       ?m_recursionLevel@UnDecorator@@0KA 10028d2c     libvcruntime:undname.obj
 0003:00000da8       ___pPurecall               10028da8     libvcruntime:purevirt_data.obj
 0003:00000dac       ?__WinRTOutOfMemoryExceptionCallback@@3P6GPAXXZA 10028dac     libvcruntime:ehhelpers.obj
 0003:00000db0       __nstream                  10028db0     libucrt:_file.obj
 0003:00000db4       ___piob                    10028db4     libucrt:_file.obj
 0003:00000db8       __cflush                   10028db8     libucrt:_file.obj
 0003:00000ed8       __environ_table            10028ed8     libucrt:environment_initialization.obj
 0003:00000edc       __wenviron_table           10028edc     libucrt:environment_initialization.obj
 0003:00000ee0       ___dcrt_initial_wide_environment 10028ee0     libucrt:environment_initialization.obj
 0003:00000ee4       ___dcrt_initial_narrow_environment 10028ee4     libucrt:environment_initialization.obj
 0003:00000ee8       ___acrt_atexit_table       10028ee8     libucrt:onexit.obj
 0003:00000ef4       ___acrt_at_quick_exit_table 10028ef4     libucrt:onexit.obj
 0003:00000ff0       ___pioinfo                 10028ff0     libucrt:ioinit.obj
 0003:000011f0       __nhandle                  100291f0     libucrt:ioinit.obj
 0003:00001200       ___acrt_stdout_buffer      10029200     libucrt:_sftbuf.obj
 0003:00001204       ___acrt_stderr_buffer      10029204     libucrt:_sftbuf.obj
 0003:00001208       ___acrt_locale_changed_data 10029208     libucrt:wsetlocale.obj
 0003:0000120c       ___acrt_current_locale_data 1002920c     libucrt:nlsdata.obj
 0003:00001364       __mbctype                  10029364     libucrt:mbctype.obj
 0003:00001368       __mbcasemap                10029368     libucrt:mbctype.obj
 0003:0000136c       ___acrt_current_multibyte_data 1002936c     libucrt:mbctype.obj
 0003:00001378       __pgmptr                   10029378     libucrt:argv_data.obj
 0003:0000137c       ___argc                    1002937c     libucrt:argv_data.obj
 0003:00001380       ___argv                    10029380     libucrt:argv_data.obj
 0003:00001384       ___wargv                   10029384     libucrt:argv_data.obj
 0003:00001388       __acmdln                   10029388     libucrt:argv_data.obj
 0003:0000138c       __wcmdln                   1002938c     libucrt:argv_data.obj
 0003:00001390       ___acrt_heap               10029390     libucrt:heap_handle.obj
 0003:000013ac       ___acrt_lconv_static_null  100293ac     libucrt:localeconv.obj
 0003:000013b0       ___acrt_lconv_static_W_null 100293b0     libucrt:localeconv.obj
 0003:000013b4       __commode                  100293b4     libucrt:ncommode.obj
 0003:000013c4       __umaskval                 100293c4     libucrt:umask.obj
 0003:000013c8       ___fastflag                100293c8     libucrt:fp_flags.obj
 0003:000013d0       __fmode                    100293d0     libucrt:txtmode.obj
 0003:000013d4       ___scrt_ucrt_dll_is_in_use 100293d4     <common>
 0003:000013d8       ___dyn_tls_init_callback   100293d8     <common>
 0003:000013dc       __pmatherr                 100293dc     <common>
 0003:000013e0       ___use_sse2_mathfcns       100293e0     <common>

 entry point at        0001:000061ef

 Static symbols

 0000:fffd3000       .debug$S                   10000000     kernel32:KERNEL32.dll
 0000:fffd3000       .debug$S                   10000000     kernel32:KERNEL32.dll
 0000:fffd3000       .debug$S                   10000000     kernel32:KERNEL32.dll
 0000:fffd3000       .debug$S                   10000000     kernel32:KERNEL32.dll
 0000:fffd3000       .debug$S                   10000000     kernel32:KERNEL32.dll
 0000:fffd3000       .debug$S                   10000000     kernel32:KERNEL32.dll
 0000:fffd3000       .debug$S                   10000000     user32:USER32.dll
 0000:fffd3000       .debug$S                   10000000     user32:USER32.dll
 0000:fffd3000       .debug$S                   10000000     kernel32:KERNEL32.dll
 0000:fffd3000       .debug$S                   10000000     kernel32:KERNEL32.dll
 0000:fffd3000       .debug$S                   10000000     kernel32:KERNEL32.dll
 0000:fffd3000       .debug$S                   10000000     kernel32:KERNEL32.dll
 0000:fffd3000       .debug$S                   10000000     kernel32:KERNEL32.dll
 0000:fffd3000       .debug$S                   10000000     kernel32:KERNEL32.dll
 0000:fffd3000       .debug$S                   10000000     kernel32:KERNEL32.dll
 0000:fffd3000       .debug$S                   10000000     kernel32:KERNEL32.dll
 0000:fffd3000       .debug$S                   10000000     kernel32:KERNEL32.dll
 0000:fffd3000       .debug$S                   10000000     kernel32:KERNEL32.dll
 0000:fffd3000       .debug$S                   10000000     kernel32:KERNEL32.dll
 0000:fffd3000       .debug$S                   10000000     kernel32:KERNEL32.dll
 0000:fffd3000       .debug$S                   10000000     kernel32:KERNEL32.dll
 0000:fffd3000       .debug$S                   10000000     kernel32:KERNEL32.dll
 0000:fffd3000       .debug$S                   10000000     kernel32:KERNEL32.dll
 0000:fffd3000       .debug$S                   10000000     kernel32:KERNEL32.dll
 0000:fffd3000       .debug$S                   10000000     kernel32:KERNEL32.dll
 0000:fffd3000       .debug$S                   10000000     kernel32:KERNEL32.dll
 0000:fffd3000       .debug$S                   10000000     kernel32:KERNEL32.dll
 0000:fffd3000       .debug$S                   10000000     kernel32:KERNEL32.dll
 0000:fffd3000       .debug$S                   10000000     kernel32:KERNEL32.dll
 0000:fffd3000       .debug$S                   10000000     kernel32:KERNEL32.dll
 0000:fffd3000       .debug$S                   10000000     user32:USER32.dll
 0000:fffd3000       .debug$S                   10000000     user32:USER32.dll
 0000:fffd3000       .debug$S                   10000000     user32:USER32.dll
 0000:fffd3000       .debug$S                   10000000     user32:USER32.dll
 0000:fffd3000       .debug$S                   10000000     user32:USER32.dll
 0000:fffd3000       .debug$S                   10000000     kernel32:KERNEL32.dll
 0000:fffd3000       .debug$S                   10000000     kernel32:KERNEL32.dll
 0000:fffd3000       .debug$S                   10000000     kernel32:KERNEL32.dll
 0000:fffd3000       .debug$S                   10000000     kernel32:KERNEL32.dll
 0000:fffd3000       .debug$S                   10000000     kernel32:KERNEL32.dll
 0000:fffd3000       .debug$S                   10000000     kernel32:KERNEL32.dll
 0000:fffd3000       .debug$S                   10000000     kernel32:KERNEL32.dll
 0000:fffd3000       .debug$S                   10000000     kernel32:KERNEL32.dll
 0000:fffd3000       .debug$S                   10000000     kernel32:KERNEL32.dll
 0000:fffd3000       .debug$S                   10000000     kernel32:KERNEL32.dll
 0000:fffd3000       .debug$S                   10000000     kernel32:KERNEL32.dll
 0000:fffd3000       .debug$S                   10000000     kernel32:KERNEL32.dll
 0000:fffd3000       .debug$S                   10000000     kernel32:KERNEL32.dll
 0000:fffd3000       .debug$S                   10000000     kernel32:KERNEL32.dll
 0000:fffd3000       .debug$S                   10000000     kernel32:KERNEL32.dll
 0000:fffd3000       .debug$S                   10000000     kernel32:KERNEL32.dll
 0000:fffd3000       .debug$S                   10000000     kernel32:KERNEL32.dll
 0000:fffd3000       .debug$S                   10000000     kernel32:KERNEL32.dll
 0000:fffd3000       .debug$S                   10000000     kernel32:KERNEL32.dll
 0000:fffd3000       .debug$S                   10000000     kernel32:KERNEL32.dll
 0000:fffd3000       .debug$S                   10000000     kernel32:KERNEL32.dll
 0000:fffd3000       .debug$S                   10000000     kernel32:KERNEL32.dll
 0000:fffd3000       .debug$S                   10000000     kernel32:KERNEL32.dll
 0000:fffd3000       .debug$S                   10000000     kernel32:KERNEL32.dll
 0000:fffd3000       .debug$S                   10000000     kernel32:KERNEL32.dll
 0000:fffd3000       .debug$S                   10000000     kernel32:KERNEL32.dll
 0000:fffd3000       .debug$S                   10000000     kernel32:KERNEL32.dll
 0000:fffd3000       .debug$S                   10000000     kernel32:KERNEL32.dll
 0000:fffd3000       .debug$S                   10000000     kernel32:KERNEL32.dll
 0000:fffd3000       .debug$S                   10000000     kernel32:KERNEL32.dll
 0000:fffd3000       .debug$S                   10000000     kernel32:KERNEL32.dll
 0000:fffd3000       .debug$S                   10000000     kernel32:KERNEL32.dll
 0000:fffd3000       .debug$S                   10000000     kernel32:KERNEL32.dll
 0000:fffd3000       .debug$S                   10000000     kernel32:KERNEL32.dll
 0000:fffd3000       .debug$S                   10000000     user32:USER32.dll
 0000:fffd3000       .debug$S                   10000000     user32:USER32.dll
 0000:fffd3000       .debug$S                   10000000     kernel32:KERNEL32.dll
 0000:fffd3000       .debug$S                   10000000     kernel32:KERNEL32.dll
 0000:fffd3000       .debug$S                   10000000     kernel32:KERNEL32.dll
 0000:fffd3000       .debug$S                   10000000     kernel32:KERNEL32.dll
 0000:fffd3000       .debug$S                   10000000     kernel32:KERNEL32.dll
 0000:fffd3000       .debug$S                   10000000     kernel32:KERNEL32.dll
 0000:fffd3000       .debug$S                   10000000     kernel32:KERNEL32.dll
 0000:fffd3000       .debug$S                   10000000     kernel32:KERNEL32.dll
 0000:fffd3000       .debug$S                   10000000     kernel32:KERNEL32.dll
 0000:fffd3000       .debug$S                   10000000     user32:USER32.dll
 0000:fffd3000       .debug$S                   10000000     user32:USER32.dll
 0000:fffd3000       .debug$S                   10000000     user32:USER32.dll
 0000:fffd3000       .debug$S                   10000000     kernel32:KERNEL32.dll
 0000:fffd3000       .debug$S                   10000000     user32:USER32.dll
 0000:fffd3000       .debug$S                   10000000     kernel32:KERNEL32.dll
 0000:fffd3000       .debug$S                   10000000     kernel32:KERNEL32.dll
 0000:fffd3000       .debug$S                   10000000     kernel32:KERNEL32.dll
 0000:fffd3000       .debug$S                   10000000     kernel32:KERNEL32.dll
 0000:fffd3000       .debug$S                   10000000     kernel32:KERNEL32.dll
 0000:fffd3000       .debug$S                   10000000     kernel32:KERNEL32.dll
 0000:fffd3000       .debug$S                   10000000     kernel32:KERNEL32.dll
 0000:fffd3000       .debug$S                   10000000     kernel32:KERNEL32.dll
 0000:fffd3000       .debug$S                   10000000     kernel32:KERNEL32.dll
 0000:fffd3000       .debug$S                   10000000     kernel32:KERNEL32.dll
 0000:fffd3000       .debug$S                   10000000     windowsaccessbridge-32.exp
 0000:fffd3000       .debug$S                   10000000     kernel32:KERNEL32.dll
 0000:fffd3000       .debug$S                   10000000     kernel32:KERNEL32.dll
 0000:fffd3000       .debug$S                   10000000     kernel32:KERNEL32.dll
 0000:fffd3000       .debug$S                   10000000     kernel32:KERNEL32.dll
 0000:fffd3000       .debug$S                   10000000     kernel32:KERNEL32.dll
 0000:fffd3000       .debug$S                   10000000     kernel32:KERNEL32.dll
 0001:00005dc0       $$000000                   10006dc0     LIBCMT:ulldiv.obj
 0001:00005ea0       $$000000                   10006ea0     LIBCMT:chkstk.obj
 0001:00005ecd       ?dllmain_crt_dispatch@@YGHQAUHINSTANCE__@@KQAX@Z 10006ecd f   LIBCMT:dll_dllmain.obj
 0001:00005f22       ?dllmain_crt_process_attach@@YAHQAUHINSTANCE__@@QAX@Z 10006f22 f   LIBCMT:dll_dllmain.obj
 0001:0000602c       ?dllmain_crt_process_detach@@YAH_N@Z 1000702c f   LIBCMT:dll_dllmain.obj
 0001:000060be       ?dllmain_dispatch@@YAHQAUHINSTANCE__@@KQAX@Z 100070be f   LIBCMT:dll_dllmain.obj
 0001:000061c4       ?dllmain_raw@@YGHQAUHINSTANCE__@@KQAX@Z 100071c4 f   LIBCMT:dll_dllmain.obj
 0001:000063d2       ___get_entropy             100073d2 f   LIBCMT:gs_support.obj
 0001:000064a5       ?find_pe_section@@YAPAU_IMAGE_SECTION_HEADER@@QAEI@Z 100074a5 f   LIBCMT:utility.obj
 0001:00006920       $$000000                   10007920     LIBCMT:sehprolg4.obj
 0001:00006b30       $$000000                   10007b30     libvcruntime:memcpy.obj
 0001:00006d94       TrailingUpVec              10007d94     libvcruntime:memcpy.obj
 0001:00006e40       TrailingDownVec            10007e40     libvcruntime:memcpy.obj
 0001:000070b0       $$000000                   100080b0     libvcruntime:memset.obj
 0001:00007300       _ValidateLocalCookies      10008300 f   libvcruntime:chandler4.obj
 0001:00007560       $$000000                   10008560     libvcruntime:exsup4.obj
 0001:000075f0       __unwind_handler4          100085f0 f   libvcruntime:exsup4.obj
 0001:000078ec       ?try_get_first_available_module@@YAPAUHINSTANCE__@@QBW4module_id@?A0x5c520fe1@@0@Z 100088ec f   libvcruntime:winapi_downlevel.obj
 0001:000079b0       ?try_get_function@@YAPAXW4function_id@?A0x5c520fe1@@QBDQBW4module_id@2@2@Z 100089b0 f   libvcruntime:winapi_downlevel.obj
 0001:00007bc0       $$000000                   10008bc0     libvcruntime:exsup.obj
 0001:00007be1       __unwind_handler           10008be1 f   libvcruntime:exsup.obj
 0001:000080a9       ??$BuildCatchObjectHelperInternal@V__FrameHandler3@@@@YAHPAUEHExceptionRecord@@PAXPBU_s_HandlerType@@PBU_s_CatchableType@@@Z 100090a9 f   libvcruntime:frame.obj
 0001:000081e8       ??$BuildCatchObjectInternal@V__FrameHandler3@@@@YAXPAUEHExceptionRecord@@PAXPBU_s_HandlerType@@PBU_s_CatchableType@@@Z 100091e8 f   libvcruntime:frame.obj
 0001:00008281       ??$CatchIt@V__FrameHandler3@@@@YAXPAUEHExceptionRecord@@PAUEHRegistrationNode@@PAU_CONTEXT@@PAXPBU_s_FuncInfo@@PBU_s_HandlerType@@PBU_s_CatchableType@@PBU_s_TryBlockMapEntry@@H1E@Z 10009281 f   libvcruntime:frame.obj
 0001:00008301       ??$FindHandler@V__FrameHandler3@@@@YAXPAUEHExceptionRecord@@PAUEHRegistrationNode@@PAU_CONTEXT@@PAXPBU_s_FuncInfo@@EH1@Z 10009301 f   libvcruntime:frame.obj
 0001:0000868f       ??$FindHandlerForForeignException@V__FrameHandler3@@@@YAXPAUEHExceptionRecord@@PAUEHRegistrationNode@@PAU_CONTEXT@@PAXPBU_s_FuncInfo@@HH1@Z 1000968f f   libvcruntime:frame.obj
 0001:00008982       ?CallCatchBlock@@YAPAXPAUEHExceptionRecord@@PAUEHRegistrationNode@@PAU_CONTEXT@@PBU_s_FuncInfo@@PAXHK@Z 10009982 f   libvcruntime:frame.obj
 0001:00008b46       ?CallUnexpected@@YAXPBU_s_ESTypeList@@@Z 10009b46 f   libvcruntime:frame.obj
 0001:00008b66       __catch$?CallUnexpected@@YAXPBU_s_ESTypeList@@@Z$0 10009b66 f   libvcruntime:frame.obj
 0001:00008b80       ?ExFilterRethrow@@YAHPAU_EXCEPTION_POINTERS@@@Z 10009b80 f   libvcruntime:frame.obj
 0001:00008cca       ?IsInExceptionSpec@@YAEPAUEHExceptionRecord@@PBU_s_ESTypeList@@@Z 10009cca f   libvcruntime:frame.obj
 0001:00008da0       $$000000                   10009da0     libvcruntime:lowhelpr.obj
 0001:00008f80       $$000000                   10009f80     libvcruntime:memmove.obj
 0001:000091e4       TrailingUpVec              1000a1e4     libvcruntime:memmove.obj
 0001:00009290       TrailingDownVec            1000a290     libvcruntime:memmove.obj
 0001:00009500       $$000000                   1000a500     libucrt:strlen.obj
 0001:00009590       $$000000                   1000a590     libucrt:strncat.obj
 0001:000096d0       $$000000                   1000a6d0     libucrt:strncpy.obj
 0001:00009940       ??$?RV<lambda_62491a2101a2aba6cc4a769149c84f1f>@@AAV<lambda_826c27fce7726908515bbc79a5266961>@@V<lambda_4e64bbd54b50a7b070e3ea8d795375b6>@@@?$__crt_seh_guarded_call@H@@QAEH$$QAV<lambda_62491a2101a2aba6cc4a769149c84f1f>@@AAV<lambda_826c27fce7726908515bbc79a5266961>@@$$QAV<lambda_4e64bbd54b50a7b070e3ea8d795375b6>@@@Z 1000a940 f   libucrt:output.obj
 0001:0000999b       ??$common_vsprintf@Vstandard_base@__crt_stdio_output@@D@@YAH_KQADIQBDAAV__crt_cached_ptd_host@@1@Z 1000a99b f   libucrt:output.obj
 0001:0000a73a       ??R<lambda_826c27fce7726908515bbc79a5266961>@@QBEHXZ 1000b73a f   libucrt:output.obj
 0001:0000ac84       $LN121                     1000bc84     libucrt:output.obj
 0001:0000af58       $LN130                     1000bf58     libucrt:output.obj
 0001:0000b8ff       $LN18                      1000c8ff     libucrt:output.obj
 0001:0000b913       $LN17                      1000c913     libucrt:output.obj
 0001:0000c0db       ?_fclose_internal@@YAHQAU_iobuf@@AAV__crt_cached_ptd_host@@@Z 1000d0db f   libucrt:fclose.obj
 0001:0000c172       ?_fclose_nolock_internal@@YAHQAU_iobuf@@AAV__crt_cached_ptd_host@@@Z 1000d172 f   libucrt:fclose.obj
 0001:0000c230       ??$common_fsopen@D@@YAPAU_iobuf@@QBD0H@Z 1000d230 f   libucrt:fopen.obj
 0001:0000c2fe       ??$common_getenv@D@@YAPADQBD@Z 1000d2fe f   libucrt:getenv.obj
 0001:0000c37d       ??$common_getenv_nolock@D@@YAPADQBD@Z 1000d37d f   libucrt:getenv.obj
 0001:0000c400       $$000000                   1000d400     libucrt:strcmp.obj
 0001:0000c490       $$000000                   1000d490     libucrt:strcat.obj
 0001:0000c85a       ??$?RV<lambda_03b1d95aef87969028cfba75ccab2455>@@AAV<lambda_6e4b09c48022b2350581041d5f6b0c4c>@@V<lambda_22bdf7517842c4b3e53723af5aa32b9e>@@@?$__crt_seh_guarded_call@X@@QAEX$$QAV<lambda_03b1d95aef87969028cfba75ccab2455>@@AAV<lambda_6e4b09c48022b2350581041d5f6b0c4c>@@$$QAV<lambda_22bdf7517842c4b3e53723af5aa32b9e>@@@Z 1000d85a f   libucrt:exit.obj
 0001:0000c8a7       ??R<lambda_6e4b09c48022b2350581041d5f6b0c4c>@@QBE@XZ 1000d8a7 f   libucrt:exit.obj
 0001:0000c98f       ?common_exit@@YAXHW4_crt_exit_cleanup_mode@@W4_crt_exit_return_mode@@@Z 1000d98f f   libucrt:exit.obj
 0001:0000ca26       ?exit_or_terminate_process@@YAXI@Z 1000da26 f   libucrt:exit.obj
 0001:0000ca57       ?is_managed_app@@YA_NXZ    1000da57 f   libucrt:exit.obj
 0001:0000ca99       ?should_call_terminate_process@@YA_NXZ 1000da99 f   libucrt:exit.obj
 0001:0000cab2       ?try_cor_exit_process@@YAXI@Z 1000dab2 f   libucrt:exit.obj
 0001:0000cb6f       ??$common_configure_argv@D@@YAHW4_crt_argv_mode@@@Z 1000db6f f   libucrt:argv_parsing.obj
 0001:0000ccac       ??$parse_command_line@D@@YAXPADPAPAD0PAI2@Z 1000dcac f   libucrt:argv_parsing.obj
 0001:0000ce7a       ??$common_get_or_create_environment_nolock@D@@YAPAPADXZ 1000de7a f   libucrt:environment_initialization.obj
 0001:0000cea6       ??$common_initialize_environment_nolock@D@@YAHXZ 1000dea6 f   libucrt:environment_initialization.obj
 0001:0000cf00       ??$create_environment@D@@YAQAPADQAD@Z 1000df00 f   libucrt:environment_initialization.obj
 0001:0000cfe2       ??$free_environment@D@@YAXQAPAD@Z 1000dfe2 f   libucrt:environment_initialization.obj
 0001:0000cfe2       ??$free_environment@_W@@YAXQAPA_W@Z 1000dfe2 f   libucrt:environment_initialization.obj
 0001:0000d011       ??$initialize_environment_by_cloning_nolock@D@@YAHXZ 1000e011 f   libucrt:environment_initialization.obj
 0001:0000d094       ??$uninitialize_environment_internal@D@@YAXAAPAPAD@Z 1000e094 f   libucrt:environment_initialization.obj
 0001:0000d0af       ??$uninitialize_environment_internal@_W@@YAXAAPAPA_W@Z 1000e0af f   libucrt:environment_initialization.obj
 0001:0000d125       ??$?RV<lambda_69a2805e680e0e292e8ba93315fe43a8>@@AAV<lambda_f03950bc5685219e0bcd2087efbe011e>@@V<lambda_03fcd07e894ec930e3f35da366ca99d6>@@@?$__crt_seh_guarded_call@H@@QAEH$$QAV<lambda_69a2805e680e0e292e8ba93315fe43a8>@@AAV<lambda_f03950bc5685219e0bcd2087efbe011e>@@$$QAV<lambda_03fcd07e894ec930e3f35da366ca99d6>@@@Z 1000e125 f   libucrt:onexit.obj
 0001:0000d180       ??R<lambda_f03950bc5685219e0bcd2087efbe011e>@@QBE@XZ 1000e180 f   libucrt:onexit.obj
 0001:0000d2c1       _initialize_global_variables 1000e2c1 f   libucrt:initialization.obj
 0001:0000d2ce       _initialize_c              1000e2ce f   libucrt:initialization.obj
 0001:0000d2e8       _report_memory_leaks       1000e2e8 f   libucrt:initialization.obj
 0001:0000d2e8       _uninitialize_c            1000e2e8 f   libucrt:initialization.obj
 0001:0000d2e8       _initialize_environment    1000e2e8 f   libucrt:initialization.obj
 0001:0000d2e8       _uninitialize_global_state_isolation 1000e2e8 f   libucrt:initialization.obj
 0001:0000d2e8       _initialize_global_state_isolation 1000e2e8 f   libucrt:initialization.obj
 0001:0000d2eb       _uninitialize_environment  1000e2eb f   libucrt:initialization.obj
 0001:0000d2f3       _initialize_pointers       1000e2f3 f   libucrt:initialization.obj
 0001:0000d321       _uninitialize_vcruntime    1000e321 f   libucrt:initialization.obj
 0001:0000d32a       _uninitialize_allocated_memory 1000e32a f   libucrt:initialization.obj
 0001:0000d341       _uninitialize_allocated_io_buffers 1000e341 f   libucrt:initialization.obj
 0001:0000d391       ??R<lambda_af42a3ee9806e9a7305d451646e05244>@@QBE@AAPAU__crt_multibyte_data@@@Z 1000e391 f   libucrt:initialization.obj
 0001:0000d4c0       $$000000                   1000e4c0     libucrt:strncmp.obj
 0001:0000d971       ?try_get_AreFileApisANSI@@YAP6GHXZXZ 1000e971 f   libucrt:winapi_thunks.obj
 0001:0000d98b       ?try_get_CompareStringEx@@YAP6GHPB_WK0H0HPAU_nlsversioninfo@@PAXJ@ZXZ 1000e98b f   libucrt:winapi_thunks.obj
 0001:0000d9a5       ?try_get_LCMapStringEx@@YAP6GHPB_WK0HPA_WHPAU_nlsversioninfo@@PAXJ@ZXZ 1000e9a5 f   libucrt:winapi_thunks.obj
 0001:0000d9bf       ?try_get_LocaleNameToLCID@@YAP6GKPB_WK@ZXZ 1000e9bf f   libucrt:winapi_thunks.obj
 0001:0000d9d9       ?try_get_first_available_module@@YAPAUHINSTANCE__@@QBW4module_id@?A0x391cf84c@@0@Z 1000e9d9 f   libucrt:winapi_thunks.obj
 0001:0000daa4       ?try_get_function@@YAPAXW4function_id@?A0x391cf84c@@QBDQBW4module_id@2@2@Z 1000eaa4 f   libucrt:winapi_thunks.obj
 0001:0000deb2       ??$?RV<lambda_2866be3712abc81a800a822484c830d8>@@AAV<lambda_39ca0ed439415581b5b15c265174cece>@@V<lambda_2b24c74d71094a6cd0cb82e44167d71b>@@@?$__crt_seh_guarded_call@X@@QAEX$$QAV<lambda_2866be3712abc81a800a822484c830d8>@@AAV<lambda_39ca0ed439415581b5b15c265174cece>@@$$QAV<lambda_2b24c74d71094a6cd0cb82e44167d71b>@@@Z 1000eeb2 f   libucrt:fflush.obj
 0001:0000df3e       ??$?RV<lambda_2cc53f568c5a2bb6f192f930a45d44ea>@@AAV<lambda_ab61a845afdef5b7c387490eaf3616ee>@@V<lambda_c2ffc0b7726aa6be21d5f0026187e748>@@@?$__crt_seh_guarded_call@X@@QAEX$$QAV<lambda_2cc53f568c5a2bb6f192f930a45d44ea>@@AAV<lambda_ab61a845afdef5b7c387490eaf3616ee>@@$$QAV<lambda_c2ffc0b7726aa6be21d5f0026187e748>@@@Z 1000ef3e f   libucrt:fflush.obj
 0001:0000dfea       ?common_flush_all@@YAH_N@Z 1000efea f   libucrt:fflush.obj
 0001:0000e037       ?common_flush_all_should_try_to_flush_stream@@YA_NV__crt_stdio_stream@@QAH@Z 1000f037 f   libucrt:fflush.obj
 0001:0000e068       ?is_stream_flushable_or_commitable@@YA_NJ@Z 1000f068 f   libucrt:fflush.obj
 0001:0000e1a2       ?initialize_inherited_file_handles_nolock@@YAXXZ 1000f1a2 f   libucrt:ioinit.obj
 0001:0000e258       ?initialize_stdio_handles_nolock@@YAXXZ 1000f258 f   libucrt:ioinit.obj
 0001:0000e7d2       ?fe_to_nearest@@YA_NQBN_KF@Z 1000f7d2 f   libucrt:cvt.obj
 0001:0000e875       ?fp_format_a@@YAHQBNPADIQADIH_NIW4__acrt_rounding_mode@@AAV__crt_cached_ptd_host@@@Z 1000f875 f   libucrt:cvt.obj
 0001:0000eba2       ?fp_format_e@@YAHQBNQADI1IH_NIW4__acrt_rounding_mode@@AAV__crt_cached_ptd_host@@@Z 1000fba2 f   libucrt:cvt.obj
 0001:0000ec46       ?fp_format_e_internal@@YAHQADIH_NIQAU_strflt@@1AAV__crt_cached_ptd_host@@@Z 1000fc46 f   libucrt:cvt.obj
 0001:0000ed99       ?fp_format_f@@YAHQBNQADI1IHW4__acrt_rounding_mode@@AAV__crt_cached_ptd_host@@@Z 1000fd99 f   libucrt:cvt.obj
 0001:0000ee2f       ?fp_format_f_internal@@YAHQADIHQAU_strflt@@_NAAV__crt_cached_ptd_host@@@Z 1000fe2f f   libucrt:cvt.obj
 0001:0000ef1d       ?fp_format_g@@YAHQBNQADI1IH_NIW4__acrt_rounding_mode@@AAV__crt_cached_ptd_host@@@Z 1000ff1d f   libucrt:cvt.obj
 0001:0000efec       ?fp_format_nan_or_infinity@@YAHW4__acrt_fp_class@@_NPADI1@Z 1000ffec f   libucrt:cvt.obj
 0001:0000f081       ?shift_bytes@@YAXQADI0H@Z  10010081 f   libucrt:cvt.obj
 0001:0000f0b5       ?should_round_up@@YA_NQBN_KFW4__acrt_rounding_mode@@@Z 100100b5 f   libucrt:cvt.obj
 0001:0000f6f6       ??$?RV<lambda_15ade71b0218206bbe3333a0c9b79046>@@AAV<lambda_da44e0f8b0f19ba52fefafb335991732>@@V<lambda_207f2d024fc103971653565357d6cd41>@@@?$__crt_seh_guarded_call@X@@QAEX$$QAV<lambda_15ade71b0218206bbe3333a0c9b79046>@@AAV<lambda_da44e0f8b0f19ba52fefafb335991732>@@$$QAV<lambda_207f2d024fc103971653565357d6cd41>@@@Z 100106f6 f   libucrt:per_thread_data.obj
 0001:0000f748       ??$?RV<lambda_38edbb1296d33220d7e4dd0ed76b244a>@@AAV<lambda_5ce1d447e08cb34b2473517608e21441>@@V<lambda_fb385d3da700c9147fc39e65dd577a8c>@@@?$__crt_seh_guarded_call@X@@QAEX$$QAV<lambda_38edbb1296d33220d7e4dd0ed76b244a>@@AAV<lambda_5ce1d447e08cb34b2473517608e21441>@@$$QAV<lambda_fb385d3da700c9147fc39e65dd577a8c>@@@Z 10010748 f   libucrt:per_thread_data.obj
 0001:0000f7b3       ??$?RV<lambda_6affb1475c98b40b75cdec977db92e3c>@@AAV<lambda_b8d4b9c228a6ecc3f80208dbb4b4a104>@@V<lambda_608742c3c92a14382c1684fc64f96c88>@@@?$__crt_seh_guarded_call@X@@QAEX$$QAV<lambda_6affb1475c98b40b75cdec977db92e3c>@@AAV<lambda_b8d4b9c228a6ecc3f80208dbb4b4a104>@@$$QAV<lambda_608742c3c92a14382c1684fc64f96c88>@@@Z 100107b3 f   libucrt:per_thread_data.obj
 0001:0000f808       ??$?RV<lambda_a7e850c220f1c8d1e6efeecdedd162c6>@@AAV<lambda_46720907175c18b6c9d2717bc0d2d362>@@V<lambda_9048902d66e8d99359bc9897bbb930a8>@@@?$__crt_seh_guarded_call@X@@QAEX$$QAV<lambda_a7e850c220f1c8d1e6efeecdedd162c6>@@AAV<lambda_46720907175c18b6c9d2717bc0d2d362>@@$$QAV<lambda_9048902d66e8d99359bc9897bbb930a8>@@@Z 10010808 f   libucrt:per_thread_data.obj
 0001:0000f862       ?construct_ptd@@YAXQAU__acrt_ptd@@QAPAU__crt_locale_data@@@Z 10010862 f   libucrt:per_thread_data.obj
 0001:0000f8fb       ?destroy_fls@@YGXPAX@Z     100108fb f   libucrt:per_thread_data.obj
 0001:0000f91c       ?destroy_ptd@@YAXQAU__acrt_ptd@@@Z 1001091c f   libucrt:per_thread_data.obj
 0001:0000f9e9       ?replace_current_thread_locale_nolock@@YAXQAU__acrt_ptd@@QAU__crt_locale_data@@@Z 100109e9 f   libucrt:per_thread_data.obj
 0001:0000fd4b       ??$?RV<lambda_e5124f882df8998aaf41531e079ba474>@@AAV<lambda_3e16ef9562a7dcce91392c22ab16ea36>@@V<lambda_e25ca0880e6ef98be67edffd8c599615>@@@?$__crt_seh_guarded_call@X@@QAEX$$QAV<lambda_e5124f882df8998aaf41531e079ba474>@@AAV<lambda_3e16ef9562a7dcce91392c22ab16ea36>@@$$QAV<lambda_e25ca0880e6ef98be67edffd8c599615>@@@Z 10010d4b f   libucrt:wsetlocale.obj
 0001:0000fdeb       ??$?RV<lambda_d422a76eb4c3bf3ad751449ab71a6ea4>@@AAV<lambda_c9ba49e555ba839a7b07aa3fbecb7617>@@V<lambda_9476263c8ee91a25d21c55370bdb50de>@@@?$__crt_seh_guarded_call@H@@QAEH$$QAV<lambda_d422a76eb4c3bf3ad751449ab71a6ea4>@@AAV<lambda_c9ba49e555ba839a7b07aa3fbecb7617>@@$$QAV<lambda_9476263c8ee91a25d21c55370bdb50de>@@@Z 10010deb f   libucrt:close.obj
 0001:00010093       ?find_or_allocate_unused_stream_nolock@@YA?AV__crt_stdio_stream@@XZ 10011093 f   libucrt:stream.obj
 0001:0001037f       ??$common_openfile@D@@YAPAU_iobuf@@QBD0HV__crt_stdio_stream@@@Z 1001137f f   libucrt:openfile.obj
 0001:00010780       ?<lambda_invoker_cdecl>@<lambda_838c7f62c73c983481e27c09e84b0b5d>@@CAHPBX0@Z 10011780 f   libucrt:argv_wildcards.obj
 0001:0001092d       ??$common_expand_argv_wildcards@D@@YAHQAPADQAPAPAD@Z 1001192d f   libucrt:argv_wildcards.obj
 0001:00010aaa       ??$copy_and_add_argument_to_buffer@D@@YAHQBD0IAAV?$argument_list@D@?A0x5f5c8891@@@Z 10011aaa f   libucrt:argv_wildcards.obj
 0001:00010b5b       ??$expand_argument_wildcards@D@@YAHQAD0AAV?$argument_list@D@?A0x5f5c8891@@@Z 10011b5b f   libucrt:argv_wildcards.obj
 0001:00010de0       ??1?$argument_list@D@?A0x5f5c8891@@QAE@XZ 10011de0 f   libucrt:argv_wildcards.obj
 0001:00010f1c       ?expand_if_necessary@?$argument_list@D@?A0x5f5c8891@@AAEHXZ 10011f1c f   libucrt:argv_wildcards.obj
 0001:0001114c       ??$?RV<lambda_ceb1ee4838e85a9d631eb091e2fbe199>@@AAV<lambda_ae742caa10f662c28703da3d2ea5e57e>@@V<lambda_cd08b5d6af4937fe54fc07d0c9bf6b37>@@@?$__crt_seh_guarded_call@X@@QAEX$$QAV<lambda_ceb1ee4838e85a9d631eb091e2fbe199>@@AAV<lambda_ae742caa10f662c28703da3d2ea5e57e>@@$$QAV<lambda_cd08b5d6af4937fe54fc07d0c9bf6b37>@@@Z 1001214c f   libucrt:mbctype.obj
 0001:00011199       ??R<lambda_ae742caa10f662c28703da3d2ea5e57e>@@QBE@XZ 10012199 f   libucrt:mbctype.obj
 0001:0001121c       ?CPtoLocaleName@@YAPB_WH@Z 1001221c f   libucrt:mbctype.obj
 0001:0001125a       ?getSystemCP@@YAHH@Z       1001225a f   libucrt:mbctype.obj
 0001:000112cb       ?setSBCS@@YAXPAU__crt_multibyte_data@@@Z 100122cb f   libucrt:mbctype.obj
 0001:0001132e       ?setSBUpLow@@YAXPAU__crt_multibyte_data@@@Z 1001232e f   libucrt:mbctype.obj
 0001:000114d3       ?setmbcp_internal@@YAHH_NQAU__acrt_ptd@@QAPAU__crt_multibyte_data@@@Z 100124d3 f   libucrt:mbctype.obj
 0001:00011628       ?update_thread_multibyte_data_internal@@YAPAU__crt_multibyte_data@@QAU__acrt_ptd@@QAPAU1@@Z 10012628 f   libucrt:mbctype.obj
 0001:00011928       _memcpy_s                  10012928 f   libucrt:cfout.obj
 0001:00011928       _memcpy_s                  10012928 f   libucrt:mbctype.obj
 0001:000119a9       ?x_ismbbtype_l@@YAHPAU__crt_locale_pointers@@IHH@Z 100129a9 f   libucrt:ismbbyte.obj
 0001:00011a2a       ?filter_mbtowcs_flags@@YAKIK@Z 10012a2a f   libucrt:multibytetowidechar.obj
 0001:00011aec       ?filter_wcstomb_flags@@YAKIK@Z 10012aec f   libucrt:widechartomultibyte.obj
 0001:00011be8       ?find_end_of_double_null_terminated_sequence@@YAPB_WQB_W@Z 10012be8 f   libucrt:get_environment_from_os.obj
 0001:00011cbf       ??$common_set_variable_in_environment_nolock@D@@YAHQADH@Z 10012cbf f   libucrt:setenv.obj
 0001:00011f1f       ??$copy_environment@D@@YAPAPADQAPAD@Z 10012f1f f   libucrt:setenv.obj
 0001:00011fcf       ??$ensure_current_environment_is_not_initial_environment_nolock@D@@YAXXZ 10012fcf f   libucrt:setenv.obj
 0001:00011fe9       ??$find_in_environment_nolock@D@@YAHQBDI@Z 10012fe9 f   libucrt:setenv.obj
 0001:0001216a       ??$?RV<lambda_cbab9ec6f41b0180b23cc171c22676b0>@@AAV<lambda_44731a7d0e6d81c3e6aa82d741081786>@@V<lambda_4b292cb8dd18144e164572427af410ab>@@@?$__crt_seh_guarded_call@P6AXH@Z@@QAEP6AXH@Z$$QAV<lambda_cbab9ec6f41b0180b23cc171c22676b0>@@AAV<lambda_44731a7d0e6d81c3e6aa82d741081786>@@$$QAV<lambda_4b292cb8dd18144e164572427af410ab>@@@Z 1001316a f   libucrt:signal.obj
 0001:000121d2       ?get_global_action_nolock@@YAPAP6AXH@ZH@Z 100131d2 f   libucrt:signal.obj
 0001:00012214       ?siglookup@@YAPAU__crt_signal_action_t@@HQAU1@@Z 10013214 f   libucrt:signal.obj
 0001:000124dc       ?GetTableIndexFromLocaleName@@YAHPB_W@Z 100134dc f   libucrt:lcidtoname_downlevel.obj
 0001:00012558       ??$?RV<lambda_9e9de3de5fa147e2223d7db92bc10aa6>@@AAV<lambda_38ce7e780aa69e748d6df282ebc68efe>@@V<lambda_8ca6da459f0f6780f1cff60fdc3d00e5>@@@?$__crt_seh_guarded_call@H@@QAEH$$QAV<lambda_9e9de3de5fa147e2223d7db92bc10aa6>@@AAV<lambda_38ce7e780aa69e748d6df282ebc68efe>@@$$QAV<lambda_8ca6da459f0f6780f1cff60fdc3d00e5>@@@Z 10013558 f   libucrt:commit.obj
 0001:00012677       ?write_double_translated_ansi_nolock@@YA?AUwrite_result@?A0x17268360@@HQBDIAAV__crt_cached_ptd_host@@@Z 10013677 f   libucrt:write.obj
 0001:00012a3e       ?write_double_translated_unicode_nolock@@YA?AUwrite_result@?A0x17268360@@QBDI@Z 10013a3e f   libucrt:write.obj
 0001:00012aa6       ?write_requires_double_translation_nolock@@YA_NHAAV__crt_cached_ptd_host@@@Z 10013aa6 f   libucrt:write.obj
 0001:00012b23       ?write_text_ansi_nolock@@YA?AUwrite_result@?A0x17268360@@HQBDI@Z 10013b23 f   libucrt:write.obj
 0001:00012bfe       ?write_text_utf16le_nolock@@YA?AUwrite_result@?A0x17268360@@HQBDI@Z 10013bfe f   libucrt:write.obj
 0001:00012ce7       ?write_text_utf8_nolock@@YA?AUwrite_result@?A0x17268360@@HQBDI@Z 10013ce7 f   libucrt:write.obj
 0001:0001394b       ?check_trailing@@YA_NPBDW4__acrt_has_trailing_digits@@@Z 1001494b f   libucrt:_fptostr.obj
 0001:0001396e       ?should_round_up@@YA_NQBD0HW4__acrt_has_trailing_digits@@W4__acrt_rounding_mode@@@Z 1001496e f   libucrt:_fptostr.obj
 0001:00015650       ??R<lambda_e96123212306c92459f955e8e4eac55d>@@QBEIPBD@Z 10016650 f   libucrt:mbrtowc.obj
 0001:000157c7       ??$common_flush_and_write_nolock@D@@YAHHV__crt_stdio_stream@@AAV__crt_cached_ptd_host@@@Z 100167c7 f   libucrt:_flsbuf.obj
 0001:000158bd       ??$write_buffer_nolock@D@@YA_NDV__crt_stdio_stream@@AAV__crt_cached_ptd_host@@@Z 100168bd f   libucrt:_flsbuf.obj
 0001:0001598f       ?stream_is_at_end_of_file_nolock@@YA_NV__crt_stdio_stream@@@Z 1001698f f   libucrt:_flsbuf.obj
 0001:00015bdc       ?free_crt_array_internal@@YAXQAPBXI@Z 10016bdc f   libucrt:inittime.obj
 0001:00015f8d       ??$common_sopen_dispatch@D@@YAHQBDHHHQAHH@Z 10016f8d f   libucrt:open.obj
 0001:00016068       ?configure_text_mode@@YAHHUfile_options@?A0xa9d50aae@@HAAW4__crt_lowio_text_mode@@@Z 10017068 f   libucrt:open.obj
 0001:000162be       ?create_file@@YAPAXQB_WQAU_SECURITY_ATTRIBUTES@@Ufile_options@?A0xa9d50aae@@@Z 100172be f   libucrt:open.obj
 0001:000162e3       ?decode_open_create_flags@@YAKH@Z 100172e3 f   libucrt:open.obj
 0001:00016353       ?decode_options@@YA?AUfile_options@?A0xa9d50aae@@HHH@Z 10017353 f   libucrt:open.obj
 0001:000164cd       ?truncate_ctrl_z_if_present@@YAHH@Z 100174cd f   libucrt:open.obj
 0001:0001692f       ?InternalCompareStringA@@YAHPAU__crt_locale_pointers@@PB_WKPBDH2HH@Z 1001792f f   libucrt:comparestringa.obj
 0001:0001710e       ??$common_tcsncpy_s@D@@YAHQADIQBDI@Z 1001810e f   libucrt:strncpy_s.obj
 0001:000171d0       $$000000                   100181d0     libucrt:strpbrk.obj
 0001:000172b4       ?__acrt_LCMapStringA_stat@@YAHPAU__crt_locale_pointers@@PB_WKPBDHPADHHH@Z 100182b4 f   libucrt:lcmapstringa.obj
 0001:000174ec       ?initialize_multibyte@@YAHXZ 100184ec f   libucrt:multibyte_initializer.obj
 0001:0001762c       ??$common_lseek@_J@@YA_JH_JHAAV__crt_cached_ptd_host@@@Z 1001862c f   libucrt:lseek.obj
 0001:00017751       ??$common_lseek_nolock@_J@@YA_JH_JHAAV__crt_cached_ptd_host@@@Z 10018751 f   libucrt:lseek.obj
 0001:000178a4       ??$translate_text_mode_nolock@D@@YAHHQADI@Z 100188a4 f   libucrt:read.obj
 0001:000179f1       ??$translate_text_mode_nolock@_W@@YAHHQA_WI@Z 100189f1 f   libucrt:read.obj
 0001:00017bab       ?translate_ansi_or_utf8_nolock@@YAHHQADIQA_WI@Z 10018bab f   libucrt:read.obj
 0001:00017d02       ?translate_utf16_from_console_nolock@@YAHHQA_WI@Z 10018d02 f   libucrt:read.obj
 0001:00018230       $$000000                   10019230     libucrt:log10_impl.obj
 0001:00018340       $$000000                   10019340     libucrt:ceil_pentium4.obj
 0001:0001845d       ?to_abstract_control@@YA?AW4__acrt_fenv_abstract_control@@W4__acrt_fenv_machine_sse_control@@@Z 1001945d f   libucrt:_fenvutils.obj
 0001:0001850d       ?to_abstract_control@@YA?AW4__acrt_fenv_abstract_control@@W4__acrt_fenv_machine_x87_control@@@Z 1001950d f   libucrt:_fenvutils.obj
 0001:000185ba       ?to_machine_sse_control@@YA?AW4__acrt_fenv_machine_sse_control@@W4__acrt_fenv_abstract_control@@@Z 100195ba f   libucrt:_fenvutils.obj
 0001:00018670       ?to_machine_x87_control@@YA?AW4__acrt_fenv_machine_x87_control@@W4__acrt_fenv_abstract_control@@@Z 10019670 f   libucrt:_fenvutils.obj
 0001:00018c30       $$000000                   10019c30     libucrt:_strnicm.obj
 0001:00018fc4       ?__dcrt_lowio_initialize_console_output@@YAXXZ 10019fc4 f   libucrt:initcon.obj
 0001:0001906e       ___hw_cw_sse2              1001a06e f   libucrt:ieee87.obj
 0001:000194f4       __hw_cw                    1001a4f4 f   libucrt:ieee87.obj
 0001:000195b0       $$000000                   1001a5b0     libucrt:log10_pentium4.obj
 0001:00019840       $$000000                   1001a840     libucrt:87tran.obj
 0001:00019a50       $$000000                   1001aa50     libucrt:87disp.obj
 0001:00019cb0       $$000000                   1001acb0     libucrt:common.obj
 0001:00019e40       $$000000                   1001ae40     libucrt:genexcep.obj
 0001:0001b080       $$000000                   1001c080     LIBCMT:ulldvrm.obj
 0001:0001b120       $$000000                   1001c120     LIBCMT:ullrem.obj
 0001:0001b1a0       $$000000                   1001c1a0     LIBCMT:llmul.obj
 0001:0001b1e0       $$000000                   1001c1e0     LIBCMT:lldiv.obj
 0001:0001b290       $$000000                   1001c290     LIBCMT:llrem.obj
 0001:0001b350       $$000000                   1001c350     LIBCMT:llshl.obj
 0001:0001b370       $$000000                   1001c370     LIBCMT:ullshr.obj
 0001:0001b390       $$000000                   1001c390     LIBCMT:ftol2.obj
 0001:0001b450       $$000000                   1001c450     LIBCMT:alloca16.obj
 0001:0001b480       $$000000                   1001c480     libvcruntime:strrchr.obj
 0001:0001b5c0       $$000000                   1001c5c0     libvcruntime:strchr.obj
 0001:0001b6eb       __ehhandler$?CallUnexpected@@YAXPBU_s_ESTypeList@@@Z 1001c6eb f   libvcruntime:frame.obj
 0001:0001b706       __ehhandler$?common_exit@@YAXHW4_crt_exit_cleanup_mode@@W4_crt_exit_return_mode@@@Z 1001c706 f   libucrt:exit.obj
 0001:0001b723       __ehhandler$?try_cor_exit_process@@YAXI@Z 1001c723 f   libucrt:exit.obj
 0001:0001b740       __ehhandler$___dcrt_uninitialize_environments_nolock 1001c740 f   libucrt:environment_initialization.obj
 0001:0001b75d       __ehhandler$__execute_onexit_table 1001c75d f   libucrt:onexit.obj
 0001:0001b77a       __ehhandler$?write_double_translated_ansi_nolock@@YA?AUwrite_result@?A0x17268360@@HQBDIAAV__crt_cached_ptd_host@@@Z 1001c77a f   libucrt:write.obj
 0002:00003510       _GS_ExceptionPointers      10020510     LIBCMT:gs_report.obj
 0002:0000353c       ?ExceptionTemplate@?1??_CxxThrowException@@9@8@4UEHExceptionRecord@@B 1002053c     libvcruntime:throw.obj
 0002:00003560       ?tokenTable@@3QBQBDB       10020560     libvcruntime:undname.obj
 0002:000035a0       ?nameTable@@3QBQBDB        100205a0     libvcruntime:undname.obj
 0002:000036e8       ?rttiTable@@3QBQBDB        100206e8     libvcruntime:undname.obj
 0002:00003cf8       ?module_names@?A0x5c520fe1@@3QBQB_WB 10020cf8     libvcruntime:winapi_downlevel.obj
 0002:00003db0       ?candidate_modules@?1??try_get_FlsAlloc@@YAP6GKP6GXPAX@Z@ZXZ@4QBW4module_id@?A0x5c520fe1@@B 10020db0     libvcruntime:winapi_downlevel.obj
 0002:00003dc4       ?candidate_modules@?1??try_get_FlsFree@@YAP6GHK@ZXZ@4QBW4module_id@?A0x5c520fe1@@B 10020dc4     libvcruntime:winapi_downlevel.obj
 0002:00003dd4       ?candidate_modules@?1??try_get_FlsGetValue@@YAP6GPAXK@ZXZ@4QBW4module_id@?A0x5c520fe1@@B 10020dd4     libvcruntime:winapi_downlevel.obj
 0002:00003de8       ?candidate_modules@?1??try_get_FlsSetValue@@YAP6GHKPAX@ZXZ@4QBW4module_id@?A0x5c520fe1@@B 10020de8     libvcruntime:winapi_downlevel.obj
 0002:00003dfc       ?candidate_modules@?1??try_get_InitializeCriticalSectionEx@@YAP6GHPAU_RTL_CRITICAL_SECTION@@KK@ZXZ@4QBW4module_id@?A0x5c520fe1@@B 10020dfc     libvcruntime:winapi_downlevel.obj
 0002:00004020       ___acrt_initializers       10021020     libucrt:initialization.obj
 0002:000040a0       ?errtable@@3QBUerrentry@?A0x31fdb9ec@@B 100210a0     libucrt:errno.obj
 0002:00004208       ?module_names@?A0x391cf84c@@3QBQB_WB 10021208     libucrt:winapi_thunks.obj
 0002:00004704       ?candidate_modules@?1??try_get_AreFileApisANSI@@YAP6GHXZXZ@4QBW4module_id@?A0x391cf84c@@B 10021704     libucrt:winapi_thunks.obj
 0002:00004718       ?candidate_modules@?1??try_get_CompareStringEx@@YAP6GHPB_WK0H0HPAU_nlsversioninfo@@PAXJ@ZXZ@4QBW4module_id@?A0x391cf84c@@B 10021718     libucrt:winapi_thunks.obj
 0002:00004730       ?candidate_modules@?1??try_get_InitializeCriticalSectionEx@@YAP6GHPAU_RTL_CRITICAL_SECTION@@KK@ZXZ@4QBW4module_id@?A0x391cf84c@@B 10021730     libucrt:winapi_thunks.obj
 0002:00004738       ?candidate_modules@?1??try_get_LCMapStringEx@@YAP6GHPB_WK0HPA_WHPAU_nlsversioninfo@@PAXJ@ZXZ@4QBW4module_id@?A0x391cf84c@@B 10021738     libucrt:winapi_thunks.obj
 0002:00004750       ?candidate_modules@?1??try_get_LocaleNameToLCID@@YAP6GKPB_WK@ZXZ@4QBW4module_id@?A0x391cf84c@@B 10021750     libucrt:winapi_thunks.obj
 0002:0000476c       ?candidate_modules@?1??try_get_AppPolicyGetProcessTerminationMethod@@YAP6GJPAXPAW4AppPolicyProcessTerminationMethod@@@ZXZ@4QBW4module_id@?A0x391cf84c@@B 1002176c     libucrt:winapi_thunks.obj
 0002:00004798       ?candidate_modules@?1??try_get_FlsAlloc@@YAP6GKP6GXPAX@Z@ZXZ@4QBW4module_id@?A0x391cf84c@@B 10021798     libucrt:winapi_thunks.obj
 0002:000047a0       ?candidate_modules@?1??try_get_FlsFree@@YAP6GHK@ZXZ@4QBW4module_id@?A0x391cf84c@@B 100217a0     libucrt:winapi_thunks.obj
 0002:000047a8       ?candidate_modules@?1??try_get_FlsGetValue@@YAP6GPAXK@ZXZ@4QBW4module_id@?A0x391cf84c@@B 100217a8     libucrt:winapi_thunks.obj
 0002:000047b0       ?candidate_modules@?1??try_get_FlsSetValue@@YAP6GHKPAX@ZXZ@4QBW4module_id@?A0x391cf84c@@B 100217b0     libucrt:winapi_thunks.obj
 0002:000047b8       ?strings@?1??fp_format_nan_or_infinity@@YAHW4__acrt_fp_class@@_NPADI1@Z@4QAY03QBDA 100217b8     libucrt:cvt.obj
 0002:00004d1c       ?_mb_locale_names@@3QBQB_WB 10021d1c     libucrt:mbctype.obj
 0002:00005360       ?LcidToLocaleNameTable@?A0x881e4c05@@3QBULcidToLocaleName@1@B 10022360     libucrt:lcidtoname_downlevel.obj
 0002:00006488       ?LocaleNameToIndexTable@?A0x881e4c05@@3QBULocaleNameIndex@1@B 10023488     libucrt:lcidtoname_downlevel.obj
 0002:00007dc0       LOG_name                   10024dc0     libucrt:log10_impl.obj
 0002:00007dd0       _One                       10024dd0     libucrt:ceil_pentium4.obj
 0002:00007de0       _Bns                       10024de0     libucrt:ceil_pentium4.obj
 0002:00007df0       _Zero                      10024df0     libucrt:ceil_pentium4.obj
 0002:00007e00       _S                         10024e00     libucrt:ceil_pentium4.obj
 0002:00007e10       _NegZero                   10024e10     libucrt:ceil_pentium4.obj
 0002:00007e30       emask                      10024e30     libucrt:log10_pentium4.obj
 0002:00007e40       CC                         10024e40     libucrt:log10_pentium4.obj
 0002:00007e50       Magic                      10024e50     libucrt:log10_pentium4.obj
 0002:00007e60       hi_mask                    10024e60     libucrt:log10_pentium4.obj
 0002:00007e70       LOG10_2                    10024e70     libucrt:log10_pentium4.obj
 0002:00007e80       place_L                    10024e80     libucrt:log10_pentium4.obj
 0002:00007ea0       One                        10024ea0     libucrt:log10_pentium4.obj
 0002:00007eb0       Zero                       10024eb0     libucrt:log10_pentium4.obj
 0002:00007ec0       Two52                      10024ec0     libucrt:log10_pentium4.obj
 0002:00007ed0       Infs                       10024ed0     libucrt:log10_pentium4.obj
 0002:00007ee0       NaN                        10024ee0     libucrt:log10_pentium4.obj
 0002:00007ef0       coeff                      10024ef0     libucrt:log10_pentium4.obj
 0002:00007f4e       _log2max                   10024f4e     libucrt:87tran.obj
 0002:00007f58       _smallarg                  10024f58     libucrt:87tran.obj
 0002:00007f62       _half                      10024f62     libucrt:87tran.obj
 0002:00007fae       One                        10024fae     libucrt:87disp.obj
 0002:00007fb6       Three                      10024fb6     libucrt:87disp.obj
 0002:00007fbe       XAMtoTagTab                10024fbe     libucrt:87disp.obj
 0002:00007fd0       One                        10024fd0     libucrt:common.obj
 0002:00007fe4       DblMax                     10024fe4     libucrt:common.obj
 0002:00007fec       DblMin                     10024fec     libucrt:common.obj
 0002:00007ff4       IeeeAdjO                   10024ff4     libucrt:common.obj
 0002:00007ffc       IeeeAdjU                   10024ffc     libucrt:common.obj
 0002:00008004       _infinity                  10025004     libucrt:common.obj
 0002:0000800c       _zero                      1002500c     libucrt:common.obj
 0002:00008048       _over                      10025048     libucrt:fpctrl.obj
 0002:00008054       _under                     10025054     libucrt:fpctrl.obj
 0002:00008888       ?_names@?1??_get_fname@@9@4QBU<unnamed-type-_names>@?1??1@YAPADI@Z@B 10025888     libucrt:fpexcept.obj
 0002:00009058       __sehtable$?dllmain_crt_process_attach@@YAHQAUHINSTANCE__@@QAX@Z 10026058     LIBCMT:dll_dllmain.obj
 0002:00009078       __sehtable$?dllmain_crt_process_detach@@YAH_N@Z 10026078     LIBCMT:dll_dllmain.obj
 0002:00009098       __sehtable$?dllmain_dispatch@@YAHQAUHINSTANCE__@@KQAX@Z 10026098     LIBCMT:dll_dllmain.obj
 0002:000090f0       __sehtable$___scrt_is_nonwritable_in_current_image 100260f0     LIBCMT:utility.obj
 0002:00009110       __sehtable$?FrameUnwindToState@__FrameHandler3@@SAXPAUEHRegistrationNode@@PAXPBU_s_FuncInfo@@H@Z 10026110     libvcruntime:frame.obj
 0002:00009138       __sehtable$?CallCatchBlock@@YAPAXPAUEHExceptionRecord@@PAUEHRegistrationNode@@PAU_CONTEXT@@PBU_s_FuncInfo@@PAXHK@Z 10026138     libvcruntime:frame.obj
 0002:00009160       __catchsym$?CallUnexpected@@YAXPBU_s_ESTypeList@@@Z$2 10026160     libvcruntime:frame.obj
 0002:00009170       __unwindtable$?CallUnexpected@@YAXPBU_s_ESTypeList@@@Z 10026170     libvcruntime:frame.obj
 0002:00009180       __tryblocktable$?CallUnexpected@@YAXPBU_s_ESTypeList@@@Z 10026180     libvcruntime:frame.obj
 0002:00009194       __ehfuncinfo$?CallUnexpected@@YAXPBU_s_ESTypeList@@@Z 10026194     libvcruntime:frame.obj
 0002:000091b8       __sehtable$??$BuildCatchObjectHelperInternal@V__FrameHandler3@@@@YAHPAUEHExceptionRecord@@PAXPBU_s_HandlerType@@PBU_s_CatchableType@@@Z 100261b8     libvcruntime:frame.obj
 0002:000091d8       __sehtable$??$BuildCatchObjectInternal@V__FrameHandler3@@@@YAXPAUEHExceptionRecord@@PAXPBU_s_HandlerType@@PBU_s_CatchableType@@@Z 100261d8     libvcruntime:frame.obj
 0002:00009230       __sehtable$___DestructExceptionObject 10026230     libvcruntime:ehhelpers.obj
 0002:00009250       __sehtable$??$?RV<lambda_62491a2101a2aba6cc4a769149c84f1f>@@AAV<lambda_826c27fce7726908515bbc79a5266961>@@V<lambda_4e64bbd54b50a7b070e3ea8d795375b6>@@@?$__crt_seh_guarded_call@H@@QAEH$$QAV<lambda_62491a2101a2aba6cc4a769149c84f1f>@@AAV<lambda_826c27fce7726908515bbc79a5266961>@@$$QAV<lambda_4e64bbd54b50a7b070e3ea8d795375b6>@@@Z 10026250     libucrt:output.obj
 0002:00009270       __sehtable$?_fclose_internal@@YAHQAU_iobuf@@AAV__crt_cached_ptd_host@@@Z 10026270     libucrt:fclose.obj
 0002:00009290       __sehtable$??$common_fsopen@D@@YAPAU_iobuf@@QBD0H@Z 10026290     libucrt:fopen.obj
 0002:000092b0       __sehtable$??$common_getenv@D@@YAPADQBD@Z 100262b0     libucrt:getenv.obj
 0002:000092d0       __sehtable$__query_new_handler 100262d0     libucrt:new_handler.obj
 0002:000092ec       __ehfuncinfo$?try_cor_exit_process@@YAXI@Z 100262ec     libucrt:exit.obj
 0002:000092ec       __ehfuncinfo$?write_double_translated_ansi_nolock@@YA?AUwrite_result@?A0x17268360@@HQBDIAAV__crt_cached_ptd_host@@@Z 100262ec     libucrt:write.obj
 0002:00009310       __unwindtable$?common_exit@@YAXHW4_crt_exit_cleanup_mode@@W4_crt_exit_return_mode@@@Z 10026310     libucrt:exit.obj
 0002:00009318       __ehfuncinfo$?common_exit@@YAXHW4_crt_exit_cleanup_mode@@W4_crt_exit_return_mode@@@Z 10026318     libucrt:exit.obj
 0002:00009340       __sehtable$??R<lambda_6e4b09c48022b2350581041d5f6b0c4c>@@QBE@XZ 10026340     libucrt:exit.obj
 0002:00009360       __sehtable$??$?RV<lambda_03b1d95aef87969028cfba75ccab2455>@@AAV<lambda_6e4b09c48022b2350581041d5f6b0c4c>@@V<lambda_22bdf7517842c4b3e53723af5aa32b9e>@@@?$__crt_seh_guarded_call@X@@QAEX$$QAV<lambda_03b1d95aef87969028cfba75ccab2455>@@AAV<lambda_6e4b09c48022b2350581041d5f6b0c4c>@@$$QAV<lambda_22bdf7517842c4b3e53723af5aa32b9e>@@@Z 10026360     libucrt:exit.obj
 0002:0000937c       __unwindtable$___dcrt_uninitialize_environments_nolock 1002637c     libucrt:environment_initialization.obj
 0002:0000938c       __ehfuncinfo$___dcrt_uninitialize_environments_nolock 1002638c     libucrt:environment_initialization.obj
 0002:000093b0       __unwindtable$__execute_onexit_table 100263b0     libucrt:onexit.obj
 0002:000093b8       __ehfuncinfo$__execute_onexit_table 100263b8     libucrt:onexit.obj
 0002:000093e0       __sehtable$??$?RV<lambda_69a2805e680e0e292e8ba93315fe43a8>@@AAV<lambda_f03950bc5685219e0bcd2087efbe011e>@@V<lambda_03fcd07e894ec930e3f35da366ca99d6>@@@?$__crt_seh_guarded_call@H@@QAEH$$QAV<lambda_69a2805e680e0e292e8ba93315fe43a8>@@AAV<lambda_f03950bc5685219e0bcd2087efbe011e>@@$$QAV<lambda_03fcd07e894ec930e3f35da366ca99d6>@@@Z 100263e0     libucrt:onexit.obj
 0002:00009400       __sehtable$_terminate      10026400     libucrt:terminate.obj
 0002:00009420       __sehtable$__fcloseall     10026420     libucrt:closeall.obj
 0002:00009440       __sehtable$??$?RV<lambda_2866be3712abc81a800a822484c830d8>@@AAV<lambda_39ca0ed439415581b5b15c265174cece>@@V<lambda_2b24c74d71094a6cd0cb82e44167d71b>@@@?$__crt_seh_guarded_call@X@@QAEX$$QAV<lambda_2866be3712abc81a800a822484c830d8>@@AAV<lambda_39ca0ed439415581b5b15c265174cece>@@$$QAV<lambda_2b24c74d71094a6cd0cb82e44167d71b>@@@Z 10026440     libucrt:fflush.obj
 0002:00009460       __sehtable$??$?RV<lambda_2cc53f568c5a2bb6f192f930a45d44ea>@@AAV<lambda_ab61a845afdef5b7c387490eaf3616ee>@@V<lambda_c2ffc0b7726aa6be21d5f0026187e748>@@@?$__crt_seh_guarded_call@X@@QAEX$$QAV<lambda_2cc53f568c5a2bb6f192f930a45d44ea>@@AAV<lambda_ab61a845afdef5b7c387490eaf3616ee>@@$$QAV<lambda_c2ffc0b7726aa6be21d5f0026187e748>@@@Z 10026460     libucrt:fflush.obj
 0002:00009480       __sehtable$___acrt_initialize_lowio 10026480     libucrt:ioinit.obj
 0002:000094a0       __sehtable$??$?RV<lambda_15ade71b0218206bbe3333a0c9b79046>@@AAV<lambda_da44e0f8b0f19ba52fefafb335991732>@@V<lambda_207f2d024fc103971653565357d6cd41>@@@?$__crt_seh_guarded_call@X@@QAEX$$QAV<lambda_15ade71b0218206bbe3333a0c9b79046>@@AAV<lambda_da44e0f8b0f19ba52fefafb335991732>@@$$QAV<lambda_207f2d024fc103971653565357d6cd41>@@@Z 100264a0     libucrt:per_thread_data.obj
 0002:000094c0       __sehtable$??$?RV<lambda_a7e850c220f1c8d1e6efeecdedd162c6>@@AAV<lambda_46720907175c18b6c9d2717bc0d2d362>@@V<lambda_9048902d66e8d99359bc9897bbb930a8>@@@?$__crt_seh_guarded_call@X@@QAEX$$QAV<lambda_a7e850c220f1c8d1e6efeecdedd162c6>@@AAV<lambda_46720907175c18b6c9d2717bc0d2d362>@@$$QAV<lambda_9048902d66e8d99359bc9897bbb930a8>@@@Z 100264c0     libucrt:per_thread_data.obj
 0002:000094e0       __sehtable$??$?RV<lambda_38edbb1296d33220d7e4dd0ed76b244a>@@AAV<lambda_5ce1d447e08cb34b2473517608e21441>@@V<lambda_fb385d3da700c9147fc39e65dd577a8c>@@@?$__crt_seh_guarded_call@X@@QAEX$$QAV<lambda_38edbb1296d33220d7e4dd0ed76b244a>@@AAV<lambda_5ce1d447e08cb34b2473517608e21441>@@$$QAV<lambda_fb385d3da700c9147fc39e65dd577a8c>@@@Z 100264e0     libucrt:per_thread_data.obj
 0002:00009500       __sehtable$??$?RV<lambda_6affb1475c98b40b75cdec977db92e3c>@@AAV<lambda_b8d4b9c228a6ecc3f80208dbb4b4a104>@@V<lambda_608742c3c92a14382c1684fc64f96c88>@@@?$__crt_seh_guarded_call@X@@QAEX$$QAV<lambda_6affb1475c98b40b75cdec977db92e3c>@@AAV<lambda_b8d4b9c228a6ecc3f80208dbb4b4a104>@@$$QAV<lambda_608742c3c92a14382c1684fc64f96c88>@@@Z 10026500     libucrt:per_thread_data.obj
 0002:00009520       __sehtable$??$?RV<lambda_e5124f882df8998aaf41531e079ba474>@@AAV<lambda_3e16ef9562a7dcce91392c22ab16ea36>@@V<lambda_e25ca0880e6ef98be67edffd8c599615>@@@?$__crt_seh_guarded_call@X@@QAEX$$QAV<lambda_e5124f882df8998aaf41531e079ba474>@@AAV<lambda_3e16ef9562a7dcce91392c22ab16ea36>@@$$QAV<lambda_e25ca0880e6ef98be67edffd8c599615>@@@Z 10026520     libucrt:wsetlocale.obj
 0002:00009540       __sehtable$??$?RV<lambda_d422a76eb4c3bf3ad751449ab71a6ea4>@@AAV<lambda_c9ba49e555ba839a7b07aa3fbecb7617>@@V<lambda_9476263c8ee91a25d21c55370bdb50de>@@@?$__crt_seh_guarded_call@H@@QAEH$$QAV<lambda_d422a76eb4c3bf3ad751449ab71a6ea4>@@AAV<lambda_c9ba49e555ba839a7b07aa3fbecb7617>@@$$QAV<lambda_9476263c8ee91a25d21c55370bdb50de>@@@Z 10026540     libucrt:close.obj
 0002:00009560       __sehtable$?__acrt_stdio_allocate_stream@@YA?AV__crt_stdio_stream@@XZ 10026560     libucrt:stream.obj
 0002:00009580       __sehtable$?update_thread_multibyte_data_internal@@YAPAU__crt_multibyte_data@@QAU__acrt_ptd@@QAPAU1@@Z 10026580     libucrt:mbctype.obj
 0002:000095a0       __sehtable$??$?RV<lambda_ceb1ee4838e85a9d631eb091e2fbe199>@@AAV<lambda_ae742caa10f662c28703da3d2ea5e57e>@@V<lambda_cd08b5d6af4937fe54fc07d0c9bf6b37>@@@?$__crt_seh_guarded_call@X@@QAEX$$QAV<lambda_ceb1ee4838e85a9d631eb091e2fbe199>@@AAV<lambda_ae742caa10f662c28703da3d2ea5e57e>@@$$QAV<lambda_cd08b5d6af4937fe54fc07d0c9bf6b37>@@@Z 100265a0     libucrt:mbctype.obj
 0002:000095c0       __sehtable$_raise          100265c0     libucrt:signal.obj
 0002:000095e0       __sehtable$??$?RV<lambda_cbab9ec6f41b0180b23cc171c22676b0>@@AAV<lambda_44731a7d0e6d81c3e6aa82d741081786>@@V<lambda_4b292cb8dd18144e164572427af410ab>@@@?$__crt_seh_guarded_call@P6AXH@Z@@QAEP6AXH@Z$$QAV<lambda_cbab9ec6f41b0180b23cc171c22676b0>@@AAV<lambda_44731a7d0e6d81c3e6aa82d741081786>@@$$QAV<lambda_4b292cb8dd18144e164572427af410ab>@@@Z 100265e0     libucrt:signal.obj
 0002:00009600       __sehtable$??$?RV<lambda_9e9de3de5fa147e2223d7db92bc10aa6>@@AAV<lambda_38ce7e780aa69e748d6df282ebc68efe>@@V<lambda_8ca6da459f0f6780f1cff60fdc3d00e5>@@@?$__crt_seh_guarded_call@H@@QAEH$$QAV<lambda_9e9de3de5fa147e2223d7db92bc10aa6>@@AAV<lambda_38ce7e780aa69e748d6df282ebc68efe>@@$$QAV<lambda_8ca6da459f0f6780f1cff60fdc3d00e5>@@@Z 10026600     libucrt:commit.obj
 0002:00009620       __sehtable$__write_internal 10026620     libucrt:write.obj
 0002:00009640       __sehtable$__alloc_osfhnd  10026640     libucrt:osfinfo.obj
 0002:00009660       __sehtable$___acrt_lowio_ensure_fh_exists 10026660     libucrt:osfinfo.obj
 0002:00009680       __sehtable$___acrt_update_thread_locale_data 10026680     libucrt:locale_refcounting.obj
 0002:000096a0       __sehtable$??$common_sopen_dispatch@D@@YAHQBDHHHQAHH@Z 100266a0     libucrt:open.obj
 0002:000096c0       __sehtable$??$common_lseek@_J@@YA_JH_JHAAV__crt_cached_ptd_host@@@Z 100266c0     libucrt:lseek.obj
 0002:000096e0       __sehtable$___set_fpsr_sse2 100266e0     libucrt:fpctrl.obj
 0002:00009700       __sehtable$__IsNonwritableInCurrentImage 10026700     LIBCMT:pesect.obj
 0002:00009720       .edata                     10026720     windowsaccessbridge-32.exp
 0002:00009748       rgpv                       10026748     windowsaccessbridge-32.exp
 0002:000098dc       rgszName                   100268dc     windowsaccessbridge-32.exp
 0002:00009a70       rgwOrd                     10026a70     windowsaccessbridge-32.exp
 0002:00009b3a       szName                     10026b3a     windowsaccessbridge-32.exp
 0002:00009b55       $N00001                    10026b55     windowsaccessbridge-32.exp
 0002:00009b77       $N00002                    10026b77     windowsaccessbridge-32.exp
 0002:00009b90       $N00003                    10026b90     windowsaccessbridge-32.exp
 0002:00009bb5       $N00004                    10026bb5     windowsaccessbridge-32.exp
 0002:00009bd1       $N00005                    10026bd1     windowsaccessbridge-32.exp
 0002:00009bdd       $N00006                    10026bdd     windowsaccessbridge-32.exp
 0002:00009bf9       $N00007                    10026bf9     windowsaccessbridge-32.exp
 0002:00009c1b       $N00008                    10026c1b     windowsaccessbridge-32.exp
 0002:00009c3f       $N00009                    10026c3f     windowsaccessbridge-32.exp
 0002:00009c53       $N00010                    10026c53     windowsaccessbridge-32.exp
 0002:00009c68       $N00011                    10026c68     windowsaccessbridge-32.exp
 0002:00009c86       $N00012                    10026c86     windowsaccessbridge-32.exp
 0002:00009c9d       $N00013                    10026c9d     windowsaccessbridge-32.exp
 0002:00009cba       $N00014                    10026cba     windowsaccessbridge-32.exp
 0002:00009cd3       $N00015                    10026cd3     windowsaccessbridge-32.exp
 0002:00009cf1       $N00016                    10026cf1     windowsaccessbridge-32.exp
 0002:00009d08       $N00017                    10026d08     windowsaccessbridge-32.exp
 0002:00009d24       $N00018                    10026d24     windowsaccessbridge-32.exp
 0002:00009d3b       $N00019                    10026d3b     windowsaccessbridge-32.exp
 0002:00009d55       $N00020                    10026d55     windowsaccessbridge-32.exp
 0002:00009d75       $N00021                    10026d75     windowsaccessbridge-32.exp
 0002:00009d88       $N00022                    10026d88     windowsaccessbridge-32.exp
 0002:00009da1       $N00023                    10026da1     windowsaccessbridge-32.exp
 0002:00009dc0       $N00024                    10026dc0     windowsaccessbridge-32.exp
 0002:00009dd9       $N00025                    10026dd9     windowsaccessbridge-32.exp
 0002:00009e00       $N00026                    10026e00     windowsaccessbridge-32.exp
 0002:00009e22       $N00027                    10026e22     windowsaccessbridge-32.exp
 0002:00009e3d       $N00028                    10026e3d     windowsaccessbridge-32.exp
 0002:00009e56       $N00029                    10026e56     windowsaccessbridge-32.exp
 0002:00009e7a       $N00030                    10026e7a     windowsaccessbridge-32.exp
 0002:00009e99       $N00031                    10026e99     windowsaccessbridge-32.exp
 0002:00009ec0       $N00032                    10026ec0     windowsaccessbridge-32.exp
 0002:00009ee3       $N00033                    10026ee3     windowsaccessbridge-32.exp
 0002:00009efb       $N00034                    10026efb     windowsaccessbridge-32.exp
 0002:00009f12       $N00035                    10026f12     windowsaccessbridge-32.exp
 0002:00009f28       $N00036                    10026f28     windowsaccessbridge-32.exp
 0002:00009f49       $N00037                    10026f49     windowsaccessbridge-32.exp
 0002:00009f65       $N00038                    10026f65     windowsaccessbridge-32.exp
 0002:00009f89       $N00039                    10026f89     windowsaccessbridge-32.exp
 0002:00009fa9       $N00040                    10026fa9     windowsaccessbridge-32.exp
 0002:00009fc5       $N00041                    10026fc5     windowsaccessbridge-32.exp
 0002:00009fdb       $N00042                    10026fdb     windowsaccessbridge-32.exp
 0002:00009ff2       $N00043                    10026ff2     windowsaccessbridge-32.exp
 0002:0000a00e       $N00044                    1002700e     windowsaccessbridge-32.exp
 0002:0000a025       $N00045                    10027025     windowsaccessbridge-32.exp
 0002:0000a03b       $N00046                    1002703b     windowsaccessbridge-32.exp
 0002:0000a05a       $N00047                    1002705a     windowsaccessbridge-32.exp
 0002:0000a06e       $N00048                    1002706e     windowsaccessbridge-32.exp
 0002:0000a07f       $N00049                    1002707f     windowsaccessbridge-32.exp
 0002:0000a0a4       $N00050                    100270a4     windowsaccessbridge-32.exp
 0002:0000a0b5       $N00051                    100270b5     windowsaccessbridge-32.exp
 0002:0000a0d2       $N00052                    100270d2     windowsaccessbridge-32.exp
 0002:0000a0f7       $N00053                    100270f7     windowsaccessbridge-32.exp
 0002:0000a11c       $N00054                    1002711c     windowsaccessbridge-32.exp
 0002:0000a12b       $N00055                    1002712b     windowsaccessbridge-32.exp
 0002:0000a13d       $N00056                    1002713d     windowsaccessbridge-32.exp
 0002:0000a157       $N00057                    10027157     windowsaccessbridge-32.exp
 0002:0000a170       $N00058                    10027170     windowsaccessbridge-32.exp
 0002:0000a182       $N00059                    10027182     windowsaccessbridge-32.exp
 0002:0000a191       $N00060                    10027191     windowsaccessbridge-32.exp
 0002:0000a1aa       $N00061                    100271aa     windowsaccessbridge-32.exp
 0002:0000a1bd       $N00062                    100271bd     windowsaccessbridge-32.exp
 0002:0000a1d5       $N00063                    100271d5     windowsaccessbridge-32.exp
 0002:0000a1fa       $N00064                    100271fa     windowsaccessbridge-32.exp
 0002:0000a21a       $N00065                    1002721a     windowsaccessbridge-32.exp
 0002:0000a237       $N00066                    10027237     windowsaccessbridge-32.exp
 0002:0000a244       $N00067                    10027244     windowsaccessbridge-32.exp
 0002:0000a251       $N00068                    10027251     windowsaccessbridge-32.exp
 0002:0000a263       $N00069                    10027263     windowsaccessbridge-32.exp
 0002:0000a288       $N00070                    10027288     windowsaccessbridge-32.exp
 0002:0000a295       $N00071                    10027295     windowsaccessbridge-32.exp
 0002:0000a2bd       $N00072                    100272bd     windowsaccessbridge-32.exp
 0002:0000a2cd       $N00073                    100272cd     windowsaccessbridge-32.exp
 0002:0000a2de       $N00074                    100272de     windowsaccessbridge-32.exp
 0002:0000a2ef       $N00075                    100272ef     windowsaccessbridge-32.exp
 0002:0000a300       $N00076                    10027300     windowsaccessbridge-32.exp
 0002:0000a30f       $N00077                    1002730f     windowsaccessbridge-32.exp
 0002:0000a321       $N00078                    10027321     windowsaccessbridge-32.exp
 0002:0000a333       $N00079                    10027333     windowsaccessbridge-32.exp
 0002:0000a347       $N00080                    10027347     windowsaccessbridge-32.exp
 0002:0000a359       $N00081                    10027359     windowsaccessbridge-32.exp
 0002:0000a36b       $N00082                    1002736b     windowsaccessbridge-32.exp
 0002:0000a37d       $N00083                    1002737d     windowsaccessbridge-32.exp
 0002:0000a38e       $N00084                    1002738e     windowsaccessbridge-32.exp
 0002:0000a3a0       $N00085                    100273a0     windowsaccessbridge-32.exp
 0002:0000a3b3       $N00086                    100273b3     windowsaccessbridge-32.exp
 0002:0000a3ca       $N00087                    100273ca     windowsaccessbridge-32.exp
 0002:0000a3ec       $N00088                    100273ec     windowsaccessbridge-32.exp
 0002:0000a40c       $N00089                    1002740c     windowsaccessbridge-32.exp
 0002:0000a430       $N00090                    10027430     windowsaccessbridge-32.exp
 0002:0000a449       $N00091                    10027449     windowsaccessbridge-32.exp
 0002:0000a45d       $N00092                    1002745d     windowsaccessbridge-32.exp
 0002:0000a476       $N00093                    10027476     windowsaccessbridge-32.exp
 0002:0000a495       $N00094                    10027495     windowsaccessbridge-32.exp
 0002:0000a4ad       $N00095                    100274ad     windowsaccessbridge-32.exp
 0002:0000a4ca       $N00096                    100274ca     windowsaccessbridge-32.exp
 0002:0000a4e3       $N00097                    100274e3     windowsaccessbridge-32.exp
 0002:0000a501       $N00098                    10027501     windowsaccessbridge-32.exp
 0002:0000a519       $N00099                    10027519     windowsaccessbridge-32.exp
 0002:0000a532       $N00100                    10027532     windowsaccessbridge-32.exp
 0002:0000a551       $N00101                    10027551     windowsaccessbridge-32.exp
 0002:0000a7b8       .idata$6                   100277b8     kernel32:KERNEL32.dll
 0002:0000a874       .idata$6                   10027874     user32:USER32.dll
 0003:00000030       ?__vcrt_flsindex@@3KA      10028030     libvcruntime:per_thread_data.obj
 0003:00000104       ?errno_no_memory@@3HA      10028104     libucrt:errno.obj
 0003:00000108       ?doserrno_no_memory@@3KA   10028108     libucrt:errno.obj
 0003:00000148       ?__acrt_flsindex@@3KA      10028148     libucrt:per_thread_data.obj
 0003:00000438       __mbctypes                 10028438     libucrt:mbctype.obj
 0003:00000540       __mbcasemaps               10028540     libucrt:mbctype.obj
 0003:00000640       ?__rgctypeflag@@3PADA      10028640     libucrt:mbctype.obj
 0003:00000648       ?__rgcode_page_info@@3PAUcode_page_info@@A 10028648     libucrt:mbctype.obj
 0003:000008a0       ?__dcrt_lowio_console_output_handle@@3PAXA 100288a0     libucrt:initcon.obj
 0003:000008b0       ?__DAZ_ENABLED@?1??__set_fpsr_sse2@@9@9 100288b0     libucrt:fpctrl.obj
 0003:00000970       _logFP                     10028970     AccessBridgeDebug.obj
 0003:000009a4       ?__proc_attached@@3HA      100289a4     LIBCMT:dll_dllmain.obj
 0003:000009a8       _GS_ExceptionRecord        100289a8     LIBCMT:gs_report.obj
 0003:000009f8       _GS_ContextRecord          100289f8     LIBCMT:gs_report.obj
 0003:00000ce0       ?is_initialized_as_dll@@3_NA 10028ce0     LIBCMT:utility.obj
 0003:00000ce1       ?module_local_atexit_table_initialized@@3_NA 10028ce1     LIBCMT:utility.obj
 0003:00000ce4       ?module_local_atexit_table@@3U_onexit_table_t@@A 10028ce4     LIBCMT:utility.obj
 0003:00000cf0       ?module_local_at_quick_exit_table@@3U_onexit_table_t@@A 10028cf0     LIBCMT:utility.obj
 0003:00000d30       ?heap@@3V_HeapManager@@A   10028d30     libvcruntime:undname.obj
 0003:00000d44       ?__vcrt_startup_thread_ptd@@3U__vcrt_ptd@@A 10028d44     libvcruntime:per_thread_data.obj
 0003:00000d6c       ___vcrt_lock_table         10028d6c     libvcruntime:locks.obj
 0003:00000d84       ___vcrt_locks_initialized  10028d84     libvcruntime:locks.obj
 0003:00000d88       ?module_handles@@3PAPAUHINSTANCE__@@A 10028d88     libvcruntime:winapi_downlevel.obj
 0003:00000d94       ?encoded_function_pointers@@3PAPAXA 10028d94     libvcruntime:winapi_downlevel.obj
 0003:00000dbc       ?__acrt_new_handler@@3V?$dual_state_global@P6AHI@Z@__crt_state_management@@A 10028dbc     libucrt:new_handler.obj
 0003:00000dc0       ?c_termination_complete@@3JA 10028dc0     libucrt:exit.obj
 0003:00000dc4       ?thread_local_exit_callback_func@@3P6GXPAXK0@ZA 10028dc4     libucrt:exit.obj
 0003:00000dc8       ?c_exit_complete@?1???R<lambda_6e4b09c48022b2350581041d5f6b0c4c>@@QBE@XZ@4_NA 10028dc8     libucrt:exit.obj
 0003:00000dd0       ?program_name@?1???$common_configure_argv@D@@YAHW4_crt_argv_mode@@@Z@4PADA 10028dd0     libucrt:argv_parsing.obj
 0003:00000f00       ?__acrt_invalid_parameter_handler@@3V?$dual_state_global@P6AXPB_W00II@Z@__crt_state_management@@A 10028f00     libucrt:invalid_parameter.obj
 0003:00000f08       ?module_handles@@3PAPAUHINSTANCE__@@A 10028f08     libucrt:winapi_thunks.obj
 0003:00000f60       ?encoded_function_pointers@@3PAPAXA 10028f60     libucrt:winapi_thunks.obj
 0003:000011f4       ?internal_state@?1??_mbtowc_internal@@9@4U_Mbstatet@@A 100291f4     libucrt:mbtowc.obj
 0003:000011fc       ?enable_percent_n@@3IA     100291fc     libucrt:printf_count_output.obj
 0003:00001210       ?__acrt_lock_table@@3PAU_RTL_CRITICAL_SECTION@@A 10029210     libucrt:locks.obj
 0003:00001360       ?__acrt_locks_initialized@@3IA 10029360     libucrt:locks.obj
 0003:00001370       ?fSystemSet@@3HA           10029370     libucrt:mbctype.obj
 0003:00001374       ?initialized@?1??__acrt_initialize_multibyte@@9@4_NA 10029374     libucrt:mbctype.obj
 0003:00001394       ?ctrlc_action@@3V?$dual_state_global@P6AXH@Z@__crt_state_management@@A 10029394     libucrt:signal.obj
 0003:00001398       ?ctrlbreak_action@@3V?$dual_state_global@P6AXH@Z@__crt_state_management@@A 10029398     libucrt:signal.obj
 0003:0000139c       ?abort_action@@3V?$dual_state_global@P6AXH@Z@__crt_state_management@@A 1002939c     libucrt:signal.obj
 0003:000013a0       ?term_action@@3V?$dual_state_global@P6AXH@Z@__crt_state_management@@A 100293a0     libucrt:signal.obj
 0003:000013a4       ?user_matherr@@3V?$dual_state_global@P6AHPAU_exception@@@Z@__crt_state_management@@A 100293a4     libucrt:matherr.obj
 0003:000013a8       ?__acrt_global_new_mode@@3V?$dual_state_global@J@__crt_state_management@@A 100293a8     libucrt:new_mode.obj
 0003:000013b8       ?__acrt_app_type@@3W4_crt_app_type@@A 100293b8     libucrt:report_runtime_error.obj
 0003:000013bc       ?internal_pst@?1??__mbrtoc32_utf8@__crt_mbstring@@YAIPA_UPBDIPAU_Mbstatet@@AAV__crt_cached_ptd_host@@@Z@4U3@A 100293bc     libucrt:mbrtoc32.obj
 0003:000013cc       __pmatherr_set             100293cc     libucrt:libm_error.obj
 0004:00000120       $R000000                   1002a120     windowsaccessbridge-32.dll.res
 0004:00000338       $R000218                   1002a338     windowsaccessbridge-32.dll.res
 0004:000003c8       $R0002A8                   1002a3c8     windowsaccessbridge-32.dll.res
